:100000000C9467030C9484030C945D5E0C9484033D
:100010000C9484030C9484030C9484030C94840344
:100020000C9484030C9402850C9484030C94840334
:100030000C9484030C9484030C9484030C94840324
:100040000C9484030C9484030C9484030C94840314
:100050000C9484030C9440A20C9484030C948403A9
:100060000C9484030C9484030C9484030C948403F4
:100070000C9484030C9484030C9484030C948403E4
:100080000C9484030C9484030C9484030C948403D4
:100090000C948403CE03C103B303A30390037A0338
:1000A0006103470329030803E602C2029E027602A7
:1000B0004F02280203026C01B80196017501560136
:1000C00039011F010601EF00DA00B5008200A5002A
:1000D0009600000043414E20310000000000000067
:1000E00000000043414E20320000000000000000EC
:1000F000000043414E2033000000000000000000DB
:100100000043414E203400000000000000000000C9
:1001100043414E2035000000000000000000004375
:10012000414E203600000000000000000000434166
:100130004E20370000000000000000000043414E48
:1001400020380000000000000000000043414E2065
:10015000390000000000000000000043414E203143
:100160003000000000000000000043414E2031310B
:1001700000000000000000000043414E203132002A
:10018000000000000000000043414E203133000019
:100190000000000000000043414E20313400000008
:1001A00000000000000043414E20313500000000F7
:1001B000000000000043414E2031360000000000E6
:1001C0000000000043414E203137000000000000D5
:1001D00000000043414E20313800000000000000C4
:1001E000000043414E2031390000000000000000B3
:1001F0000043414E203230000000000000000000AB
:1002000043414E2032310000000000000000004356
:10021000414E203232000000000000000000434147
:100220004E20323300000000000000000043414E29
:1002300020323400000000000000000043414E2046
:10024000323500000000000000000043414E203223
:100250003600000000000000000043414E2032370D
:1002600000000000000000000043414E2032380032
:10027000000000000000000043414E203239000021
:100280000000000000000043414E20333000000019
:1002900000000000000043414E2033310000000008
:1002A000000000000043414E2033320000000000F7
:1002B00000000000466C61736820310000000000FF
:1002C000000000466C6173682032000000000000EE
:1002D0000000466C617368203300000000000000DD
:1002E00000466C61736820340000000000000000CC
:1002F000466C617368203500000000000000005368
:100300005749544348203100000000000000535773
:100310004954434820320000000000000053574970
:100320005443482033000000000000005357495454
:100330004348203400000000000000535749544354
:10034000482035000000000000005357495443483E
:100350002036000000000000005357495443482055
:10036000370000000000000053574954434820382C
:100370000000000000000053574954434820390052
:10038000000000000000535749544348203130001A
:100390000000000000535749544348203131000009
:1003A000000000004348414E4E454C203100000003
:1003B0000000004348414E4E454C203200000000F2
:1003C00000004348414E4E454C20330000000000E1
:1003D000004348414E4E454C2034000000000000D0
:1003E0004348414E4E454C2035000000000000437C
:1003F00048414E4E454C2036000000000000434866
:10040000414E4E454C20370000000000004348415B
:100410004E4E454C20380000000000004348414E3D
:100420004E454C20390000000000004348414E4E2C
:10043000454C20313000000000004348414E4E45FD
:100440004C20313100000000004348414E4E454CE5
:1004500020313200000000004348414E4E454C2000
:10046000313300000000004348414E4E454C2031DE
:100470003400000000004348414E4E454C203135C9
:1004800000000000004348414E4E454C20313600EC
:10049000000000004348414E4E454C2031370000DB
:1004A0000000004348414E4E454C203138000000CA
:1004B00000004348414E4E454C20313900000000B9
:1004C000004348414E4E454C2032300000000000B1
:1004D0004348414E4E454C2032310000000000435D
:1004E00048414E4E454C2032320000000000434847
:1004F000414E4E454C20323300000000004348413D
:100500004E4E454C20323400000000004348414E1E
:100510004E454C20323500000000004348414E4E0D
:10052000454C20323600000000004348414E4E4505
:100530004C20323700000000004348414E4E454CED
:1005400020323800000000004348414E4E454C2008
:10055000323900000000004348414E4E454C2033E4
:100560003000000000004348414E4E454C203331DE
:1005700000000000004348414E4E454C20333200FD
:10058000000000004348414E4E454C2033330000EC
:100590000000004348414E4E454C203334000000DB
:1005A00000005649525455414C20310000000000D3
:1005B000005649525455414C2032000000000000C2
:1005C0005649525455414C2033000000000000565B
:1005D00049525455414C2034000000000000564957
:1005E000525455414C20350000000000005649523D
:1005F0005455414C2036000000000000564952542A
:1006000055414C2037000000000000564952545517
:10061000414C20380000000000005649525455411A
:100620004C20390000000000005649525455414CFE
:1006300020313000000000005649525455414C20F2
:10064000313100000000005649525455414C2031D0
:100650003200000000005649525455414C203133BD
:1006600000000000005649525455414C20313400DE
:10067000000000005649525455414C2031350000CD
:100680000000005649525455414C203136000000BC
:1006900000005649525455414C20313700000000AB
:1006A000005649525455414C20313800000000009A
:1006B0005649525455414C20313900000000005633
:1006C00049525455414C20323000000000001124A2
:1006D0001FBECFEFD0E1DEBFCDBF11E0A0E0B1E0A3
:1006E000EAEBFBE701E00BBF02C007900D92A43BD1
:1006F000B107D9F71FE0A4EBB1E001C01D92AF3103
:10070000B107E1F70C94B7710C940000CF93DF931D
:10071000CDB7DEB729970FB6F894DEBF0FBECDBFB9
:100720008983898187708A8389819927887F9070DE
:100730009595879595958795959587958B838A81CE
:10074000282F332739872887888599858330910515
:1007500009F45EC0288539852430310584F4888504
:10076000998581309105A1F128853985223031059F
:100770000CF03EC0888599850097D1F098C02885F7
:1007800039852530310509F463C088859985853020
:1007900091050CF44DC0288539852630310509F4C2
:1007A00067C0888599858730910509F471C07FC03D
:1007B000809134008E7F80933400809134008D7F4F
:1007C00080933400809134008B7F809334006FC01D
:1007D00080913400816080933400809134008D7F5B
:1007E00080933400809134008B7F809334005FC00D
:1007F000809134008E7F8093340080913400826039
:1008000080933400809134008B7F809334004FC0FC
:100810008091340081608093340080913400826044
:1008200080933400809134008B7F809334003FC0EC
:10083000809134008E7F80933400809134008D7FCE
:1008400080933400809134008460809334002FC002
:1008500080913400816080933400809134008D7FDA
:1008600080933400809134008460809334001FC0F2
:10087000809134008E7F80933400809134008260B8
:1008800080933400809134008460809334000FC0E2
:1008900080913400816080933400809134008260C4
:1008A00080933400809134008460809334008B8185
:1008B000806280937C001D828D818A3F20F48D812F
:1008C0008F5F8D83F9CF80917A00806180937A0069
:1008D00080917A00806480937A0080917A009927D1
:1008E00080719070009709F4F8CF809178008D8323
:1008F000809179008C838C8199279C01220F331F72
:10090000220F331F8D818295869586958370992756
:10091000820F931F9F838E838E819F8129960FB6AE
:10092000F894DEBF0FBECDBFDF91CF910895CF9376
:10093000DF93CDB7DEB725970FB6F894DEBF0FBEB5
:10094000CDBF8983898187708A8389819927887F30
:1009500090709595879595958795959587958B83B7
:100960008A81282F33273D832C838C819D8183307E
:10097000910509F45EC02C813D812430310584F459
:100980008C819D8181309105A1F12C813D812230A6
:1009900031050CF03EC08C819D810097D1F098C04C
:1009A0002C813D812530310509F463C08C819D8106
:1009B000853091050CF44DC02C813D8126303105E8
:1009C00009F467C08C819D818730910509F471C05D
:1009D0007FC0809134008E7F8093340080913400FA
:1009E0008D7F80933400809134008B7F809334001E
:1009F0006FC0809134008160809334008091340016
:100A00008D7F80933400809134008B7F80933400FD
:100A10005FC0809134008E7F8093340080913400D9
:100A2000826080933400809134008B7F8093340007
:100A30004FC08091340081608093340080913400F5
:100A4000826080933400809134008B7F80933400E7
:100A50003FC0809134008E7F8093340080913400B9
:100A60008D7F8093340080913400846080933400C3
:100A70002FC08091340081608093340080913400D5
:100A80008D7F8093340080913400846080933400A3
:100A90001FC0809134008E7F809334008091340099
:100AA00082608093340080913400846080933400AD
:100AB0000FC08091340081608093340080913400B5
:100AC000826080933400809134008460809334008D
:100AD0008B81806280937C0080917A008064809317
:100AE0007A0080917A00992780719070009709F4BC
:100AF000F8CF80917A00806180937A0080917900AC
:100B0000992725960FB6F894DEBF0FBECDBFDF91B3
:100B1000CF910895CF93DF93CDB7DEB72A970FB665
:100B2000F894DEBF0FBECDBF9A8389837C836B832D
:100B30001E821D8289819A819C0102969A838983F3
:100B400038872F83EF81F885859194919A878987DB
:100B5000CF0198878F8329853A858B819C81821765
:100B6000930758F48D819E818639910534F48D81E7
:100B70009E8105969E838D83DDCF8D819E812A96F1
:100B80000FB6F894DEBF0FBECDBFDF91CF910895B1
:100B9000CF93DF93CDB7DEB722970FB6F894DEBFC1
:100BA0000FBECDBF9A838983809100018130C1F44B
:100BB0001092000189819A819093BD018093BC01BC
:100BC0009093BB018093BA019093B9018093B801CF
:100BD0009093B7018093B6019093B5018093B401CF
:100BE0008091BA019091BB019093BD018093BC01AB
:100BF0008091B8019091B9019093BB018093BA01A3
:100C00008091B6019091B7019093B9018093B8019A
:100C10008091B4019091B5019093B7018093B60192
:100C200089819A819093B5018093B4012091B40198
:100C30003091B5018091B6019091B701280F391F0D
:100C40008091B8019091B901280F391F8091BA01A4
:100C50009091BB01280F391F8091BC019091BD017B
:100C6000820F931F25E030E0B9010E942EBDCB0119
:100C70009A83898389819A8122960FB6F894DEBF80
:100C80000FBECDBFDF91CF910895CF93DF93CDB746
:100C9000DEB726970FB6F894DEBF0FBECDBF80E15A
:100CA0000E9486039E838D8384E990E09C838B83DE
:100CB0008D819E810E94C8059E838D836D817E817A
:100CC0008B819C810E948A059A83898389819927D7
:100CD00026960FB6F894DEBF0FBECDBFDF91CF9141
:100CE0000895CF93DF93CDB7DEB723970FB6F8946F
:100CF000DEBF0FBECDBF83E10E9497049B838A8332
:100D00008091C70D282F33278A819B81829FA00164
:100D1000839F500D929F500D1124CA019B838A839B
:100D20008A819B81880F892F881F990B91959B83BE
:100D30008A838A819B818F3F910521F018F08FEF84
:100D4000898302C08A8189838091BE01882341F40E
:100D500089818093C0018093BF018093BE0130C020
:100D60008091C001282F33278A819B81820F931F96
:100D70009B838A838091BF01282F33278A819B819F
:100D8000820F931F9B838A838091BE01282F332774
:100D90008A819B81820F931F9B838A838091BF01ED
:100DA0008093C0018091BE018093BF0189818093AF
:100DB000BE018A819B8196958795969587958983B3
:100DC0008981992723960FB6F894DEBF0FBECDBF59
:100DD000DF91CF910895CF93DF93CDB7DEB780E257
:100DE00080937C0087E880937A0080913300816053
:100DF0008093330080913300826080933300809130
:100E00003300846080933300809134008E7F809320
:100E10003400809134008D7F8093340080913400C1
:100E20008B7F80933400DF91CF910895CF93DF9330
:100E3000CDB7DEB722970FB6F894DEBF0FBECDBF99
:100E4000198289818F3038F589818295807F8093DE
:100E5000ED001092EE001092EF001092F000109250
:100E6000F1001092F2001092F3001092F400109230
:100E7000F5001092F6001092F7001A828A818830ED
:100E800030F41092FA008A818F5F8A83F7CF8981CC
:100E90008F5F8983D6CF22960FB6F894DEBF0FBE40
:100EA000CDBFDF91CF910895CF93DF93CDB7DEB75C
:100EB00024970FB6F894DEBF0FBECDBF8091ED0032
:100EC0008A83198289818F30B8F489818295807FE5
:100ED0008093ED0090EC8091EF008923882341F40A
:100EE0008A818093ED00898199279C838B830BC035
:100EF00089818F5F8983E6CF8A818093ED008FEFB0
:100F000090E09C838B838B819C8124960FB6F89410
:100F1000DEBF0FBECDBFDF91CF910895CF93DF939A
:100F2000CDB7DEB722970FB6F894DEBF0FBECDBFA8
:100F30008091EE00992780749070009719F01A82C2
:100F400019821BC08091EE009927807290700097E3
:100F500029F081E090E09A8389830FC080EC909122
:100F6000EF008923882329F48FEF90E09A83898307
:100F700004C082E090E09A83898389819A812296D5
:100F80000FB6F894DEBF0FBECDBFDF91CF910895AD
:100F9000CF93DF93CDB7DEB723970FB6F894DEBFBC
:100FA0000FBECDBF9A8389831B828B81282F332765
:100FB0008091EF0099278F709070281739077CF483
:100FC0008B81282F332789819A81F901E80FF91F36
:100FD0008091FA0080838B818F5F8B83E6CF23968D
:100FE0000FB6F894DEBF0FBECDBFDF91CF9108954D
:100FF000CF93DF93CDB7DEB78EEC9CE00E94836C7D
:1010000064E77DE080E00E94246D6CE27DE081E099
:101010000E94246D66EE7CE082E00E94246D81E0F7
:101020008093C2018091CE0C813071F48091CF0CFD
:101030009091D00C2AE030E0B9010E942EBDCB0186
:101040009093CC0C8093CB0C8091750D813071F412
:101050008091760D9091770D2AE030E0B9010E94E1
:101060002EBDCB019093C70C8093C60C80912D0DA3
:10107000813071F480912E0D90912F0D2AE030E097
:10108000B9010E942EBDCB019093CA0C8093C90C6C
:101090008091E70C813071F48091E80C9091E90C1B
:1010A0002AE030E0B9010E942EBDCB019093730D70
:1010B0008093720DDF91CF910895CF93DF93CDB7D9
:1010C000DEB7CF55D0400FB6F894DEBF0FBECDBF10
:1010D00019828CE0888F84E690E09B838A831D824E
:1010E0001C821E821F82188619861A861B86FE01A4
:1010F000E15AFF4F1082FE01E15AFF4F80818C3090
:10110000B0F4FE01E15AFF4F8081282F3327CE0132
:101110000C96FC01E20FF31F1082DE01A15ABF4FB3
:10112000FE01E15AFF4F80818F5F8C93E4CFCE01A7
:1011300001960E94466CA895198E1A8E84E690E05E
:101140009C8F8B8F1E8E1D8EFE01E15AFF4F1082E9
:10115000FE01E15AFF4F80818232B8F4FE01E15A6C
:10116000FF4F8081282F3327CE010196820F931FD6
:10117000FC017E961082DE01A15ABF4FFE01E15AAA
:10118000FF4F80818F5F8C93E3CFCE0149960E9401
:10119000C06CA89581E0898F1A8E84E690E09C8FC0
:1011A0008B8F1E8E1D8EFE01E15AFF4F1082FE01B5
:1011B000E15AFF4F80818232B8F4FE01E15AFF4FBD
:1011C0008081282F3327CE010196820F931FFC01C7
:1011D0007E961082DE01A15ABF4FFE01E15AFF4FF9
:1011E00080818F5F8C93E3CFCE0149960E94C06CC3
:1011F000A89582E0898F1A8E84E690E09C8F8B8F71
:101200001E8E1D8EFE01E15AFF4F1082FE01E15A33
:10121000FF4F80818034B8F4FE01E15AFF4F808196
:10122000282F3327CE010196820F931FFC017E9653
:101230001082DE01A15ABF4FFE01E15AFF4F8081AB
:101240008F5F8C93E3CFCE0149960E94C06CC15A48
:10125000DF4F0FB6F894DEBF0FBECDBFDF91CF9149
:101260000895CF93DF93CDB7DEB725970FB6F894E7
:10127000DEBF0FBECDBF89838981282F33273D83F1
:101280002C838C819D818832910509F470C02C815A
:101290003D81293231051CF58C819D818532910576
:1012A00009F450C02C813D81263231055CF48C81DB
:1012B0009D8183329105C1F12C813D81243231051C
:1012C000D1F17FC08C819D818632910509F441C0A6
:1012D0002C813D812732310509F442C072C08C81D6
:1012E0009D818B32910509F457C02C813D812C32B0
:1012F00031056CF48C819D818932910509F43EC0E1
:101300002C813D812A32310509F43FC05AC08C81BD
:101310009D818C32910509F446C02C813D812D328E
:10132000310509F447C04DC080EC0E9456839927CF
:101330009B838A8348C081EC0E94568399279B83B4
:101340008A8341C082EC0E94568399279B838A83BB
:101350003AC081ED0E94568399279B838A8333C0CC
:1013600084EC0E94568399279B838A832CC085EC4A
:101370000E94568399279B838A8325C086EC0E940E
:10138000568399279B838A831EC087EC0E945683CD
:1013900099279B838A8317C083EC0E9456839927E1
:1013A0009B838A8310C082ED0E94568399279B837A
:1013B0008A8309C083ED0E94568399279B838A8381
:1013C00002C01B821A828A819B8125960FB6F894EF
:1013D000DEBF0FBECDBFDF91CF910895CF93DF93D6
:1013E000CDB7DEB7A8970FB6F894DEBF0FBECDBF5E
:1013F0008091C40D9091C50D009709F49AC6809113
:10140000C40D9091C50D28E08030920708F091C678
:101410008091C30D882309F48CC68091C80C8F5F1E
:101420008093C80C9091C30D8091C80C891708F463
:1014300080C61092C80C88E08F83188A888988300B
:1014400070F48889282F3327CE010196820F931FCD
:10145000FC013796108288898F5F888BEFCF80914F
:10146000CD0C482F552758A74FA38FA198A586309C
:10147000910509F415C42FA138A5273031052CF5A5
:101480004FA158A54330510509F4FDC28FA198A57D
:10149000843091056CF42FA138A52130310509F471
:1014A00040C24FA158A54230510509F493C237C03C
:1014B0008FA198A58430910509F46CC32FA138A59C
:1014C0002530310509F4A8C32AC04FA158A54930D9
:1014D000510509F4D5C48FA198A58A3091056CF403
:1014E0002FA138A52730310509F41EC44FA158A5F6
:1014F0004830510509F486C412C08FA198A58B30DD
:10150000910509F437C52FA138A52B3031050CF40E
:1015100005C54FA158A54C30510509F4CAC58091A5
:10152000C40D9091C50DAA27BB278B839C83AD83E7
:10153000BE8381E08093CD0C1B8A80EC0E94568391
:10154000882319F08B8981608B8B81EC0E945683F4
:10155000882319F08B8982608B8B82EC0E945683E2
:10156000882319F08B8984608B8B81ED0E945683D0
:10157000882319F08B8988608B8B84EC0E945683BA
:10158000882319F08B8980618B8B85EC0E945683B0
:10159000882319F08B8980628B8B86EC0E9456839E
:1015A000882319F08B8980648B8B87EC0E9456838B
:1015B000882319F08B8980688B8B8B8988871B8A9D
:1015C00083EC0E945683882319F08B8981608B8B72
:1015D00082ED0E945683882319F08B8982608B8B61
:1015E00083ED0E945683882319F08B8984608B8B4E
:1015F0008B8989871B8A81E00E94F3A8882319F0D0
:101600008B8981608B8B82E00E94F3A8882319F07C
:101610008B8982608B8B83E00E94F3A8882319F06A
:101620008B8984608B8B84E00E94F3A8882319F057
:101630008B8988608B8B85E00E94F3A8882319F042
:101640008B8980618B8B86E00E94F3A8882319F038
:101650008B8980628B8B87E00E94F3A8882319F026
:101660008B8980648B8B88E00E94F3A8882319F013
:101670008B8980688B8B8B898A871B8A89E00E9483
:10168000F3A8882319F08B8981608B8B8AE00E94F4
:10169000F3A8882319F08B8982608B8B8BE00E94E2
:1016A000F3A8882319F08B8984608B8B8CE00E94CF
:1016B000F3A8882319F08B8988608B8B8DE00E94BA
:1016C000F3A8882319F08B8980618B8B8EE00E94B0
:1016D000F3A8882319F08B8980628B8B8FE00E949E
:1016E000F3A8882319F08B8980648B8B80E10E949A
:1016F000F3A8882319F08B8980688B8B8B898B8763
:101700001B8A81E00E94571A882319F08B89816017
:101710008B8B82E00E94571A882319F08B89826094
:101720008B8B83E00E94571A882319F08B89846081
:101730008B8B84E00E94571A882319F08B8988606C
:101740008B8B85E00E94571A882319F08B89806162
:101750008B8B86E00E94571A882319F08B89806250
:101760008B8B87E00E94571A882319F08B8980643D
:101770008B8B88E00E94571A882319F08B89806828
:101780008B8B8B898C871B8A89E00E94571A882350
:1017900019F08B8981608B8B8AE00E94571A88230D
:1017A00019F08B8982608B8B8BE00E94571A8823FB
:1017B00019F08B8984608B8B8CE00E94571A8823E8
:1017C00019F08B8988608B8B8DE00E94571A8823D3
:1017D00019F08B8980618B8B8EE00E94571A8823C9
:1017E00019F08B8980628B8B8FE00E94571A8823B7
:1017F00019F08B8980648B8B80E10E94571A8823B3
:1018000019F08B8980688B8B8B898D871B8A81E18E
:101810000E94571A882319F08B8981608B8B82E193
:101820000E94571A882319F08B8982608B8B83E181
:101830000E94571A882319F08B8984608B8B84E16E
:101840000E94571A882319F08B8988608B8B85E159
:101850000E94571A882319F08B8980618B8B86E14F
:101860000E94571A882319F08B8980628B8B87E13D
:101870000E94571A882319F08B8980648B8B88E12A
:101880000E94571A882319F08B8980688B8B8B896B
:101890008E871B8A89E10E94571A882319F08B8949
:1018A00081608B8B8AE10E94571A882319F08B89FB
:1018B00082608B8B8BE10E94571A882319F08B89E9
:1018C00084608B8B8CE10E94571A882319F08B89D6
:1018D00088608B8B8DE10E94571A882319F08B89C1
:1018E00080618B8B8EE10E94571A882319F08B89B7
:1018F00080628B8B8FE10E94571A882319F08B89A5
:1019000080648B8B80E20E94571A882319F08B89A0
:1019100080688B8B8B898F87CE0103960E94207FF6
:1019200008C48091C40D9091C50D0196AA27BB27CC
:101930008B839C83AD83BE8382E08093CD0C188A19
:101940008889883008F041C088898F5F0E948B5A4F
:101950009D8F8C8FEC8DFD8D878599278170907080
:10196000009719F084E68B8B21C0EC8DFD8D878567
:10197000992788709070009719F085E68B8B16C0B8
:10198000EC8DFD8D8785992780749070009719F0F4
:1019900086E68B8B0BC0EC8DFD8D90EF81818923CA
:1019A000882319F081E08B8B01C01B8A8889282F3E
:1019B0003327CE010196820F931FFC0137968B8946
:1019C000808388898F5F888BBBCFCE0103960E946E
:1019D000207FAFC38091C40D9091C50D0296AA27B8
:1019E000BB278B839C83AD83BE8383E08093CD0C28
:1019F000188A8889883008F041C08889875F0E94EA
:101A00008B5A9D8F8C8FEC8DFD8D878599278170EA
:101A10009070009719F084E68B8B21C0EC8DFD8DC2
:101A20008785992788709070009719F085E68B8BD1
:101A300016C0EC8DFD8D8785992780749070009776
:101A400019F086E68B8B0BC0EC8DFD8D90EF8181BC
:101A50008923882319F081E08B8B01C01B8A888938
:101A6000282F3327CE010196820F931FFC01379652
:101A70008B89808388898F5F888BBBCFCE0103964B
:101A80000E94207F56C38091C40D9091C50D03968E
:101A9000AA27BB278B839C83AD83BE8384E080937E
:101AA000CD0C188A8889823008F041C088898F5E01
:101AB0000E948B5A9D8F8C8FEC8DFD8D8785992789
:101AC00081709070009719F084E68B8B21C0EC8DAB
:101AD000FD8D8785992788709070009719F085E6AD
:101AE0008B8B16C0EC8DFD8D878599278074907047
:101AF000009719F086E68B8B0BC0EC8DFD8D90EF77
:101B000081818923882319F081E08B8B01C01B8A96
:101B10008889282F3327CE010196820F931FFC015D
:101B200037968B89808388898F5F888BBBCF888924
:101B3000883058F588898F5E0E948B5A9D8F8C8FD4
:101B4000EC8DFD8D8785992781709070009719F035
:101B500084E68B8B0BC0EC8DFD8D90EF818189230A
:101B6000882319F081E08B8B01C01B8A8889282F7C
:101B70003327CE010196820F931FFC0137968B8984
:101B8000808388898F5F888BD2CFCE0103960E9495
:101B9000207FCFC28091C40D9091C50D0496AA27D5
:101BA000BB278B839C83AD83BE8385E08093CD0C64
:101BB000188A8889883058F58889875E0E948B5AF0
:101BC0009D8F8C8FEC8DFD8D87859927817090700E
:101BD000009719F084E68B8B0BC0EC8DFD8D90EF98
:101BE00081818923882319F081E08B8B01C01B8AB6
:101BF0008889282F3327CE010196820F931FFC017D
:101C000037968B89808388898F5F888BD2CFCE016E
:101C100003960E94207F8DC28091C40D9091C50DC6
:101C20000596AA27BB278B839C83AD83BE8386E062
:101C30008093CD0C188A8889883068F588898F5FF1
:101C40000E948B5A9D8F8C8FEC8DFD8D90EF818142
:101C50008923882391F08889282F3327CE01019684
:101C6000820F931FDC011796EC8DFD8D8089918981
:101C70000196969587958C930AC08889282F3327DB
:101C8000CE010196820F931FFC013796108288893E
:101C90008F5F888BD0CFCE0103960E94207F49C2F0
:101CA0008091C40D9091C50D0696AA27BB278B8302
:101CB0009C83AD83BE8387E08093CD0C188A88898E
:101CC000883068F58889875F0E948B5A9D8F8C8F3A
:101CD000EC8DFD8D90EF81818923882391F0888997
:101CE000282F3327CE010196820F931FDC01179610
:101CF000EC8DFD8D808991890196969587958C93C1
:101D00000AC08889282F3327CE010196820F931F9E
:101D1000FC013796108288898F5F888BD0CFCE01E7
:101D200003960E94207F05C28091C40D9091C50D3D
:101D30000796AA27BB278B839C83AD83BE8388E04D
:101D40008093CD0C188A8889823068F588898F5EE7
:101D50000E948B5A9D8F8C8FEC8DFD8D90EF818131
:101D60008923882391F08889282F3327CE01019673
:101D7000820F931FDC011796EC8DFD8D8089918970
:101D80000196969587958C930AC08889282F3327CA
:101D9000CE010196820F931FFC013796108288892D
:101DA0008F5F888BD0CF8889883038F588898F5E9F
:101DB0000E948B5A9D8F8C8FEC8DFD8D90EF8181D1
:101DC0008923882361F08889282F3327CE01019643
:101DD000820F931FFC0137968FE080830AC08889A9
:101DE000282F3327CE010196820F931FFC013796CF
:101DF000108288898F5F888BD6CFCE0103960E9490
:101E0000207F97C18091C40D9091C50D0896AA2797
:101E1000BB278B839C83AD83BE8389E08093CD0CED
:101E2000188A8889883038F58889875E0E948B5A9D
:101E30009D8F8C8FEC8DFD8D90EF81818923882380
:101E400061F08889282F3327CE010196820F931FD6
:101E5000FC0137968FE080830AC08889282F3327BA
:101E6000CE010196820F931FFC013796108288895C
:101E70008F5F888BD6CFCE0103960E94207F59C1F9
:101E80008091C40D9091C50D0996AA27BB278B831D
:101E90009C83AD83BE838AE08093CD0CCE014496B3
:101EA0000E94505A8E8999279A83898329813A8181
:101EB000C901880F991F880F991F880F991F820FDA
:101EC000931F820F931F9A83898389819A81892F17
:101ED00099278887898189878F8999279A83898318
:101EE00029813A8184E690E0289FA001299F500D26
:101EF000389F500D1124CA019A83898389819A8160
:101F0000892F99278A8789818B871C861D861E8643
:101F10001F86CE0103960E94207F0BC18091C40DC5
:101F20009091C50D0A96AA27BB278B839C83AD830E
:101F3000BE838BE08093CD0CCE0144960E94505A14
:101F4000188619861A861B868C899D890196969516
:101F500087959A83898389819A81892F99278C878C
:101F600089818D8781E08E871F86CE0103960E942E
:101F7000207FDFC08091C40D9091C50D0B96AA27DC
:101F8000BB278B839C83AD83BE838091C101882353
:101F900041F08091C10181508093C1011092CD0C1C
:101FA00006C08AE08093C1018CE08093CD0C1B8A2F
:101FB00081E10E94F3A8882319F08B8981608B8BC3
:101FC00082E10E94F3A8882319F08B8982608B8BB1
:101FD00083E10E94F3A8882319F08B8984608B8B9E
:101FE00084E10E94F3A8882319F08B8988608B8B89
:101FF0008B89888781E20E948B5A9D8F8C8FEC8D14
:10200000FD8D8785992781709070009719F084E67F
:102010008B8B14C0EC8DFD8D87859927887090700F
:10202000009719F085E68B8B09C0EC8DFD8D8181C1
:10203000803F19F481E08B8B01C01B8A8B898987D3
:102040008B89813019F48FE08B8701C01B8682E277
:102050000E948B5A9D8F8C8FEC8DFD8D87859927E3
:1020600081709070009719F084E68B8B14C0EC8D12
:10207000FD8D8785992788709070009719F085E607
:102080008B8B09C0EC8DFD8D8181803F19F481E03F
:102090008B8B01C01B8A8B898A878B89813019F4CD
:1020A0008FE08C8701C01C86CE0103960E94207FA2
:1020B00040C08091C40D9091C50D0C96AA27BB27F6
:1020C0008B839C83AD83BE831092CD0C8091800165
:1020D0008887809181018987CE01039607969F8F1B
:1020E0008E8F86E090E099A388A382E090E09BA386
:1020F0008AA38AA19BA19DA38CA38CA19DA1A8A129
:10210000B9A1EE8DFF8D019724F00E94C9BD019207
:10211000FACF9DA38CA3CD0199A388A3CF019F8F54
:102120008E8F1C861D861E861F86CE0103960E94FA
:10213000207F8091CB0C9091CC0C009709F498C033
:102140008091CB0C9091CC0C01979093CC0C809308
:10215000CB0C8091CB0C9091CC0C009709F088C0EF
:102160008091CF0C9091D00C2AE030E0B9010E9410
:102170002EBDCB019093CC0C8093CB0C8091D10CD5
:102180009091D20CAA27BB278B839C83AD83BE83FF
:1021900088E08F838091C20188878091D30C0E9450
:1021A000985B9A83898389819A8101969695879510
:1021B00089878091D40C0E94985B9A838983898156
:1021C0009A810196969587958A878091D50C0E9471
:1021D000985B9A83898389819A81019696958795E0
:1021E0008B878091D60C0E94985B9A838983898122
:1021F0009A810196969587958C878091D70C0E943D
:10220000985B9A83898389819A81019696958795AF
:102210008D878091D80C0E94985B9A8389838981ED
:102220009A810196969587958E878091C20199270C
:10223000FC01E852F34F80810E94985B9A83898366
:1022400089819A810196969587958F878091C201A1
:102250008F5F8093C2019091E50C8091C201981725
:1022600018F481E08093C201CE0103960E94207F82
:102270008091C60C9091C70C009709F48EC1809193
:10228000C60C9091C70C01979093C70C8093C60C15
:102290008091C60C9091C70C009709F07EC1CE01C9
:1022A00044960E94505A8091760D9091770D2AE0C5
:1022B00030E0B9010E942EBDCB019093C70C8093F2
:1022C000C60C8091780D9091790DAA27BB278B833E
:1022D0009C83AD83BE8388E08F831A8A80E8898BD4
:1022E000188A88898830B0F588899927FC01E658D2
:1022F000F24F80818B8B8B89833250F48B890E94C3
:102300009D59882301F18A899989892B8A8B1BC061
:102310008B898E3250F48B890E943109882399F081
:102320008A899989892B8A8B0EC08B898E3259F4C0
:1023300080913400992780719070009721F08A89EC
:102340009989892B8A8B89898695898B88898F5F62
:10235000888BC7CF8A8988871A8A80E8898B188AF0
:1023600088898830B0F588899927FC01EE57F24FAB
:1023700080818B8B8B89833250F48B890E949D598D
:10238000882301F18A899989892B8A8B1BC08B89C3
:102390008E3250F48B890E943109882399F08A8902
:1023A0009989892B8A8B0EC08B898E3259F4809142
:1023B0003400992780719070009721F08A8999895B
:1023C000892B8A8B89898695898B88898F5F888BF1
:1023D000C7CF8A8989871A8A80E8898B188A888971
:1023E0008830B0F588899927FC01E657F24F808143
:1023F0008B8B8B89833250F48B890E949D59882363
:1024000001F18A899989892B8A8B1BC08B898E322D
:1024100050F48B890E943109882399F08A8999891F
:10242000892B8A8B0EC08B898E3259F480913400AF
:10243000992780719070009721F08A899989892B5A
:102440008A8B89898695898B88898F5F888BC7CF8E
:102450008A898A871A8A80E8898B188A88898830CD
:10246000B0F588899927FC01EE56F24F80818B8B5D
:102470008B89833250F48B890E949D59882301F106
:102480008A899989892B8A8B1BC08B898E3250F45B
:102490008B890E943109882399F08A899989892B2F
:1024A0008A8B0EC08B898E3259F480913400992723
:1024B00080719070009721F08A899989892B8A8B85
:1024C00089898695898B88898F5F888BC7CF8A8910
:1024D0008B871A8A80919A0D8B8B8B89833248F473
:1024E0008B890E949D598823F1F08A8980688A8BA4
:1024F0001AC08B898E3248F48B890E943109882357
:1025000091F08A8980688A8B0EC08B898E3259F44B
:1025100080913400992780719070009721F08A890A
:102520009989892B8A8B80919B0D8B8B8B89833228
:1025300048F48B890E949D598823F1F08A89806430
:102540008A8B1AC08B898E3248F48B890E9431099C
:10255000882391F08A8980648A8B0EC08B898E32A1
:1025600059F480913400992780719070009721F080
:102570008A899989892B8A8B8A898C878C899D89FC
:102580002AE030E0B9010E942EBDCB018D871E8666
:102590001F86CE0103960E94207F8091C90C9091E6
:1025A000CA0C009709F483C18091C90C9091CA0CA0
:1025B00001979093CA0C8093C90C8091C90C90919B
:1025C000CA0C009709F073C180912E0D90912F0DC8
:1025D0002AE030E0B9010E942EBDCB019093CA0CD5
:1025E0008093C90C8091300D9091310DAA27BB27A3
:1025F0008B839C83AD83BE8388E08F831A8A80E8B7
:10260000898B188A88898830B0F588899927FC01D8
:10261000EE5CF24F80818B8B8B89833250F48B89F7
:102620000E94015A882301F18A899989892B8A8B12
:102630001BC08B898E3250F48B890E94310988230C
:1026400099F08A899989892B8A8B0EC08B898E3261
:1026500059F480913400992780719070009721F08F
:102660008A899989892B8A8B89898695898B88891A
:102670008F5F888BC7CF8A8988871A8A80E8898B81
:10268000188A88898830B0F588899927FC01E65C2A
:10269000F24F80818B8B8B89833250F48B890E941F
:1026A000015A882301F18A899989892B8A8B1BC059
:1026B0008B898E3250F48B890E943109882399F0DE
:1026C0008A899989892B8A8B0EC08B898E3259F41D
:1026D00080913400992780719070009721F08A8949
:1026E0009989892B8A8B89898695898B88898F5FBF
:1026F000888BC7CF8A8989871A8A80E8898B188A4C
:1027000088898830B0F588899927FC01EE5BF24F03
:1027100080818B8B8B89833250F48B890E94015A84
:10272000882301F18A899989892B8A8B1BC08B891F
:102730008E3250F48B890E943109882399F08A895E
:102740009989892B8A8B0EC08B898E3259F480919E
:102750003400992780719070009721F08A899989B7
:10276000892B8A8B89898695898B88898F5F888B4D
:10277000C7CF8A898A871A8A80E8898B188A8889CC
:102780008830B0F588899927FC01E65BF24F80819B
:102790008B8B8B89833250F48B890E94015A88235A
:1027A00001F18A899989892B8A8B1BC08B898E328A
:1027B00050F48B890E943109882399F08A8999897C
:1027C000892B8A8B0EC08B898E3259F4809134000C
:1027D000992780719070009721F08A899989892BB7
:1027E0008A8B89898695898B88898F5F888BC7CFEB
:1027F0008A898B871A8A8091520D8B8B8B898332C1
:1028000048F48B890E94015A8823F1F08A898068F4
:102810008A8B1AC08B898E3248F48B890E943109C9
:10282000882391F08A8980688A8B0EC08B898E32CA
:1028300059F480913400992780719070009721F0AD
:102840008A899989892B8A8B8091530D8B8B8B89EF
:10285000833248F48B890E94015A8823F1F08A89D7
:1028600080648A8B1AC08B898E3248F48B890E94CF
:102870003109882391F08A8980648A8B0EC08B8904
:102880008E3259F4809134009927807190700097AE
:1028900021F08A899989892B8A8B8A898C878E89EC
:1028A0008D871E861F86CE0103960E94207F809111
:1028B000720D9091730D009709F466C28091720DAC
:1028C0009091730D01979093730D8093720D809189
:1028D000720D9091730D009709F056C28091E80C2B
:1028E0009091E90C2AE030E0B9010E942EBDCB01A5
:1028F0009093730D8093720D8091EA0C9091EB0C84
:10290000AA27BB278B839C83AD83BE8388E08F83FC
:102910001A8A80E8898B188A8889883008F052C022
:1029200088899927FC01E451F34F80818B8B8B8937
:10293000833250F48B890E949D598823E1F18A8962
:102940009989892B8A8B37C08B898E3250F48B8979
:102950000E943109882379F18A899989892B8A8B88
:102960002AC08B898E3458F48B898D520E94571A55
:10297000882309F18A899989892B8A8B1CC08B89C4
:10298000823658F48B898D520E9456A9882399F07B
:102990008A899989892B8A8B0EC08B89823659F452
:1029A00080913400992780719070009721F08A8976
:1029B0009989892B8A8B89898695898B88898F5FEC
:1029C000888BAACF8A8988871A8A80E8898B188A97
:1029D0008889883008F052C088899927FC01EC501A
:1029E000F34F80818B8B8B89833250F48B890E94CB
:1029F0009D598823E1F18A899989892B8A8B37C06F
:102A00008B898E3250F48B890E943109882379F1A9
:102A10008A899989892B8A8B2AC08B898E3458F4AC
:102A20008B898D520E94571A882309F18A899989C6
:102A3000892B8A8B1CC08B89823658F48B898D52E6
:102A40000E9456A9882399F08A899989892B8A8BB3
:102A50000EC08B89823659F4809134009927807199
:102A60009070009721F08A899989892B8A8B8989AE
:102A70008695898B88898F5F888BAACF8A89898779
:102A80001A8A80E8898B188A8889883008F052C0B1
:102A900088899927FC01E450F34F80818B8B8B89C7
:102AA000833250F48B890E949D598823E1F18A89F1
:102AB0009989892B8A8B37C08B898E3250F48B8908
:102AC0000E943109882379F18A899989892B8A8B17
:102AD0002AC08B898E3458F48B898D520E94571AE4
:102AE000882309F18A899989892B8A8B1CC08B8953
:102AF000823658F48B898D520E9456A9882399F00A
:102B00008A899989892B8A8B0EC08B89823659F4E0
:102B100080913400992780719070009721F08A8904
:102B20009989892B8A8B89898695898B88898F5F7A
:102B3000888BAACF8A898A871A8A80E8898B188A23
:102B40008889883008F052C088899927FC01EC5F99
:102B5000F24F80818B8B8B89833250F48B890E945A
:102B60009D598823E1F18A899989892B8A8B37C0FD
:102B70008B898E3250F48B890E943109882379F138
:102B80008A899989892B8A8B2AC08B898E3458F43B
:102B90008B898D520E94571A882309F18A89998955
:102BA000892B8A8B1CC08B89823658F48B898D5275
:102BB0000E9456A9882399F08A899989892B8A8B42
:102BC0000EC08B89823659F4809134009927807128
:102BD0009070009721F08A899989892B8A8B89893D
:102BE0008695898B88898F5F888BAACF8A898B8706
:102BF0001A8A80E8898B188A8889883048F58889FC
:102C00009927FC01E45FF24F80818B8B8B898332A3
:102C100050F48B890E94015A882399F08A899989F6
:102C2000892B8A8B0EC08B89833259F480913400B2
:102C3000992780719070009721F08A899989892B52
:102C40008A8B89898695898B88898F5F888BD4CF79
:102C50008A898C871A8A80E8898B188A88898830C3
:102C600048F588899927FC01EC5EF24F80818B8BB7
:102C70008B89833250F48B890E94015A882399F002
:102C80008A899989892B8A8B0EC08B89833259F462
:102C900080913400992780719070009721F08A8983
:102CA0009989892B8A8B89898695898B88898F5FF9
:102CB000888BD4CF8A898D871A8A80E8898B188A75
:102CC0008889883048F588899927FC01E45EF24FAD
:102CD00080818B8B8B89833250F48B890E94015ABF
:102CE000882399F08A899989892B8A8B0EC08B89D0
:102CF000833259F480913400992780719070009745
:102D000021F08A899989892B8A8B89898695898B73
:102D100088898F5F888BD4CF8A898E871A8A80E8CA
:102D2000898B188A8889883048F588899927FC0119
:102D3000EC5DF24F80818B8B8B89833250F48B89D1
:102D40000E94015A882399F08A899989892B8A8B54
:102D50000EC08B89833259F4809134009927807199
:102D60009070009721F08A899989892B8A8B8989AB
:102D70008695898B88898F5F888BD4CF8A898F8746
:102D8000CE0103960E94207FA8960FB6F894DEBF6E
:102D90000FBECDBFDF91CF910895CF93DF93CDB715
:102DA000DEB729970FB6F894DEBF0FBECDBF809176
:102DB000BA0D9091BB0D23E0883E920731F084EF6D
:102DC00091E09093BB0D8093BA0D8FE090E09093CB
:102DD000BD0D8093BC0D89E999E09093BF0D809360
:102DE000BE0D1092C00D1092C10D1092C20D109226
:102DF000C30D1092C50D1092C40D8AEB9DE09A830D
:102E0000898380E890E09C838B8380E190E09E83BF
:102E10008D838D819E8198878F838F819885AB81EB
:102E2000BC81E981FA81019724F001900E94D1BD13
:102E3000FACF98878F83CD019C838B83CF019A83B0
:102E4000898329960FB6F894DEBF0FBECDBFDF9100
:102E5000CF910895CF92DF92EF92FF920F931F933D
:102E6000CF93DF93CDB7DEB7E8970FB6F894DEBF08
:102E70000FBECDBF1DA68DA5803208F034C2BE01A5
:102E80006F5F7F4F8DA50E94A2688DA599278295BF
:102E90009295907F9827807F9827FC01EE52FE4FF5
:102EA00089818170982F917080818E7F892B80839A
:102EB0008DA5992782959295907F9827807F982756
:102EC000FC01EE52FE4F8981869583708370982FA6
:102ED000990F8081897F892B80838DA59927829581
:102EE0009295907F9827807F9827FC01ED53FE4FA5
:102EF0008A819B81918380838DA599278295929564
:102F0000907F9827807F9827FC01EB53FE4F8C81A0
:102F10009D81918380838DA5992782959295907F3D
:102F20009827807F9827FC01E953FE4F8E819F816F
:102F3000918380838DA5992782959295907F98277C
:102F4000807F9827FC01E753FE4F88859985918300
:102F500080838DA5992782959295907F9827807F71
:102F60009827FC01E553FE4F8A85982F9F7080813A
:102F7000807F892B80838DA5992782959295907F5C
:102F80009827807F9827FC01E553FE4F8B85982F6B
:102F90009295907F80818F70892B80838DA5992752
:102FA00082959295907F9827807F9827FC01E45323
:102FB000FE4F8C8580838DA5992782959295907F71
:102FC0009827807F9827FC01E353FE4F8D858083EF
:102FD0008DA5992782959295907F9827807F982735
:102FE000FC01E253FE4F8E8580838DA59927829543
:102FF0009295907F9827807F9827FC01E153FE4FA0
:103000008F8580838DA5992782959295907F9827AB
:10301000807F9827FC01EE52FE4F8F8D8170982F94
:10302000990F990F990F8081877F892B80838DA5B8
:10303000992782959295907F9827807F9827FC0109
:10304000E053FE4F88A180838DA5992782959295A4
:10305000907F9827807F9827FC01EF52FE4F89A12F
:1030600080838DA5992782959295907F9827807F60
:103070009827FC01EE52FE4F8AA18170982F9295FD
:10308000907F80818F7E892B80838DA59927829563
:103090009295907F9827807F9827FC01E553FE4FFB
:1030A00080818F708823F9F08DA59927829592955C
:1030B000907F9827807F9827FC01E553FE4F808101
:1030C0008F70813081F08DA5992782959295907FA0
:1030D0009827807F9827FC01E553FE4F80818F70F1
:1030E000823009F043C08DA5992782959295907FF3
:1030F0009827807F98270F2EF7ECCF2EF1E0DF2E58
:10310000F02DC80ED91E8E819F81AA2797FDA0950C
:10311000BA2FBC01CD010E943DBADC01CB0128A52C
:1031200039A54AA55BA5BC01CD010E9457B97B0119
:103130008C018CA5992787FD9095A92FB92FBC01EB
:10314000CD010E943DBADC01CB019C01AD01C8015B
:10315000B7010E9422B9DC01CB01BC01CD010E9464
:10316000A3B7DC01CB01F601918380838DA599275C
:1031700082959295907F9827807F9827FC01E55350
:10318000FE4F808182958F70882309F18DA5992744
:1031900082959295907F9827807F9827FC01E55330
:1031A000FE4F808182958F70813089F08DA599279F
:1031B00082959295907F9827807F9827FC01E55310
:1031C000FE4F808182958F70823009F043C08DA5BB
:1031D000992782959295907F9827807F98270F2E28
:1031E000F9ECCF2EF1E0DF2EF02DC80ED91E888528
:1031F0009985AA2797FDA095BA2FBC01CD010E9401
:103200003DBADC01CB0128A539A54AA55BA5BC01C7
:10321000CD010E9457B97B018C018CA5992787FDB0
:103220009095A92FB92FBC01CD010E943DBADC01B8
:10323000CB019C01AD01C801B7010E9422B9DC019C
:10324000CB01BC01CD010E94A3B7DC01CB01F6018B
:10325000918380838DA5992782959295907F982759
:10326000807F9827FC01EE52FE4F80818695837007
:10327000813041F48DA59927FC01ED53FC4F81E08D
:10328000808306C08DA59927FC01ED53FC4F108269
:103290008DA5992782959295907F9827807F982772
:1032A000FC01EE52FE4F80818F7D80838DA5992792
:1032B00082959295907F9827807F9827FC01EE5207
:1032C000FE4F80818F7B80838DA5282F3327C901F6
:1032D000820F931FFC01EE50FC4F118210828DA5CE
:1032E0008F5F8DA7C8CDCE018E9699AB88AB83E357
:1032F00098E09BAB8AAB82E090E09DAB8CAB8CA955
:103300009DA99FAB8EAB8EA99FA9AAA9BBA9E8A92D
:10331000F9A9019724F00E94C9BD0192FACF9FAB91
:103320008EABCD019BAB8AABCF0199AB88AB8EA5A1
:103330008093F0038FA58093F1031092E403109221
:10334000E303E8960FB6F894DEBF0FBECDBFDF9162
:10335000CF911F910F91FF90EF90DF90CF90089544
:10336000CF93DF93CDB7DEB7E8970FB6F894DEBF03
:103370000FBECDBF1DA68DA5803208F04CC0A8950C
:1033800089818E7F89838981897F89831B821A82C3
:103390001D821C821F821E82198618861A861B8631
:1033A0001C8681E08D871E8681E08F871F8E18A284
:1033B00019A21AA280E090E0A0E8BFE388A799A72D
:1033C000AAA7BBA71CA6CE01839645E050E060E00B
:1033D00070E00E94E9BCCE0140964FE050E060E012
:1033E00070E00E94E9BC9DA58FE0989FC001112468
:1033F0008C529F4F9E01205F3F4FBC01C9010E942C
:10340000C8BCBE016F5F7F4F8DA50E9452688DA51D
:103410008F5F8DA7B0CFCE018E9642E050E060E086
:1034200070E00E94E9BCCE018E9699AB88AB83E335
:1034300098E09BAB8AAB82E090E09DAB8CAB8CA913
:103440009DA99FAB8EAB8EA99FA9AAA9BBA9E8A9EC
:10345000F9A9019724F001900E94D1BDFACF9FAB4A
:103460008EABCD019BAB8AABCF0199AB88ABE89615
:103470000FB6F894DEBF0FBECDBFDF91CF91089598
:10348000CF93DF93CDB7DEB721970FB6F894DEBFA9
:103490000FBECDBF898389818093E30321960FB648
:1034A000F894DEBF0FBECDBFDF91CF9108950F938B
:1034B000CF93DF93CDB7DEB723970FB6F894DEBF77
:1034C0000FBECDBF89838981882321F08981813214
:1034D00008F40EC000E021E0AE014F5F5F4F6EE0E8
:1034E00071E081E091E00E942F601B821A8209C086
:1034F00089819927FC01EE53FC4F808199279B839A
:103500008A838A819B8123960FB6F894DEBF0FBE13
:10351000CDBFDF91CF910F910895CF93DF93CDB7BA
:10352000DEB723970FB6F894DEBF0FBECDBF8091F4
:10353000F0038823A1F08091F1030E945683882331
:1035400071F419828981803250F489819927FC01B4
:10355000ED53FC4F108289818F5F8983F3CF1982ED
:103560008981803208F07EC08981282F3327C901E4
:10357000820F931FFC01EE50FC4F808191810097D8
:1035800009F46CC08981282F3327C901820F931F4A
:10359000DC01AE50BC4F8981282F3327C901820F2F
:1035A000931FFC01EE50FC4F808191810197119691
:1035B0009C938E938981282F3327C901820F931FF3
:1035C000FC01EE50FC4F80819181009709F046C0CC
:1035D0008981992782959295907F9827807F982757
:1035E000FC01EE52FE4F808186958370282F332791
:1035F0003B832A838A819B818130910561F02A81F6
:103600003B812230310571F089819927FC01ED530E
:10361000FC4F108207C089819927FC01ED53FC4FB4
:1036200081E080838981992782959295907F982760
:10363000807F9827FC01EE52FE4F80818F7D808332
:103640008981992782959295907F9827807F9827E6
:10365000FC01EE52FE4F80818F7B808389818F5FDA
:1036600089837ECF23960FB6F894DEBF0FBECDBF01
:10367000DF91CF910895CF93DF93CDB7DEB78091DF
:10368000E303882381F08091E403882361F048EE0E
:1036900053E06091E7038091E5039091E6030E9477
:1036A0004D9E1092E403DF91CF910895CF93DF9365
:1036B000CDB7DEB760970FB6F894DEBF0FBECDBFB3
:1036C0009A8389831A8619861F828091F003882342
:1036D00039F08091F1030E945683882309F4D3C303
:1036E000E981FA818091BE0D9091BF0D9C01442724
:1036F000552780819181A281B38182179307A40706
:10370000B507D1F429813A818091C00D9927820FA4
:10371000931FFC01359690818091C10D9823809173
:10372000C10D981749F40E94C2A00E943F47109211
:10373000E90D82E2809311011D828D81803208F0B3
:1037400046C38D81992782959295907F9827807F97
:1037500098278D539E4F9C838B83EB81FC818081C6
:1037600091819C0144275527E981FA8180819181CB
:10377000A281B381281739074A075B0799F0EB81CB
:10378000FC81828193819C0144275527E981FA813C
:1037900080819181A281B381281739074A075B078D
:1037A00009F022C08D81282F3327C901820F931F72
:1037B000FC01EE50FC4F8091BC0D9091BD0D9183AA
:1037C00080838091E303833068F08091E30399273D
:1037D0009C012F7330708D81992703962817390724
:1037E00009F002C081E08F83EB81FC8187858870BE
:1037F0008823A9F0AB81BC8129813A81EB81FC81CE
:1038000085859927820F931F0596988B8F87FD01D9
:103810009685EF85F8898081981709F0D4C2EB81ED
:10382000FC8180819181009709F4CDC2EB81FC81FC
:10383000808191819C0144275527E981FA8180810B
:103840009181A281B381281739074A075B0709F0E4
:1038500057C181E08E83EB81FC818185882321F132
:1038600029813A81EB81FC8181859927820F931F01
:10387000FC01349680819927982F88279A87898719
:1038800029813A81EB81FC8182859927820F931FE0
:10389000FC0134968081282F332789859A85820FF1
:1038A000931F9A87898724C0EB81FC8182858823B6
:1038B000F1F029813A81EB81FC8182859927820F81
:1038C000931FFC013496808199279A878987EB8121
:1038D000FC8187858071882359F0898580788823C9
:1038E00039F089859A859F6F9A87898701C01E82E2
:1038F0008E81882309F404C1EB81FC8180858F705F
:10390000282F33273C872B878B859C858330910517
:1039100009F48EC0EB85FC85E430F10584F42B8539
:103920003C852130310581F18B859C858230910564
:103930000CF054C0EB85FC853097A1F0E1C02B85DD
:103940003C852530310509F499C08B859C858530EF
:1039500091050CF480C0EB85FC85E630F10509F497
:103960009EC0CEC0EB81FC812481358189859A85FA
:103970002817390709F0C4C08D819927FC01ED5340
:10398000FC4F81E08083BCC0EB81FC818785807126
:10399000882391F0EB81FC8129853A85848195818A
:1039A000821793070CF0ACC08D819927FC01ED5371
:1039B000FC4F81E08083A4C0EB81FC8124813581B0
:1039C00089859A852817390708F09AC08D8199272B
:1039D000FC01ED53FC4F81E0808392C0EB81FC81C0
:1039E00087858071882391F0EB81FC8129853A8558
:1039F00084819581281739070CF082C08D81992721
:103A0000FC01ED53FC4F81E080837AC0EB81FC81A7
:103A10002481358189859A858217930708F070C0C3
:103A20008D819927FC01ED53FC4F81E0808368C0B4
:103A3000EB81FC812481358189859A8582239323BA
:103A4000009709F45DC08D819927FC01ED53FC4F6F
:103A500081E0808355C0EB81FC812481358189859B
:103A60009A8582239323009709F04AC08D81992774
:103A7000FC01ED53FC4F81E0808342C0EB81FC816F
:103A80002481358189859A8528173907C9F18D8167
:103A90009927FC01ED53FC4F81E0808331C0EB811D
:103AA000FC812481358189859A858223932300971F
:103AB00011F1EB81FC8187858072882309F5EB8108
:103AC000FC818785806287878D819927FC01ED5372
:103AD000FC4F8081813039F48D819927FC01ED53B1
:103AE000FC4F10820DC08D819927FC01ED53FC4FD6
:103AF00081E0808305C0EB81FC8187858F7D87878E
:103B0000EB81FC81828193819C0144275527E981C7
:103B1000FA8180819181A281B381281739074A07F0
:103B20005B0709F050C181E08E83EB81FC818385C6
:103B3000882321F129813A81EB81FC8183859927B2
:103B4000820F931FFC01349680819927982F882734
:103B50009A87898729813A81EB81FC81848599271D
:103B6000820F931FFC0134968081282F332789858B
:103B70009A85820F931F9A87898724C0EB81FC81E5
:103B800084858823F1F029813A81EB81FC81848549
:103B90009927820F931FFC013496808199279A8779
:103BA0008987EB81FC8187858071882359F089851D
:103BB0008078882339F089859A859F6F9A878987CD
:103BC00001C01E828E81882309F4FDC0EB81FC8137
:103BD000808582958F70282F33273E872D878D858E
:103BE0009E858330910509F489C0ED85FE85E4301A
:103BF000F10584F42D853E852130310579F18D85DF
:103C00009E85823091050CF051C0ED85FE85309780
:103C1000A1F0D9C02D853E852530310509F492C02B
:103C20008D859E85853091050CF47AC0ED85FE85E5
:103C3000E630F10509F496C0C6C0EB81FC8126810F
:103C4000378189859A852817390709F0BCC08D818D
:103C50009927FC01ED53FC4F1082B5C0EB81FC812C
:103C600087858071882389F0EB81FC8129853A85DD
:103C700086819781821793070CF0A5C08D819927C3
:103C8000FC01ED53FC4F10829EC0EB81FC8126812C
:103C9000378189859A852817390708F094C08D8166
:103CA0009927FC01ED53FC4F10828DC0EB81FC8104
:103CB00087858071882389F0EB81FC8129853A858D
:103CC00086819781281739070CF07DC08D8199274F
:103CD000FC01ED53FC4F108276C0EB81FC81268104
:103CE000378189859A858217930708F06CC08D818A
:103CF0009927FC01ED53FC4F108265C0EB81FC81DC
:103D00002681378189859A8582239323009709F438
:103D10005AC08D819927FC01ED53FC4F108253C08E
:103D2000EB81FC812681378189859A8582239323C3
:103D3000009709F048C08D819927FC01ED53FC4F95
:103D4000108241C0EB81FC812681378189859A856B
:103D500028173907C1F18D819927FC01ED53FC4FDC
:103D6000108231C0EB81FC812681378189859A855B
:103D700082239323009711F1EB81FC818785807466
:103D8000882309F5EB81FC818785806487878D8195
:103D90009927FC01ED53FC4F8081813039F48D81EE
:103DA0009927FC01ED53FC4F10820DC08D8199279E
:103DB000FC01ED53FC4F81E0808305C0EB81FC8169
:103DC00087858F7B87878D818F5F8D83B6CC809130
:103DD000E303882309F457C08F81882329F4809155
:103DE000E303823009F04FC08091E403823009F48C
:103DF0004AC08091E5039091E6039C014427552732
:103E0000E981FA8180819181A281B38128173907E4
:103E10004A075B07B9F4E981FA819091E70384814D
:103E2000981781F48091E703282F332789819A819D
:103E30000596A901BC0188EE93E00E94CFBC0097D3
:103E400009F41EC082E08093E403E981FA81848151
:103E50008093E703E981FA81808191819093E60361
:103E60008093E5038091E703282F332789819A8186
:103E70000596A901BC0188EE93E00E94DCBC03C05A
:103E800081E08093E40360960FB6F894DEBF0FBE26
:103E9000CDBFDF91CF910895CF93DF93CDB7DEB73C
:103EA0000E9416078091D80082608093D800DF912D
:103EB000CF910895CF93DF93CDB7DEB728970FB694
:103EC000F894DEBF0FBECDBF9A838983E981FA8162
:103ED00081818330D1F4E981FA818185882309F4D5
:103EE000ABC1E981FA8180818295807F8093ED006A
:103EF0009FE38091EF0089238093EF00E981FA81AD
:103F00001082E981FA81118697C10E9454078B8340
:103F1000E981FA8181E081878B818F3F09F487C134
:103F2000E981FA818B8180838B818295807F809368
:103F3000ED001092EE001092EF001092F700109238
:103F4000F6001092F5001092F4001092F000E98152
:103F5000FA818181282F332738872F838F81988595
:103F60008130910509F4BAC02F813885223031059E
:103F70002CF48F819885009741F055C12F813885A9
:103F80002230310509F443C14EC1E981FA818285AD
:103F90008270882309F458C089819A81FC01359682
:103FA000808199279C01220F331F220F331F220F7C
:103FB000331F89819A81FC01349680818295869590
:103FC0008770820F8093F30089819A81FC01349677
:103FD000808199279C01220F331F220F331F220F4C
:103FE000331F89819A81FC01339680818295869561
:103FF0008770820F8093F20089819A81FC01339649
:10400000808199279C01220F331F220F331F220F1B
:10401000331F89819A81FC01329680818295869531
:104020008770820F8093F10089819A81FC0132961A
:104030008081880F880F880F8093F0008091EF00B7
:1040400080618093EF0024C089819A81FC013396BE
:10405000808199279C01220F331F22953295307F52
:104060003227207F322789819A81FC013296808114
:10407000869586958695820F8093F30089819A8133
:10408000FC01329680818295880F807E8093F200B9
:104090001C82E981FA8196818C81891788F4E981F3
:1040A000FA818C81282F332787819085F901E80FC9
:1040B000F91F80818093FA008C818F5F8C83E9CF18
:1040C000E981FA819091EF008681892B8093EF003E
:1040D0008091EF0080648093EF00AEC0E981FA81A7
:1040E00082858270882309F45DC089819A81FC01F0
:1040F0003596808199279C01220F331F220F331F91
:10410000220F331F89819A81FC0134968081829528
:1041100086958770820F8093F30089819A81FC01D4
:104120003496808199279C01220F331F220F331F61
:10413000220F331F89819A81FC01339680818295F9
:1041400086958770820F8093F20089819A81FC01A5
:104150003396808199279C01220F331F220F331F32
:10416000220F331F89819A81FC01329680818295CA
:1041700086958770820F8093F10089819A81FC0176
:1041800032968081880F880F880F8093F00080918D
:10419000EF0080618093EF008091F0008460809355
:1041A000F00027C089819A81FC013396808199278C
:1041B0009C01220F331F22953295307F3227207FBA
:1041C000322789819A81FC01329680818695869575
:1041D0008695820F8093F30089819A81FC01329643
:1041E00080818295880F807E8093F20084E08093A6
:1041F000F000E981FA819091EF008681892B80930C
:10420000EF008091EF0080648093EF0015C09FE382
:104210008091EF0089238093EF008091EF00806808
:104220008093EF0009C0E981FA81118605C08FEF04
:1042300090E09E838D8302C01E821D828D819E81AF
:1042400028960FB6F894DEBF0FBECDBFDF91CF9199
:104250000895CF93DF93CDB7DEB725970FB6F894C7
:10426000DEBF0FBECDBF9A838983E981FA81818544
:10427000882329F482E090E09D838C83CBC0E98180
:10428000FA8180818295807F8093ED000E948E0765
:104290008B838B81813009F0AAC0E981FA81118674
:1042A000E981FA818091EF008F708683E981FA813C
:1042B000878190850E94C807E981FA818091F0008A
:1042C0009927847090709595879595958795982FE7
:1042D000917082858E7F892B82878091EF0099274C
:1042E00080719070009709F455C0E981FA81828548
:1042F0008260828789819A81FC0135968091F300E2
:10430000869586958695808389819A81FC0134966D
:104310008091F200282F2695269526958091F3000E
:104320009927880F991F82959295907F9827807F73
:104330009827820F808389819A81FC01339680912E
:10434000F100282F2695269526958091F200992731
:10435000880F991F82959295907F9827807F982744
:10436000820F808389819A81FC0132968091F000CE
:10437000282F2695269526958091F1009927880F5C
:10438000991F82959295907F9827807F9827820F1A
:10439000808324C0E981FA8182858D7F828789812B
:1043A0009A81FC0133968091F300829586958770FF
:1043B000808389819A81FC0132968091F200282FB6
:1043C0002295269527708091F3009927880F991FD1
:1043D000880F991F880F991F820F80838FE3909118
:1043E000EF0089238093EF001D821C8213C08B8114
:1043F000882361F4E981FA8111869FE38091EF00BF
:1044000089238093EF001D821C8204C08B81992731
:104410009D838C838C819D8125960FB6F894DEBF99
:104420000FBECDBFDF91CF910895CF93DF93CDB76E
:10443000DEB723970FB6F894DEBF0FBECDBF8983DA
:1044400089818F3F29F481E090E09B838A8336C085
:104450008981803C50F08981843D38F489810E94B3
:10446000568399279B838A8329C08981882351F0A9
:104470008981813238F489810E94571A99279B8358
:104480008A831CC08981813250F08981853338F458
:1044900089810E9456A999279B838A830FC08981AD
:1044A000873350F08981833438F489810E947847BA
:1044B00099279B838A8302C01B821A828A819B81EF
:1044C00023960FB6F894DEBF0FBECDBFDF91CF911C
:1044D0000895CF93DF93CDB7DEB723970FB6F89447
:1044E000DEBF0FBECDBF898389818F3F29F481E074
:1044F00090E09B838A8336C08981803C50F089811B
:10450000843D38F489810E94348199279B838A8372
:1045100029C08981882351F08981813238F48981C9
:104520000E94571A99279B838A831CC089818132F4
:1045300050F08981853338F489810E9456A99927E2
:104540009B838A830FC08981873350F089818334AC
:1045500038F489810E94784799279B838A8302C017
:104560001B821A828A819B8123960FB6F894DEBF44
:104570000FBECDBFDF91CF910895CF93DF93CDB71D
:10458000DEB78091D00D9091D10D01969093D10D11
:104590008093D00D8091DB0D9091DC0D019690936E
:1045A000DC0D8093DB0D8091CD0D9091CE0D0196A9
:1045B0009093CE0D8093CD0D8091DA0D833008F469
:1045C00074C08091DA0D8F5F8093DA0D8091DA0DDF
:1045D000843031F441E061E484E00E94F47665C007
:1045E0008091D00D9091D10D8035910598F48091F6
:1045F000DA0D853031F441E061E484E00E946877AF
:1046000054C08091DA0D883009F04FC083E0809368
:10461000DA0D4BC08091D00D9091D10D803A91056B
:1046200090F48091DA0D853031F441E061E484E06A
:104630000E9468773AC08091DA0D8730B0F183E04C
:104640008093DA0D32C08091D00D9091D10D21E090
:104650008836920790F48091DA0D863031F441E08B
:1046600061E484E00E94687720C08091DA0D873091
:10467000E0F083E08093DA0D18C08091D00D909126
:10468000D10D21E08E3F920768F48091DA0D8730DA
:1046900060F041E061E484E00E94687783E0809309
:1046A000DA0D03C081E08093DA0D8091CC0D833068
:1046B00008F474C08091CC0D8F5F8093CC0D8091F5
:1046C000CC0D843031F440E061E486E00E94F47661
:1046D00065C08091DB0D9091DC0D8035910598F4DB
:1046E0008091CC0D853031F440E061E486E00E9499
:1046F000687754C08091CC0D883009F04FC083E0BA
:104700008093CC0D4BC08091DB0D9091DC0D803AF5
:10471000910590F48091CC0D853031F440E061E456
:1047200086E00E9468773AC08091CC0D8730B0F166
:1047300083E08093CC0D32C08091DB0D9091DC0D35
:1047400021E08836920790F48091CC0D863031F4C8
:1047500040E061E486E00E94687720C08091CC0D43
:104760008730E0F083E08093CC0D18C08091DB0DA2
:104770009091DC0D21E08E3F920768F48091CC0D82
:10478000873060F040E061E486E00E94687783E073
:104790008093CC0D03C081E08093CC0D8091CF0D30
:1047A000833008F474C08091CF0D8F5F8093CF0D5C
:1047B0008091CF0D843031F441E061E486E00E94C5
:1047C000F47665C08091CD0D9091CE0D8035910528
:1047D00098F48091CF0D853031F441E061E486E0BA
:1047E0000E94687754C08091CF0D883009F04FC087
:1047F00083E08093CF0D4BC08091CD0D9091CE0D75
:10480000803A910590F48091CF0D853031F441E0EC
:1048100061E486E00E9468773AC08091CF0D8730CE
:10482000B0F183E08093CF0D32C08091CD0D909197
:10483000CE0D21E08836920790F48091CF0D86301E
:1048400031F441E061E486E00E94687720C0809105
:10485000CF0D8730E0F083E08093CF0D18C08091BA
:10486000CD0D9091CE0D21E08E3F920768F480919E
:10487000CF0D873060F041E061E486E00E94687708
:1048800083E08093CF0D03C081E08093CF0DDF9153
:10489000CF910895CF93DF93CDB7DEB78091D30D3D
:1048A0000E941522882321F085E08093CB0D48C01B
:1048B0008091D80D0E941522882341F08091D90D56
:1048C0008093030A83E08093CB0D3AC08091D20D90
:1048D0000E941522882321F084E08093CB0D30C004
:1048E0008091D40D0E941522882379F08091CB0D00
:1048F000873059F08091CB0D863039F086E0809377
:10490000CB0D8AE08093020A1BC08091CB0D8530CD
:1049100021F482E08093CB0D13C08091CB0D8330C6
:1049200041F48091030A882321F481E08093CB0D28
:1049300007C08091CB0D843019F481E08093CB0DBA
:104940008091CB0D813029F08091CB0D823009F020
:104950000CC08091D50D0E946922982F8091D60DB0
:10496000891719F41092CB0D18C08091020A882380
:10497000A1F48091CB0D863081F48091D50D0E94F9
:104980006922982F8091D60D891739F487E080939A
:10499000CB0D8091D70D8093010A86E699E00E94A5
:1049A000A35D0E940C28DF91CF910895CF93DF93F0
:1049B000CDB7DEB72A970FB6F894DEBF0FBECDBFD6
:1049C0001A828A81843008F0A3C18A81282F332774
:1049D000C901880F991F820F931FFC01E252F24F09
:1049E00080818823F9F08A81282F3327C901880F15
:1049F000991F820F931FFC01E252F24F80810E94A7
:104A00001522882379F08A81282F3327C901880F3E
:104A1000991F820F931FFC01E152F24F80818F7822
:104A2000808372C18A81282F3327C901880F991F7B
:104A3000820F931FFC01E352F24F8081882309F417
:104A400055C18A81282F3327C901880F991F820FEA
:104A5000931FFC01E352F24F80810E9415228823AC
:104A600009F444C18A81282F3327C901880F991F6F
:104A7000820F931FFC01E152F24F8081869586954B
:104A800086958170882309F03FC18A81282F3327BA
:104A9000C901880F991F820F931FFC01E152F24F49
:104AA0008081886080838A81282F3327C901880FFD
:104AB000991F820F931FFC01E152F24F8081877092
:104AC000282F33273A87298789859A85823091054F
:104AD00009F448C0E985FA85E330F10534F4298505
:104AE0003A852130310571F00FC189859A8583306F
:104AF000910509F483C0E985FA85E430F10509F4EC
:104B0000E5C002C18A81282F3327C901880F991F68
:104B1000820F931FFC01E152F24F808182958F70CA
:104B20008770882379F08A81282F3327C901880F5D
:104B3000991F820F931FFC01E152F24F80818F7801
:104B40008083E2C08A81282F3327C901880F991FEB
:104B5000820F931FFC01E152F24F80818F788061B8
:104B60008083D2C08A81282F3327C901880F991FDB
:104B7000820F931FFC01E152F24F808182958F706A
:104B80008770282F33273E832D838D819E81009748
:104B900031F0ED81FE81E130F10589F020C08A819C
:104BA000282F3327C901880F991F820F931FFC01FB
:104BB000E152F24F80818F7880618083A5C08A8125
:104BC000282F3327C901880F991F820F931FFC01DB
:104BD000E152F24F80818F788062808395C08A8114
:104BE000282F3327C901880F991F820F931FFC01BB
:104BF000E152F24F80818F78808386C08A81282F8E
:104C00003327C901880F991F820F931FFC01E152BE
:104C1000F24F808182958F708770282F33273887D5
:104C20002F838F8198858130910509F1EF81F88577
:104C3000E230F10534F42F8138852115310539F042
:104C400036C08F8198858230910509F130C08A8104
:104C5000282F3327C901880F991F820F931FFC014A
:104C6000E152F24F80818F78806180834DC08A81CC
:104C7000282F3327C901880F991F820F931FFC012A
:104C8000E152F24F80818F78806280833DC08A81BB
:104C9000282F3327C901880F991F820F931FFC010A
:104CA000E152F24F80818F78806380832DC08A81AA
:104CB000282F3327C901880F991F820F931FFC01EA
:104CC000E152F24F80818F7880831EC08A81282F25
:104CD0003327C901880F991F820F931FFC01E152EE
:104CE000F24F80818F78806180830EC08A81282F67
:104CF0003327C901880F991F820F931FFC01E152CE
:104D0000F24F8081877F80838A818F5F8A8359CE2B
:104D10000E9485480E9431460E94284C1982898150
:104D2000823208F098C0998185E2989FC0011124D1
:104D3000875C9B4F9C838B83EB81FC818489958965
:104D4000009751F0AB81BC81EB81FC81848995890E
:104D50000197FD01958B848BEB81FC818585968580
:104D60000097D9F0AB81BC81EB81FC81858596856C
:104D70000197FD0196878587EB81FC8181858F3FB7
:104D800061F0AB81BC81EB81FC81918585E0989FCE
:104D9000C0011124FD0193878287EB81FC8182850C
:104DA00093850097E9F0EB81FC8181858F3FC1F00D
:104DB000AB81BC81EB81FC81828593850197FD01EC
:104DC00093878287EB81FC8182859385009741F4EC
:104DD000AB81BC81EB81FC8187858062FD01878787
:104DE000EB81FC81828D938D009721F1AB81BC8199
:104DF000EB81FC81828D938D0197FD01938F828FD2
:104E0000EB81FC81828D938D0097A1F4EB81FC8175
:104E10008785992780749070009721F489818F5F2E
:104E20000E94B865AB81BC81EB81FC818785806481
:104E3000FD018787EB81FC818781882341F0AB816D
:104E4000BC81EB81FC8187818150FD018783898151
:104E50008F5F898364CF2A960FB6F894DEBF0FBEAA
:104E6000CDBFDF91CF910895CF93DF93CDB7DEB75C
:104E700021970FB6F894DEBF0FBECDBF8091020A16
:104E8000882329F08091020A81508093020A809140
:104E9000CB0D8730C9F48091010A882331F08091CD
:104EA000010A81508093010A0FC08091D40D0E94A5
:104EB0001522882339F086E08093CB0D8AE0809319
:104EC000020A02C01092CB0D8091030A882329F0B8
:104ED0008091030A81508093030A809134009927BE
:104EE00080719070009781F18091FE09898389819A
:104EF0008F3720F48981880F898302C08FEF8983DF
:104F00008091C20D8A3010F19091C20D8091CA0D2E
:104F1000891730F09091CA0D8981981708F006C062
:104F20008091CA0D8F5F8093CA0D10C08091E90DEA
:104F3000882361F48091E90D8F5F8093E90D0E94D1
:104F4000C2A00E943F4702C01092CA0D90915D0915
:104F500080916D09981748F5198289818C3008F085
:104F600052C089819927FC01E159F64F8081823234
:104F7000C0F489819927FC01E159F64F8081282FDF
:104F8000332785E290E0289FA001299F500D389F8C
:104F9000500D1124CA01FC01E35CFB4F808181604C
:104FA000808389818F5F8983D8CF90915D098091BB
:104FB0006E09891740F5198289818C3020F5898125
:104FC0009927FC01E159F64F80818232C0F4898132
:104FD0009927FC01E159F64F8081282F332785E27C
:104FE00090E0289FA001299F500D389F500D11245B
:104FF000CA01FC01E35CFB4F80818E7F8083898145
:105000008F5F8983D9CF21960FB6F894DEBF0FBE8C
:10501000CDBFDF91CF910895CF93DF93CDB7DEB7AA
:1050200027970FB6F894DEBF0FBECDBF8091330433
:10503000882309F01EC219828981853008F019C2BF
:105040008981992782959295907F9827807F9827CC
:105050008255964F9D838C831B82EC81FD818281DA
:105060008F3F19F481E08B8371C0EC81FD818281D7
:10507000803C60F0EC81FD818281843D38F4EC81DC
:10508000FD8182810E9456838B8360C0EC81FD810B
:105090008281882361F0EC81FD818281813238F444
:1050A000EC81FD8182810E94571A8B834FC0EC8175
:1050B000FD818281813260F0EC81FD8182818533C6
:1050C00038F4EC81FD8182810E9456A98B833EC019
:1050D000EC81FD8182818336B1F48091CB0D8330E8
:1050E00069F08091CB0D843049F08091CB0D8130F7
:1050F00029F08091CB0D863009F003C081E08B83CD
:1051000025C01B8223C0EC81FD818281843671F42D
:105110008091CB0D853029F08091CB0D823009F044
:1051200003C081E08B8312C01B8210C0EC81FD8123
:105130008281873358F0EC81FD818281833430F4A1
:10514000EC81FD8182810E9478478B83EC81FD8117
:105150008181282F33273F832E834E815F81413009
:10516000510509F465C08E819F81823091052CF430
:10517000EE81FF81309741F078C12E813F8122304E
:10518000310509F46CC171C18B81813009F06DC1A9
:10519000AC81BD81EC81FD8197818AE0989FC0013F
:1051A0001124FD0194838383AC81BD81EC81FD8159
:1051B00091858AE0989FC0011124FD019683858323
:1051C000EC81FD818081846080831A828A818630AF
:1051D00050F52C813D818A819927820F931FFC0114
:1051E0003A9680818F3FD9F02C813D818A81992721
:1051F000820F931FFC013A968081282F332785E286
:1052000090E0289FA001299F500D389F500D112438
:10521000CA01FC01E35CFB4F8081846080838A814A
:105220008F5F8A83D3CFEC81FD8181E081831DC1B3
:10523000EC81FD8183819481009709F416C1AC81D2
:10524000BD81EC81FD81838194810197FD0194836F
:105250008383EC81FD8183819481009709F067C08D
:10526000EC81FD8180818470882389F1AC81BD81CE
:10527000EC81FD8197818AE0989FC0011124FD0196
:1052800094838383EC81FD8180818B7F80831A826C
:105290008A81863008F04BC02C813D818A81992714
:1052A000820F931FFC013A9680818F3F61F02C8121
:1052B0003D818A819927820F931FFC013A9660E015
:1052C00080810E94422A8A818F5F8A83E1CFAC81EC
:1052D000BD81EC81FD8190858AE0989FC0011124F9
:1052E000FD0194838383EC81FD81808184608083D0
:1052F0001A828A818630D8F42C813D818A8199274F
:10530000820F931FFC013A9680818F3F61F02C81C0
:105310003D818A819927820F931FFC013A9661E0B3
:1053200080810E94422A8A818F5F8A83E2CFEC814A
:10533000FD8180818270882309F04BC0EC81FD8162
:1053400085819681009709F490C0AC81BD81EC8184
:10535000FD81858196810197FD0196838583EC818E
:10536000FD8185819681009709F07FC0EC81FD81E8
:1053700082E081831A828A81863008F076C02C818F
:105380003D818A819927820F931FFC013A96808183
:105390008F3FD9F02C813D818A819927820F931FFD
:1053A000FC013A968081282F332785E290E0289FE0
:1053B000A001299F500D389F500D1124CA01FC01F6
:1053C000E35CFB4F80818B7F80838A818F5F8A8340
:1053D000D2CF8B81882309F048C01A828A81863017
:1053E000D0F52C813D818A819927820F931FFC0182
:1053F0003A9680818F3F39F12C813D818A819927AE
:10540000820F931FFC013A968081282F332785E273
:1054100090E0289FF001299FF00D389FF00D112496
:10542000CF01FC01E35CFB4F80818B7F80832C816B
:105430003D818A819927820F931FFC013A9661E092
:1054400080810E94422AEC81FD81148213828A812C
:105450008F5F8A83C3CFEC81FD81118206C08B816F
:10546000882319F4EC81FD81118289818F5F898302
:10547000E3CD27960FB6F894DEBF0FBECDBFDF9108
:10548000CF9108950F93CF93DF93CDB7DEB72597D4
:105490000FB6F894DEBF0FBECDBF89836A831B822F
:1054A0008981833260F000E021E0AE014F5F5F4F01
:1054B00062E273E082E191E00E942F6080C09981F6
:1054C00085E2989FC0011124875C9B4F9D838C834C
:1054D000EC81FD81858D9927807F9070803A9105C0
:1054E00019F481E48B8317C0EC81FD81858D9927A8
:1054F000807F9070803B910519F482E48B830BC010
:1055000000E021E0AE014F5F5F4F6EE273E082E1A9
:1055100091E00E942F608A818823E1F4EC81FD8173
:1055200083E08783EC81FD8180EF8183AC81BD8145
:10553000EC81FD8187858F7BFD018787AC81BD81F3
:10554000EC81FD81858D8F70FD0141A16B810E94F1
:10555000F47635C08A81813091F5EC81FD81178226
:10556000EC81FD818FE08183AC81BD81EC81FD8187
:1055700087858F7DFD018787AC81BD81EC81FD81B1
:1055800087858E7FFD018787AC81BD81EC81FD81A0
:105590008785877FFD018787AC81BD81EC81FD8197
:1055A00087858F7BFD018787AC81BD81EC81FD8183
:1055B000858D8F70FD0141A16B810E9468772596D2
:1055C0000FB6F894DEBF0FBECDBFDF91CF910F9124
:1055D0000895CF93DF93CDB7DEB722970FB6F89437
:1055E000DEBF0FBECDBF89831A821A828A818431C1
:1055F00048F58A819927FC01E458F64F8081823270
:10560000E8F48A819927FC01E458F64F8081282F1D
:10561000332785E290E0289FA001299F500D389FF5
:10562000500D1124CA01FC01E35CFB4F898181709C
:10563000982F990F80818D7F892B80838A818F5F3E
:105640008A83D4CF22960FB6F894DEBF0FBECDBFAB
:10565000DF91CF910895CF93DF93CDB7DEB7229737
:105660000FB6F894DEBF0FBECDBF89831A821A82AF
:105670008A81843148F58A819927FC01EE56F64FDC
:1056800080818232E8F48A819927FC01EE56F64F38
:105690008081282F332785E290E0289FA001299F51
:1056A000500D389F500D1124CA01FC01E35CFB4FE3
:1056B00089818170982F990F80818D7F892B8083BC
:1056C0008A818F5F8A83D4CF22960FB6F894DEBF8B
:1056D0000FBECDBFDF91CF910895CF93DF93CDB7AC
:1056E000DEB78091350490913604DF91CF91089513
:1056F000CF93DF93CDB7DEB7809134049927DF9144
:10570000CF910895CF93DF93CDB7DEB726970FB62D
:10571000F894DEBF0FBECDBF89836A835C834B8361
:10572000898180936D098A8180936E091D828D81A4
:105730008C30D0F48D81282F33278B819C81F90107
:10574000E80FF91F80810E948C568E838E818232F1
:1057500038F48D819927FC01E159F64F8E818083C1
:105760008D818F5F8D83E3CF26960FB6F894DEBFD1
:105770000FBECDBFDF91CF910895CF93DF93CDB70B
:10578000DEB721970FB6F894DEBF0FBECDBF1982EA
:105790000E94B75A0E94B15C0E94F25C86E699E0D2
:1057A0000E947D5D10925B0910925A0910925C096B
:1057B00010925E0910925F091092600910926109BF
:1057C00042E150E060E070E083E299E00E94E9BCD1
:1057D00019828981823188F48981282F3327C90170
:1057E000820F931FFC01EB5CF64F88EB91E09183F5
:1057F000808389818F5F8983ECCF1982898185308D
:10580000C0F58981992782959295907F9827807F0E
:105810009827FC01E155F64F1082898199278295DE
:105820009295907F9827807F9827FC01EF54F64F40
:10583000118210828981992782959295907F98276D
:10584000807F9827FC01ED54F64F118210828981E8
:10585000992782959295907F9827807F9827FC01C1
:10586000E255F64F80818460808389818F5F8983D0
:10587000C5CF0E94846D803221F487E680931001A9
:1058800003C08EE68093100119828981282F332767
:1058900085E290E0289FA001299F500D389F500D70
:1058A0001124CA01FC01E75CFB4F81E08083898100
:1058B000282F332785E290E0289FA001299F500DD3
:1058C000389F500D1124CA01FC01E55BFB4F88ECA9
:1058D00090E0918380838981282F332785E290E0AF
:1058E000289FA001299F500D389F500D1124CA01F7
:1058F000FC01EA5AFB4F82EA80838981282F3327F3
:1059000085E290E0289FA001299F500D389F500DFF
:105910001124CA01FC01E95AFB4F82EB8083898183
:10592000282F332785E290E0289FA001299F500D62
:10593000389F500D1124CA01FC01E65AFB4F10821A
:105940008981282F332785E290E0289FA001299F95
:10595000500D389F500D1124CA01FC01E85AFB4F2D
:105960008FEF80838981282F332785E290E0289F5D
:10597000A001299F500D389F500D1124CA01FC0130
:10598000E75AFB4F82EA80838981282F332785E2FB
:1059900090E0289FA001299F500D389F500D1124A1
:1059A000CA01FC01E55AFB4F83E0808381E08983D3
:1059B0008981282F332785E290E0289FA001299F25
:1059C000500D389F500D1124CA01FC01E75CFB4FBC
:1059D00081E080838981282F332785E290E0289F0A
:1059E000A001299F500D389F500D1124CA01FC01C0
:1059F000E55BFB4F88EC90E0918380838981282FC1
:105A0000332785E290E0289FA001299F500D389F01
:105A1000500D1124CA01FC01EA5AFB4F82EA80832F
:105A20008981282F332785E290E0289FA001299FB4
:105A3000500D389F500D1124CA01FC01E95AFB4F4B
:105A400082EB80838981282F332785E290E0289F8D
:105A5000A001299F500D389F500D1124CA01FC014F
:105A6000E65AFB4F81E080838981282F332785E226
:105A700090E0289FA001299F500D389F500D1124C0
:105A8000CA01FC01E85AFB4F8FEF80838981282FE0
:105A9000332785E290E0289FA001299F500D389F71
:105AA000500D1124CA01FC01E75AFB4F87EA80839D
:105AB0008981282F332785E290E0289FA001299F24
:105AC000500D389F500D1124CA01FC01E55AFB4FBF
:105AD0008FE0808382E089838981282F332785E2C4
:105AE00090E0289FA001299F500D389F500D112450
:105AF000CA01FC01E75CFB4F81E080838981282F8C
:105B0000332785E290E0289FA001299F500D389F00
:105B1000500D1124CA01FC01E55BFB4F88EC90E0BD
:105B2000918380838981282F332785E290E0289F05
:105B3000A001299F500D389F500D1124CA01FC016E
:105B4000EA5AFB4F83EA80838981282F332785E235
:105B500090E0289FA001299F500D389F500D1124DF
:105B6000CA01FC01E95AFB4F83EB80838981282F0E
:105B7000332785E290E0289FA001299F500D389F90
:105B8000500D1124CA01FC01E65AFB4F81E08083CD
:105B90008981282F332785E290E0289FA001299F43
:105BA000500D389F500D1124CA01FC01E85AFB4FDB
:105BB0008FEF80838981282F332785E290E0289F0B
:105BC000A001299F500D389F500D1124CA01FC01DE
:105BD000E75AFB4F8FEF80838981282F332785E297
:105BE00090E0289FA001299F500D389F500D11244F
:105BF000CA01FC01E55AFB4F89E0808383E0898379
:105C00008981282F332785E290E0289FA001299FD2
:105C1000500D389F500D1124CA01FC01E75CFB4F69
:105C200081E080838981282F332785E290E0289FB7
:105C3000A001299F500D389F500D1124CA01FC016D
:105C4000E55BFB4F88EC90E0918380838981282F6E
:105C5000332785E290E0289FA001299F500D389FAF
:105C6000500D1124CA01FC01EA5AFB4F87EA8083D8
:105C70008981282F332785E290E0289FA001299F62
:105C8000500D389F500D1124CA01FC01E95AFB4FF9
:105C900087EB80838981282F332785E290E0289F36
:105CA000A001299F500D389F500D1124CA01FC01FD
:105CB000E65AFB4F81E080838981282F332785E2D4
:105CC00090E0289FA001299F500D389F500D11246E
:105CD000CA01FC01E85AFB4F8FEF80838981282F8E
:105CE000332785E290E0289FA001299F500D389F1F
:105CF000500D1124CA01FC01E75AFB4F8FEF80833E
:105D00008981282F332785E290E0289FA001299FD1
:105D1000500D389F500D1124CA01FC01E55AFB4F6C
:105D20008BE0808384E089838981282F332785E273
:105D300090E0289FA001299F500D389F500D1124FD
:105D4000CA01FC01E75CFB4F81E080838981282F39
:105D5000332785E290E0289FA001299F500D389FAE
:105D6000500D1124CA01FC01E55BFB4F88EC90E06B
:105D7000918380838981282F332785E290E0289FB3
:105D8000A001299F500D389F500D1124CA01FC011C
:105D9000EA5AFB4F81EA80838981282F332785E2E5
:105DA00090E0289FA001299F500D389F500D11248D
:105DB000CA01FC01E95AFB4F81EB80838981282FBE
:105DC000332785E290E0289FA001299F500D389F3E
:105DD000500D1124CA01FC01E65AFB4F81E080837B
:105DE0008981282F332785E290E0289FA001299FF1
:105DF000500D389F500D1124CA01FC01E85AFB4F89
:105E00008FEF80838981282F332785E290E0289FB8
:105E1000A001299F500D389F500D1124CA01FC018B
:105E2000E75AFB4F8FEF80838981282F332785E244
:105E300090E0289FA001299F500D389F500D1124FC
:105E4000CA01FC01E55AFB4F8EE0808385E089831F
:105E50008981282F332785E290E0289FA001299F80
:105E6000500D389F500D1124CA01FC01E75CFB4F17
:105E700081E080838981282F332785E290E0289F65
:105E8000A001299F500D389F500D1124CA01FC011B
:105E9000E55BFB4F88EC90E0918380838981282F1C
:105EA000332785E290E0289FA001299F500D389F5D
:105EB000500D1124CA01FC01EA5AFB4F85EA808388
:105EC0008981282F332785E290E0289FA001299F10
:105ED000500D389F500D1124CA01FC01E95AFB4FA7
:105EE00085EB80838981282F332785E290E0289FE6
:105EF000A001299F500D389F500D1124CA01FC01AB
:105F0000E65AFB4F81E080838981282F332785E281
:105F100090E0289FA001299F500D389F500D11241B
:105F2000CA01FC01E85AFB4F8FEF80838981282F3B
:105F3000332785E290E0289FA001299F500D389FCC
:105F4000500D1124CA01FC01E75AFB4F8FEF8083EB
:105F50008981282F332785E290E0289FA001299F7F
:105F6000500D389F500D1124CA01FC01E55AFB4F1A
:105F70008DE0808386E089838981282F332785E21D
:105F800090E0289FA001299F500D389F500D1124AB
:105F9000CA01FC01E75CFB4F81E080838981282FE7
:105FA000332785E290E0289FA001299F500D389F5C
:105FB000500D1124CA01FC01E55BFB4F88EC90E019
:105FC000918380838981282F332785E290E0289F61
:105FD000A001299F500D389F500D1124CA01FC01CA
:105FE000EA5AFB4F80EA80838981282F332785E294
:105FF00090E0289FA001299F500D389F500D11243B
:10600000CA01FC01E95AFB4F80EB80838981282F6C
:10601000332785E290E0289FA001299F500D389FEB
:10602000500D1124CA01FC01E65AFB4F10828981F0
:10603000282F332785E290E0289FA001299F500D4B
:10604000389F500D1124CA01FC01E85AFB4F8FEF15
:1060500080838981282F332785E290E0289FA00143
:10606000299F500D389F500D1124CA01FC01E75A99
:10607000FB4F85EA80838981282F332785E290E0D2
:10608000289FA001299F500D389F500D1124CA014F
:10609000FC01E55AFB4F86E0808387E08983898194
:1060A000282F332785E290E0289FA001299F500DDB
:1060B000389F500D1124CA01FC01E75CFB4F81E0C1
:1060C00080838981282F332785E290E0289FA001D3
:1060D000299F500D389F500D1124CA01FC01E55B2A
:1060E000FB4F88EC90E0918380838981282F3327B0
:1060F00085E290E0289FA001299F500D389F500D08
:106100001124CA01FC01EA5AFB4F85EA8083898188
:10611000282F332785E290E0289FA001299F500D6A
:10612000389F500D1124CA01FC01E95AFB4F85EB41
:1061300080838981282F332785E290E0289FA00162
:10614000299F500D389F500D1124CA01FC01E65AB9
:10615000FB4F10828981282F332785E290E0289F0A
:10616000A001299F500D389F500D1124CA01FC0138
:10617000E85AFB4F8FEF80838981282F332785E2F0
:1061800090E0289FA001299F500D389F500D1124A9
:10619000CA01FC01E75AFB4F8FEF80838981282FCA
:1061A000332785E290E0289FA001299F500D389F5A
:1061B000500D1124CA01FC01E55AFB4F84E0808395
:1061C00088E089838981282F332785E290E0289F02
:1061D000A001299F500D389F500D1124CA01FC01C8
:1061E000E75CFB4F81E080838981282F332785E29C
:1061F00090E0289FA001299F500D389F500D112439
:10620000CA01FC01E55BFB4F88EC90E09183808341
:106210008981282F332785E290E0289FA001299FBC
:10622000500D389F500D1124CA01FC01EA5AFB4F52
:1062300080EA80838981282F332785E290E0289F98
:10624000A001299F500D389F500D1124CA01FC0157
:10625000E95AFB4F80EB80838981282F332785E221
:1062600090E0289FA001299F500D389F500D1124C8
:10627000CA01FC01E65AFB4F81E080838981282F07
:10628000332785E290E0289FA001299F500D389F79
:10629000500D1124CA01FC01E85AFB4F8FEF808397
:1062A0008981282F332785E290E0289FA001299F2C
:1062B000500D389F500D1124CA01FC01E75AFB4FC5
:1062C00080EA80838981282F332785E290E0289F08
:1062D000A001299F500D389F500D1124CA01FC01C7
:1062E000E55AFB4F8AE0808389E089838981282FE2
:1062F000332785E290E0289FA001299F500D389F09
:10630000500D1124CA01FC01E75CFB4F81E0808342
:106310008981282F332785E290E0289FA001299FBB
:10632000500D389F500D1124CA01FC01E55BFB4F55
:1063300088EC90E0918380838981282F332785E240
:1063400090E0289FA001299F500D389F500D1124E7
:10635000CA01FC01EA5AFB4F80EB80838981282F18
:10636000332785E290E0289FA001299F500D389F98
:10637000500D1124CA01FC01E95AFB4F84EB8083C4
:106380008981282F332785E290E0289FA001299F4B
:10639000500D389F500D1124CA01FC01E65AFB4FE5
:1063A00085E080838981282F332785E290E0289F2C
:1063B000A001299F500D389F500D1124CA01FC01E6
:1063C000E85AFB4F8FEF80838981282F332785E29E
:1063D00090E0289FA001299F500D389F500D112457
:1063E000CA01FC01E75AFB4F8FEF80838981282F78
:1063F000332785E290E0289FA001299F500D389F08
:10640000500D1124CA01FC01E55AFB4F82E1808343
:106410008AE089838981282F332785E290E0289FAD
:10642000A001299F500D389F500D1124CA01FC0175
:10643000E75CFB4F81E080838981282F332785E249
:1064400090E0289FA001299F500D389F500D1124E6
:10645000CA01FC01E55BFB4F88EC90E091838083EF
:106460008981282F332785E290E0289FA001299F6A
:10647000500D389F500D1124CA01FC01EA5AFB4F00
:1064800084EA80838981282F332785E290E0289F42
:10649000A001299F500D389F500D1124CA01FC0105
:1064A000E95AFB4F84EB80838981282F332785E2CB
:1064B00090E0289FA001299F500D389F500D112476
:1064C000CA01FC01E65AFB4F81E080838981282FB5
:1064D000332785E290E0289FA001299F500D389F27
:1064E000500D1124CA01FC01E85AFB4F8FEF808345
:1064F0008981282F332785E290E0289FA001299FDA
:10650000500D389F500D1124CA01FC01E75AFB4F72
:1065100083EA80838981282F332785E290E0289FB2
:10652000A001299F500D389F500D1124CA01FC0174
:10653000E55AFB4F88E080838BE089838981282F8F
:10654000332785E290E0289FA001299F500D389FB6
:10655000500D1124CA01FC01E75CFB4F81E08083F0
:106560008981282F332785E290E0289FA001299F69
:10657000500D389F500D1124CA01FC01E55BFB4F03
:1065800088EC90E0918380838981282F332785E2EE
:1065900090E0289FA001299F500D389F500D112495
:1065A000CA01FC01EA5AFB4F86EA80838981282FC1
:1065B000332785E290E0289FA001299F500D389F46
:1065C000500D1124CA01FC01E95AFB4F86EB808370
:1065D0008981282F332785E290E0289FA001299FF9
:1065E000500D389F500D1124CA01FC01E65AFB4F93
:1065F00010828981282F332785E290E0289FA0010F
:10660000299F500D389F500D1124CA01FC01E85AF2
:10661000FB4F8FEF80838981282F332785E290E01D
:10662000289FA001299F500D389F500D1124CA01A9
:10663000FC01E75AFB4F84EA80838981282F3327A6
:1066400085E290E0289FA001299F500D389F500DB2
:106650001124CA01FC01E55AFB4F81E080838CE0E4
:1066600089838981282F332785E290E0289FA00124
:10667000299F500D389F500D1124CA01FC01E75C81
:10668000FB4F81E080838981282F332785E290E0CA
:10669000289FA001299F500D389F500D1124CA0139
:1066A000FC01E55BFB4F88EC90E09183808389815E
:1066B000282F332785E290E0289FA001299F500DC5
:1066C000389F500D1124CA01FC01EA5AFB4F86EA9B
:1066D00080838981282F332785E290E0289FA001BD
:1066E000299F500D389F500D1124CA01FC01E95A11
:1066F000FB4F86EB80838981282F332785E290E04A
:10670000289FA001299F500D389F500D1124CA01C8
:10671000FC01E65AFB4F81E080838981282F3327D3
:1067200085E290E0289FA001299F500D389F500DD1
:106730001124CA01FC01E85AFB4F8FEF8083898145
:10674000282F332785E290E0289FA001299F500D34
:10675000389F500D1124CA01FC01E75AFB4F81EA12
:1067600080838981282F332785E290E0289FA0012C
:10677000299F500D389F500D1124CA01FC01E55A84
:10678000FB4F8CE080838DE089838981282F33271C
:1067900085E290E0289FA001299F500D389F500D61
:1067A0001124CA01FC01E75CFB4F81E080838981F1
:1067B000282F332785E290E0289FA001299F500DC4
:1067C000389F500D1124CA01FC01E55BFB4F88EC9A
:1067D00090E0918380838981282F332785E290E0A0
:1067E000289FA001299F500D389F500D1124CA01E8
:1067F000FC01EA5AFB4F87EA80838981282F3327DF
:1068000085E290E0289FA001299F500D389F500DF0
:106810001124CA01FC01E95AFB4F87EB808389816F
:10682000282F332785E290E0289FA001299F500D53
:10683000389F500D1124CA01FC01E65AFB4F10820B
:106840008981282F332785E290E0289FA001299F86
:10685000500D389F500D1124CA01FC01E85AFB4F1E
:106860008FEF80838981282F332785E290E0289F4E
:10687000A001299F500D389F500D1124CA01FC0121
:10688000E75AFB4F8FEF80838981282F332785E2DA
:1068900090E0289FA001299F500D389F500D112492
:1068A000CA01FC01E55AFB4F82E080838EE08983B8
:1068B0008981282F332785E290E0289FA001299F16
:1068C000500D389F500D1124CA01FC01E75CFB4FAD
:1068D00081E080838981282F332785E290E0289FFB
:1068E000A001299F500D389F500D1124CA01FC01B1
:1068F000E55BFB4F88EC90E0918380838981282FB2
:10690000332785E290E0289FA001299F500D389FF2
:10691000500D1124CA01FC01EA5AFB4F81EA808321
:106920008981282F332785E290E0289FA001299FA5
:10693000500D389F500D1124CA01FC01E95AFB4F3C
:1069400081EB80838981282F332785E290E0289F7F
:10695000A001299F500D389F500D1124CA01FC0140
:10696000E65AFB4F10828981282F332785E290E079
:10697000289FA001299F500D389F500D1124CA0156
:10698000FC01E85AFB4F8FEF80838981282F332742
:1069900085E290E0289FA001299F500D389F500D5F
:1069A0001124CA01FC01E75AFB4F8FEF80838981D4
:1069B000282F332785E290E0289FA001299F500DC2
:1069C000389F500D1124CA01FC01E55AFB4F87E0A6
:1069D00080838FE089838981282F332785E290E0A7
:1069E000289FA001299F500D389F500D1124CA01E6
:1069F000FC01E75CFB4F81E080838981282F3327EE
:106A000085E290E0289FA001299F500D389F500DEE
:106A10001124CA01FC01E55BFB4F88EC90E09183F7
:106A200080838981282F332785E290E0289FA00169
:106A3000299F500D389F500D1124CA01FC01EA5ABC
:106A4000FB4F81EB80838981282F332785E290E0FB
:106A5000289FA001299F500D389F500D1124CA0175
:106A6000FC01E95AFB4F85EB80838981282F33276E
:106A700085E290E0289FA001299F500D389F500D7E
:106A80001124CA01FC01E65AFB4F85E0808389810D
:106A9000282F332785E290E0289FA001299F500DE1
:106AA000389F500D1124CA01FC01E85AFB4F8FEFAB
:106AB00080838981282F332785E290E0289FA001D9
:106AC000299F500D389F500D1124CA01FC01E75A2F
:106AD000FB4F8FEF80838981282F332785E290E059
:106AE000289FA001299F500D389F500D1124CA01E5
:106AF000FC01E55AFB4F81E1808380E18983898134
:106B0000282F332785E290E0289FA001299F500D70
:106B1000389F500D1124CA01FC01E75CFB4F81E056
:106B200080838981282F332785E290E0289FA00168
:106B3000299F500D389F500D1124CA01FC01E55BBF
:106B4000FB4F88EC90E0918380838981282F332745
:106B500085E290E0289FA001299F500D389F500D9D
:106B60001124CA01FC01EA5AFB4F84EA808389811F
:106B7000282F332785E290E0289FA001299F500D00
:106B8000389F500D1124CA01FC01E95AFB4F84EBD8
:106B900080838981282F332785E290E0289FA001F8
:106BA000299F500D389F500D1124CA01FC01E65A4F
:106BB000FB4F10828981282F332785E290E0289FA0
:106BC000A001299F500D389F500D1124CA01FC01CE
:106BD000E85AFB4F8FEF80838981282F332785E286
:106BE00090E0289FA001299F500D389F500D11243F
:106BF000CA01FC01E75AFB4F86EA80838981282F6E
:106C0000332785E290E0289FA001299F500D389FEF
:106C1000500D1124CA01FC01E55AFB4F85E0808329
:106C200081E189838981282F332785E290E0289F9D
:106C3000A001299F500D389F500D1124CA01FC015D
:106C4000E75CFB4F81E080838981282F332785E231
:106C500090E0289FA001299F500D389F500D1124CE
:106C6000CA01FC01E55BFB4F88EC90E091838083D7
:106C70008981282F332785E290E0289FA001299F52
:106C8000500D389F500D1124CA01FC01EA5AFB4FE8
:106C900083EA80838981282F332785E290E0289F2B
:106CA000A001299F500D389F500D1124CA01FC01ED
:106CB000E95AFB4F83EB80838981282F332785E2B4
:106CC00090E0289FA001299F500D389F500D11245E
:106CD000CA01FC01E65AFB4F10828981282F332715
:106CE00085E290E0289FA001299F500D389F500D0C
:106CF0001124CA01FC01E85AFB4F8FEF8083898180
:106D0000282F332785E290E0289FA001299F500D6E
:106D1000389F500D1124CA01FC01E75AFB4F8FEF39
:106D200080838981282F332785E290E0289FA00166
:106D3000299F500D389F500D1124CA01FC01E55ABE
:106D4000FB4F108282E189838981282F332785E2D6
:106D500090E0289FA001299F500D389F500D1124CD
:106D6000CA01FC01E75CFB4F80E480838981282F06
:106D7000332785E290E0289FA001299F500D389F7E
:106D8000500D1124CA01FC01E55BFB4F8FEF9FEF13
:106D9000918380838981282F332785E290E0289F83
:106DA000A001299F500D389F500D1124CA01FC01EC
:106DB000EA5AFB4F87EA80838981282F332785E2AF
:106DC00090E0289FA001299F500D389F500D11245D
:106DD000CA01FC01E95AFB4F84EB80838981282F8B
:106DE000332785E290E0289FA001299F500D389F0E
:106DF000500D1124CA01FC01E65AFB4F83E0808349
:106E00008981282F332785E290E0289FA001299FC0
:106E1000500D389F500D1124CA01FC01E85AFB4F58
:106E200086EA80838981282F332785E290E0289F96
:106E3000A001299F500D389F500D1124CA01FC015B
:106E4000E75AFB4F8FEF80838981282F332785E214
:106E500090E0289FA001299F500D389F500D1124CC
:106E6000CA01FC01E55AFB4F8FEF808383E18983E0
:106E70008981282F332785E290E0289FA001299F50
:106E8000500D389F500D1124CA01FC01E75CFB4FE7
:106E900080E480838981282F332785E290E0289F32
:106EA000A001299F500D389F500D1124CA01FC01EB
:106EB000E55BFB4F8FEF9FEF918380838981282FC4
:106EC000332785E290E0289FA001299F500D389F2D
:106ED000500D1124CA01FC01EA5AFB4F86EA808357
:106EE0008981282F332785E290E0289FA001299FE0
:106EF000500D389F500D1124CA01FC01E95AFB4F77
:106F000085EB80838981282F332785E290E0289FB5
:106F1000A001299F500D389F500D1124CA01FC017A
:106F2000E65AFB4F83E080838981282F332785E24F
:106F300090E0289FA001299F500D389F500D1124EB
:106F4000CA01FC01E85AFB4F86EA80838981282F19
:106F5000332785E290E0289FA001299F500D389F9C
:106F6000500D1124CA01FC01E75AFB4F8FEF8083BB
:106F70008981282F332785E290E0289FA001299F4F
:106F8000500D389F500D1124CA01FC01E55AFB4FEA
:106F90008FEF808384E189838981282F332785E2DD
:106FA00090E0289FA001299F500D389F500D11247B
:106FB000CA01FC01E75CFB4F80E480838981282FB4
:106FC000332785E290E0289FA001299F500D389F2C
:106FD000500D1124CA01FC01E55BFB4F8FEF9FEFC1
:106FE000918380838981282F332785E290E0289F31
:106FF000A001299F500D389F500D1124CA01FC019A
:10700000EA5AFB4F85EA80838981282F332785E25E
:1070100090E0289FA001299F500D389F500D11240A
:10702000CA01FC01E95AFB4F86EB80838981282F36
:10703000332785E290E0289FA001299F500D389FBB
:10704000500D1124CA01FC01E65AFB4F83E08083F6
:107050008981282F332785E290E0289FA001299F6E
:10706000500D389F500D1124CA01FC01E85AFB4F06
:1070700087EA80838981282F332785E290E0289F43
:10708000A001299F500D389F500D1124CA01FC0109
:10709000E75AFB4F8FEF80838981282F332785E2C2
:1070A00090E0289FA001299F500D389F500D11247A
:1070B000CA01FC01E55AFB4F8FEF808385E189838C
:1070C0008981282F332785E290E0289FA001299FFE
:1070D000500D389F500D1124CA01FC01E75CFB4F95
:1070E00080E480838981282F332785E290E0289FE0
:1070F000A001299F500D389F500D1124CA01FC0199
:10710000E55BFB4F8FEF9FEF918380838981282F71
:10711000332785E290E0289FA001299F500D389FDA
:10712000500D1124CA01FC01EA5AFB4F84EA808306
:107130008981282F332785E290E0289FA001299F8D
:10714000500D389F500D1124CA01FC01E95AFB4F24
:1071500087EB80838981282F332785E290E0289F61
:10716000A001299F500D389F500D1124CA01FC0128
:10717000E65AFB4F83E080838981282F332785E2FD
:1071800090E0289FA001299F500D389F500D112499
:10719000CA01FC01E85AFB4F87EA80838981282FC6
:1071A000332785E290E0289FA001299F500D389F4A
:1071B000500D1124CA01FC01E75AFB4F8FEF808369
:1071C0008981282F332785E290E0289FA001299FFD
:1071D000500D389F500D1124CA01FC01E55AFB4F98
:1071E0008FEF808386E189838981282F332785E289
:1071F00090E0289FA001299F500D389F500D112429
:10720000CA01FC01E75CFB4F80E480838981282F61
:10721000332785E290E0289FA001299F500D389FD9
:10722000500D1124CA01FC01E55BFB4F8FEF9FEF6E
:10723000918380838981282F332785E290E0289FDE
:10724000A001299F500D389F500D1124CA01FC0147
:10725000EA5AFB4F80EA80838981282F332785E211
:1072600090E0289FA001299F500D389F500D1124B8
:10727000CA01FC01E95AFB4F83EB80838981282FE7
:10728000332785E290E0289FA001299F500D389F69
:10729000500D1124CA01FC01E65AFB4F83E08083A4
:1072A0008981282F332785E290E0289FA001299F1C
:1072B000500D389F500D1124CA01FC01E85AFB4FB4
:1072C00085EA80838981282F332785E290E0289FF3
:1072D000A001299F500D389F500D1124CA01FC01B7
:1072E000E75AFB4F8FEF80838981282F332785E270
:1072F00090E0289FA001299F500D389F500D112428
:10730000CA01FC01E55AFB4F8FEF808387E1898337
:107310008981282F332785E290E0289FA001299FAB
:10732000500D389F500D1124CA01FC01E75CFB4F42
:1073300080E480838981282F332785E290E0289F8D
:10734000A001299F500D389F500D1124CA01FC0146
:10735000E55BFB4F8FEF9FEF918380838981282F1F
:10736000332785E290E0289FA001299F500D389F88
:10737000500D1124CA01FC01EA5AFB4F81EA8083B7
:107380008981282F332785E290E0289FA001299F3B
:10739000500D389F500D1124CA01FC01E95AFB4FD2
:1073A00082EB80838981282F332785E290E0289F14
:1073B000A001299F500D389F500D1124CA01FC01D6
:1073C000E65AFB4F83E080838981282F332785E2AB
:1073D00090E0289FA001299F500D389F500D112447
:1073E000CA01FC01E85AFB4F85EA80838981282F76
:1073F000332785E290E0289FA001299F500D389FF8
:10740000500D1124CA01FC01E75AFB4F8FEF808316
:107410008981282F332785E290E0289FA001299FAA
:10742000500D389F500D1124CA01FC01E55AFB4F45
:107430008FEF808388E189838981282F332785E234
:1074400090E0289FA001299F500D389F500D1124D6
:10745000CA01FC01E75CFB4F80E480838981282F0F
:10746000332785E290E0289FA001299F500D389F87
:10747000500D1124CA01FC01E55BFB4F8FEF9FEF1C
:10748000918380838981282F332785E290E0289F8C
:10749000A001299F500D389F500D1124CA01FC01F5
:1074A000EA5AFB4F82EA80838981282F332785E2BD
:1074B00090E0289FA001299F500D389F500D112466
:1074C000CA01FC01E95AFB4F81EB80838981282F97
:1074D000332785E290E0289FA001299F500D389F17
:1074E000500D1124CA01FC01E65AFB4F83E0808352
:1074F0008981282F332785E290E0289FA001299FCA
:10750000500D389F500D1124CA01FC01E85AFB4F61
:1075100084EA80838981282F332785E290E0289FA1
:10752000A001299F500D389F500D1124CA01FC0164
:10753000E75AFB4F8FEF80838981282F332785E21D
:1075400090E0289FA001299F500D389F500D1124D5
:10755000CA01FC01E55AFB4F8FEF808389E18983E3
:107560008981282F332785E290E0289FA001299F59
:10757000500D389F500D1124CA01FC01E75CFB4FF0
:1075800080E480838981282F332785E290E0289F3B
:10759000A001299F500D389F500D1124CA01FC01F4
:1075A000E55BFB4F8FEF9FEF918380838981282FCD
:1075B000332785E290E0289FA001299F500D389F36
:1075C000500D1124CA01FC01EA5AFB4F83EA808363
:1075D0008981282F332785E290E0289FA001299FE9
:1075E000500D389F500D1124CA01FC01E95AFB4F80
:1075F00080EB80838981282F332785E290E0289FC4
:10760000A001299F500D389F500D1124CA01FC0183
:10761000E65AFB4F83E080838981282F332785E258
:1076200090E0289FA001299F500D389F500D1124F4
:10763000CA01FC01E85AFB4F84EA80838981282F24
:10764000332785E290E0289FA001299F500D389FA5
:10765000500D1124CA01FC01E75AFB4F8FEF8083C4
:107660008981282F332785E290E0289FA001299F58
:10767000500D389F500D1124CA01FC01E55AFB4FF3
:107680008FEF80838AE189838981282F332785E2E0
:1076900090E0289FA001299F500D389F500D112484
:1076A000CA01FC01E75CFB4F80E480838981282FBD
:1076B000332785E290E0289FA001299F500D389F35
:1076C000500D1124CA01FC01E55BFB4F8FEF9FEFCA
:1076D000918380838981282F332785E290E0289F3A
:1076E000A001299F500D389F500D1124CA01FC01A3
:1076F000EA5AFB4F80EA80838981282F332785E26D
:1077000090E0289FA001299F500D389F500D112413
:10771000CA01FC01E95AFB4F83EB80838981282F42
:10772000332785E290E0289FA001299F500D389FC4
:10773000500D1124CA01FC01E65AFB4F82E0808300
:107740008981282F332785E290E0289FA001299F77
:10775000500D389F500D1124CA01FC01E85AFB4F0F
:1077600085EB80838981282F332785E290E0289F4D
:10777000A001299F500D389F500D1124CA01FC0112
:10778000E75AFB4F8FEF80838981282F332785E2CB
:1077900090E0289FA001299F500D389F500D112483
:1077A000CA01FC01E55AFB4F8FEF80838BE189838F
:1077B0008981282F332785E290E0289FA001299F07
:1077C000500D389F500D1124CA01FC01E75CFB4F9E
:1077D00080E480838981282F332785E290E0289FE9
:1077E000A001299F500D389F500D1124CA01FC01A2
:1077F000E55BFB4F8FEF9FEF918380838981282F7B
:10780000332785E290E0289FA001299F500D389FE3
:10781000500D1124CA01FC01EA5AFB4F81EA808312
:107820008981282F332785E290E0289FA001299F96
:10783000500D389F500D1124CA01FC01E95AFB4F2D
:1078400082EB80838981282F332785E290E0289F6F
:10785000A001299F500D389F500D1124CA01FC0131
:10786000E65AFB4F82E080838981282F332785E207
:1078700090E0289FA001299F500D389F500D1124A2
:10788000CA01FC01E85AFB4F85EB80838981282FD0
:10789000332785E290E0289FA001299F500D389F53
:1078A000500D1124CA01FC01E75AFB4F8FEF808372
:1078B0008981282F332785E290E0289FA001299F06
:1078C000500D389F500D1124CA01FC01E55AFB4FA1
:1078D0008FEF80838CE189838981282F332785E28C
:1078E00090E0289FA001299F500D389F500D112432
:1078F000CA01FC01E75CFB4F80E480838981282F6B
:10790000332785E290E0289FA001299F500D389FE2
:10791000500D1124CA01FC01E55BFB4F8FEF9FEF77
:10792000918380838981282F332785E290E0289FE7
:10793000A001299F500D389F500D1124CA01FC0150
:10794000EA5AFB4F82EA80838981282F332785E218
:1079500090E0289FA001299F500D389F500D1124C1
:10796000CA01FC01E95AFB4F81EB80838981282FF2
:10797000332785E290E0289FA001299F500D389F72
:10798000500D1124CA01FC01E65AFB4F82E08083AE
:107990008981282F332785E290E0289FA001299F25
:1079A000500D389F500D1124CA01FC01E85AFB4FBD
:1079B00084EB80838981282F332785E290E0289FFC
:1079C000A001299F500D389F500D1124CA01FC01C0
:1079D000E75AFB4F8FEF80838981282F332785E279
:1079E00090E0289FA001299F500D389F500D112431
:1079F000CA01FC01E55AFB4F8FEF80838DE189833B
:107A00008981282F332785E290E0289FA001299FB4
:107A1000500D389F500D1124CA01FC01E75CFB4F4B
:107A200080E480838981282F332785E290E0289F96
:107A3000A001299F500D389F500D1124CA01FC014F
:107A4000E55BFB4F8FEF9FEF918380838981282F28
:107A5000332785E290E0289FA001299F500D389F91
:107A6000500D1124CA01FC01EA5AFB4F83EA8083BE
:107A70008981282F332785E290E0289FA001299F44
:107A8000500D389F500D1124CA01FC01E95AFB4FDB
:107A900080EB80838981282F332785E290E0289F1F
:107AA000A001299F500D389F500D1124CA01FC01DF
:107AB000E65AFB4F82E080838981282F332785E2B5
:107AC00090E0289FA001299F500D389F500D112450
:107AD000CA01FC01E85AFB4F84EB80838981282F7F
:107AE000332785E290E0289FA001299F500D389F01
:107AF000500D1124CA01FC01E75AFB4F8FEF808320
:107B00008981282F332785E290E0289FA001299FB3
:107B1000500D389F500D1124CA01FC01E55AFB4F4E
:107B20008FEF80838EE189838981282F332785E237
:107B300090E0289FA001299F500D389F500D1124DF
:107B4000CA01FC01E75CFB4F80E480838981282F18
:107B5000332785E290E0289FA001299F500D389F90
:107B6000500D1124CA01FC01E55BFB4F8FEF9FEF25
:107B7000918380838981282F332785E290E0289F95
:107B8000A001299F500D389F500D1124CA01FC01FE
:107B9000EA5AFB4F87EA80838981282F332785E2C1
:107BA00090E0289FA001299F500D389F500D11246F
:107BB000CA01FC01E95AFB4F84EB80838981282F9D
:107BC000332785E290E0289FA001299F500D389F20
:107BD000500D1124CA01FC01E65AFB4F82E080835C
:107BE0008981282F332785E290E0289FA001299FD3
:107BF000500D389F500D1124CA01FC01E85AFB4F6B
:107C000086EB80838981282F332785E290E0289FA7
:107C1000A001299F500D389F500D1124CA01FC016D
:107C2000E75AFB4F8FEF80838981282F332785E226
:107C300090E0289FA001299F500D389F500D1124DE
:107C4000CA01FC01E55AFB4F8FEF80838FE18983E6
:107C50008981282F332785E290E0289FA001299F62
:107C6000500D389F500D1124CA01FC01E75CFB4FF9
:107C700080E480838981282F332785E290E0289F44
:107C8000A001299F500D389F500D1124CA01FC01FD
:107C9000E55BFB4F8FEF9FEF918380838981282FD6
:107CA000332785E290E0289FA001299F500D389F3F
:107CB000500D1124CA01FC01EA5AFB4F86EA808369
:107CC0008981282F332785E290E0289FA001299FF2
:107CD000500D389F500D1124CA01FC01E95AFB4F89
:107CE00085EB80838981282F332785E290E0289FC8
:107CF000A001299F500D389F500D1124CA01FC018D
:107D0000E65AFB4F82E080838981282F332785E262
:107D100090E0289FA001299F500D389F500D1124FD
:107D2000CA01FC01E85AFB4F86EB80838981282F2A
:107D3000332785E290E0289FA001299F500D389FAE
:107D4000500D1124CA01FC01E75AFB4F8FEF8083CD
:107D50008981282F332785E290E0289FA001299F61
:107D6000500D389F500D1124CA01FC01E55AFB4FFC
:107D70008FEF808380E289838981282F332785E2F2
:107D800090E0289FA001299F500D389F500D11248D
:107D9000CA01FC01E75CFB4F80E480838981282FC6
:107DA000332785E290E0289FA001299F500D389F3E
:107DB000500D1124CA01FC01E55BFB4F8FEF9FEFD3
:107DC000918380838981282F332785E290E0289F43
:107DD000A001299F500D389F500D1124CA01FC01AC
:107DE000EA5AFB4F85EA80838981282F332785E271
:107DF00090E0289FA001299F500D389F500D11241D
:107E0000CA01FC01E95AFB4F86EB80838981282F48
:107E1000332785E290E0289FA001299F500D389FCD
:107E2000500D1124CA01FC01E65AFB4F82E0808309
:107E30008981282F332785E290E0289FA001299F80
:107E4000500D389F500D1124CA01FC01E85AFB4F18
:107E500087EB80838981282F332785E290E0289F54
:107E6000A001299F500D389F500D1124CA01FC011B
:107E7000E75AFB4F8FEF80838981282F332785E2D4
:107E800090E0289FA001299F500D389F500D11248C
:107E9000CA01FC01E55AFB4F8FEF808381E28983A1
:107EA0008981282F332785E290E0289FA001299F10
:107EB000500D389F500D1124CA01FC01E75CFB4FA7
:107EC00080E480838981282F332785E290E0289FF2
:107ED000A001299F500D389F500D1124CA01FC01AB
:107EE000E55BFB4F8FEF9FEF918380838981282F84
:107EF000332785E290E0289FA001299F500D389FED
:107F0000500D1124CA01FC01EA5AFB4F84EA808318
:107F10008981282F332785E290E0289FA001299F9F
:107F2000500D389F500D1124CA01FC01E95AFB4F36
:107F300087EB80838981282F332785E290E0289F73
:107F4000A001299F500D389F500D1124CA01FC013A
:107F5000E65AFB4F82E080838981282F332785E210
:107F600090E0289FA001299F500D389F500D1124AB
:107F7000CA01FC01E85AFB4F87EB80838981282FD7
:107F8000332785E290E0289FA001299F500D389F5C
:107F9000500D1124CA01FC01E75AFB4F8FEF80837B
:107FA0008981282F332785E290E0289FA001299F0F
:107FB000500D389F500D1124CA01FC01E55AFB4FAA
:107FC0008FEF808319828981823208F08DC1898187
:107FD000282F332785E290E0289FA001299F500D8C
:107FE000389F500D1124CA01FC01E35BFB4F118245
:107FF00010828981282F332785E290E0289FA001F5
:10800000299F500D389F500D1124CA01FC01E35CDB
:10801000FB4F80818F7D80838981282F332785E2E4
:1080200090E0289FA001299F500D389F500D1124EA
:10803000CA01FC01E35CFB4F80818E7F80838981D4
:10804000282F332785E290E0289FA001299F500D1B
:10805000389F500D1124CA01FC01E35CFB4F808165
:108060008D7F80838981282F332785E290E0289FA8
:10807000A001299F500D389F500D1124CA01FC0109
:10808000E85BFB4F10828981282F332785E290E03F
:10809000289FA001299F500D389F500D1124CA011F
:1080A000FC01E15BFB4F10828981282F332785E299
:1080B00090E0289FA001299F500D389F500D11245A
:1080C000CA01FC01E65CFB4F8FE080838981282F89
:1080D000332785E290E0289FA001299F500D389F0B
:1080E000500D1124CA01FC01E45AFB4F1182108289
:1080F0008981282F332785E290E0289FA001299FBE
:10810000500D389F500D1124CA01FC01EA5BFB4F52
:10811000118210828981282F332785E290E0289FE1
:10812000A001299F500D389F500D1124CA01FC0158
:10813000EB5BFB4F10828981282F332785E290E08B
:10814000289FA001299F500D389F500D1124CA016E
:10815000FC01ED5BFB4F118210828981282F3327B0
:1081600085E290E0289FA001299F500D389F500D77
:108170001124CA01FC01EE5BFB4F10828981282F7C
:10818000332785E290E0289FA001299F500D389F5A
:10819000500D1124CA01FC01E35CFB4F80818B7FF1
:1081A00080838981282F332785E290E0289FA001D2
:1081B000299F500D389F500D1124CA01FC01E05B2E
:1081C000FB4F10828981282F332785E290E0289F7A
:1081D000A001299F500D389F500D1124CA01FC01A8
:1081E000E05CFB4F10828981282F332785E290E0E5
:1081F000289FA001299F500D389F500D1124CA01BE
:10820000FC01EF5BFB4F81E280838981282F3327BC
:1082100085E290E0289FA001299F500D389F500DC6
:108220001124CA01FC01E15CFB4F8EE1808389814E
:10823000282F332785E290E0289FA001299F500D29
:10824000389F500D1124CA01FC01E25CFB4F80E114
:1082500080838981282F332785E290E0289FA00121
:10826000299F500D389F500D1124CA01FC01E55C77
:10827000FB4F8FE080838981282F332785E290E0B0
:10828000289FA001299F500D389F500D1124CA012D
:10829000FC01EF5AFB4F118210828981282F33276E
:1082A00085E290E0289FA001299F500D389F500D36
:1082B0001124CA01FC01ED5AFB4F11821082898101
:1082C000282F332785E290E0289FA001299F500D99
:1082D000389F500D1124CA01FC01EB5AFB4F10824C
:1082E00089818F5F89836FCE21960FB6F894DEBFA8
:1082F0000FBECDBFDF91CF910895CF93DF93CDB760
:10830000DEB721970FB6F894DEBF0FBECDBF42E1B6
:1083100050E060E070E083E299E00E94E9BC83E213
:1083200099E00E94626B19828981823188F4898187
:10833000282F3327C901820F931FFC01EB5CF64FF6
:1083400088EB91E09183808389818F5F8983ECCF73
:1083500085E399E00E94D46B21960FB6F894DEBFB6
:108360000FBECDBFDF91CF910895CF93DF93CDB7EF
:10837000DEB7CE5DD0400FB6F894DEBF0FBECDBFE6
:10838000198219828981823208F044C0FE01E959BC
:10839000FF4F1082FE01E959FF4F88EC8183FE01F7
:1083A000E959FF4F1282FE01E959FF4F15821482ED
:1083B000FE01E959FF4F1682FE01E959FF4F80E1A6
:1083C0008383FE01E959FF4F178299818FE0989FBF
:1083D000C00111249C012C553C4FCE0189599F4F5F
:1083E0000896B9010E94C8BCFE01E959FF4F178ADF
:1083F000FE01E959FF4F108E8981282F2F5FCE0192
:1084000089599F4F622F0E949269A89589818F5F39
:108410008983B8CFFE01E058FF4F84E68083FE01D8
:10842000E058FF4F88E78183CE0180589F4F029626
:108430004CE050E06FEF70E00E94E9BCCE01805844
:108440009F4F0E944866FE01E257FF4F81EC8083F8
:10845000CE0182579F4F019644E150E06FEF70E0EC
:108460000E94E9BCFE01E257FF4F158AFE01E25768
:10847000FF4F8AE0868BCE0182579F4F479644E19B
:1084800050E06FEF70E00E94E9BCCE0182579F4F31
:108490000E94C666A895198289818B3020F5CE018D
:1084A000039644E150E060E070E00E94E9BC9981ED
:1084B0008FE0989FC001112481509D4F9E012D5F38
:1084C0003F4FBC01C9010E94C8BC81E08A8B9E015C
:1084D0002D5F3F4F89818F5FB9010E94816A898139
:1084E0008F5F8983D9CFA89519828981853008F05B
:1084F00052C0CE0187549F4F0C964FE050E060E091
:1085000070E00E94E9BC99818FE0989FC00111241E
:108510009C012C543D4FCE0187549F4F0C96B901BE
:108520000E94C8BCFE01E754FF4F1082FE01E754D1
:10853000FF4F1182FE01E754FF4F1282FE01E75404
:10854000FF4F81E08383FE01E754FF4F81E0848386
:10855000FE01E754FF4F8AE085831A828A818630C4
:1085600078F49E0127543F4F8A819927820F931FE9
:10857000FC0136968FEF80838A818F5F8A83EECFEE
:10858000CE0187549F4FBC0189810E94AA678981CF
:108590008F5F8983AACF48E050E060E070E086EA10
:1085A00099E00E94E9BC86EA99E00E9438670E943F
:1085B0009A5CA89548E050E060E070E082ED9DE0B4
:1085C0000E94E9BC81E08093D60D8EE18093D70DA7
:1085D00082E38093D90DFE01EC52FF4F82ED9DE0C6
:1085E00091838083FE01EA52FF4F8EEA9EE09183E1
:1085F0008083FE01E852FF4F88E090E09183808302
:10860000DE01A652BF4FFE01E852FF4F80819181EB
:108610008D939C939E0126523F4FF9018081918159
:10862000FE01EA52FF4FA081B181FE01EC52FF4FE3
:108630000190F081E02DC352DF4FF983E883CD5DD7
:10864000D040C352DF4FE881F981CD5DD040019722
:1086500024F001900E94D1BDFACFAF01F9019183BE
:108660008083FE01EA52FF4FCD0191838083FE019A
:10867000EC52FF4FCA0191838083CE01479640E5BB
:1086800050E060E070E00E94E9BCCE01479603969E
:1086900060E271E00E94F3BCCE01479647966CE21F
:1086A00071E00E94F3BCCE0147968B9668E371E0BF
:1086B0000E94F3BCCE014796CF9664E471E00E941D
:1086C000F3BCFE01E652FF4FCE01479691838083B3
:1086D000FE01E852FF4F8EEC9EE091838083FE0105
:1086E000EA52FF4F80E590E091838083DE01AC5237
:1086F000BF4FFE01EA52FF4F808191818D939C9381
:108700009E012C523F4FF90180819181FE01E85278
:10871000FF4FA081B181FE01E652FF4F0190F08131
:10872000E02DC352DF4FF983E883CD5DD040C352C3
:10873000DF4FE881F981CD5DD040019724F00190B1
:108740000E94D1BDFACFAF01F90191838083FE0170
:10875000E852FF4FCD0191838083FE01E652FF4F27
:10876000CA01918380834CE050E060E070E08DEDC1
:108770009DE00E94E9BCC252DF4F0FB6F894DEBF05
:108780000FBECDBFDF91CF910895CF93DF93CDB7CB
:10879000DEB7C354D0400FB6F894DEBF0FBECDBFD6
:1087A000198219828981823208F0A6C08981282F16
:1087B0002F5FCE010296622F0E94006A8981282FC6
:1087C000332785E290E0289FA001299F500D389F14
:1087D000500D1124CA01FC01E55BFB4F8A819927EA
:1087E000382F22278B819927820F931F91838083B3
:1087F0008981282F332785E290E0289FF001299F67
:10880000F00D389FF00D1124CF01FC01E15CFB4F0E
:108810008C8180838981282F332785E290E0289FEF
:10882000A001299F500D389F500D1124CA01FC0151
:10883000EF5BFB4F898580838981282F332785E271
:1088400090E0289FF001299FF00D389FF00D112432
:10885000CF01FC01E25CFB4F8D8180838981282F51
:10886000332785E290E0289FA001299F500D389F73
:10887000500D1124CA01FC01EB5BFB4F898D8083F5
:108880008981282F332785E290E0289FF001299FD6
:10889000F00D389FF00D1124CF01FC01EE5BFB4F72
:1088A0008A8D80838981282F332785E290E0289F55
:1088B000A001299F500D389F500D1124CA01FC01C1
:1088C000EF5AFB4F8E819F81918380838981282F6E
:1088D000332785E290E0289FF001299FF00D389F13
:1088E000F00D1124CF01FC01EB5AFB4F88858083EA
:1088F00089818F5F898356CF8DE699E00E948D66CE
:108900008BE799E00E94FF6683E299E00E949B6BEF
:1089100085E399E00E940D6C86EA99E00E947167F8
:108920000E949A5C19828981853008F077C0CE0157
:108930004B96BC0189810E94FE67898199278295A7
:108940009295907F9827807F9827FC01E255F64FFB
:108950008B8D982F917080818E7F892B8083898168
:10896000992782959295907F9827807F9827FC0180
:10897000E255F64F8C8D8170982F990F80818D7FF5
:10898000892B80838981992782959295907F98275A
:10899000807F9827FC01E055F64F8D8D808389817B
:1089A000992782959295907F9827807F9827FC0140
:1089B000EB54F64F8E8D808389819927829592950D
:1089C000907F9827807F9827FC01EA54F64F8F8D7F
:1089D00080838981992782959295907F9827807FBF
:1089E0009827FC01E954F64F88A18083CE014B966D
:1089F0009C012A5F3F4F8981992782959295907FAC
:108A00009827807F98278854964F46E050E0B90118
:108A10000E94DCBC89818F5F898385CF82ED9DE0D8
:108A20009AAF89AF8EEA9EE09CAF8BAF88E090E072
:108A30009EAF8DAF8DAD9EADFE01FF96918380837D
:108A4000FE01FF9680819181ABADBCAD29AD3AAD01
:108A500024963FAF2EAF24972496EEADFFAD24971A
:108A6000019724F00E94C9BD0192FACF9F01FE0137
:108A7000FF9691838083CD019CAF8BAFC9019AAFE4
:108A800089AF19828981843008F07CC0CE01C696F6
:108A9000FE01FF9691838083998184E1989FC001B4
:108AA00011248253914F9EAF8DAF83E090E09CAF35
:108AB0008BAF8BAD9CAD9AAF89AF89AD9AADADADA3
:108AC000BEADFE01FF960190F081E02D019724F0EC
:108AD0000E94C9BD0192FACF9AAF89AFCD019EAF76
:108AE0008DAFCF01FE01FF96918380838981282F6E
:108AF0003327C901880F991F820F931FFC01E3528E
:108B0000F24F8EA980838981282F3327C901880FCE
:108B1000991F820F931FFC01E252F24F88AD8083B0
:108B20008981282F3327C901880F991F820F931F2E
:108B3000FC01E152F24F8FA9982F97708081887FB6
:108B4000892B80838981282F3327C901880F991F9A
:108B5000820F931FFC01E152F24F8081877F808357
:108B60008981282F3327C901880F991F820F931FEE
:108B7000FC01E152F24F80818F78808389818F5F81
:108B8000898380CFCD5BDF4F0FB6F894DEBF0FBE79
:108B9000CDBFDF91CF910895CF93DF93CDB7DEB7EF
:108BA00024970FB6F894DEBF0FBECDBF9A8389839A
:108BB0006B831C828B810E948C568C838C818332C8
:108BC00008F046C08C81282F332785E290E0289F4B
:108BD000A001299F500D389F500D1124CA01DC01BE
:108BE000AB5BBB4FE981FA8187898C938C81282FFD
:108BF000332785E290E0289FA001299F500D389FE0
:108C0000500D1124CA01DC01A55BBB4FE981FA813B
:108C100080819927382F2227E981FA81818199273C
:108C2000820F931F8D939C938C81282F332785E28D
:108C300090E0289FA001299F500D389F500D1124CE
:108C4000CA01DC01A15CBB4FE981FA8182818C936E
:108C500024960FB6F894DEBF0FBECDBFDF91CF9143
:108C60000895CF93DF93CDB7DEB723970FB6F8946F
:108C7000DEBF0FBECDBF1A821B8280917B09882385
:108C800069F080917B09813248F480917B090E94D0
:108C9000571A8823F1F081E08A831BC080917B09F9
:108CA000813268F080917B09853348F480917B099B
:108CB0000E9456A9882369F081E08A830AC08091C6
:108CC0007B090E94568389838981813011F481E078
:108CD0008A8380919009882351F080919009813294
:108CE00030F4809190090E94571A898313C08091B3
:108CF0009009813250F080919009853330F4809151
:108D000090090E9456A9898305C0809190090E940C
:108D10005683898389818E3F21F189818130E1F4F5
:108D20008091FF09843030F48091FF098F5F809338
:108D3000FF090BC01092FF098091000A882329F0D7
:108D40008091000A81508093000A8091000A882354
:108D500061F481E08B8309C0809191098093000ABE
:108D600004C0809191098093000A8A81813021F4A6
:108D700081E00E94E92A0DC08B81813021F481E0DD
:108D80000E942B2B06C080E00E94E92A80E00E940E
:108D90002B2B23960FB6F894DEBF0FBECDBFDF910D
:108DA000CF910895CF93DF93CDB7DEB722970FB65B
:108DB000F894DEBF0FBECDBF9A838983E981FA8123
:108DC000848188608483E981FA8180EF8283A9812C
:108DD000BA81E981FA8187858E7FFD018787A98124
:108DE000BA81E981FA818785877FFD018787A9811B
:108DF000BA81E981FA8187858F7DFD018787A98105
:108E0000BA81E981FA8187858F7BFD018787E981B6
:108E1000FA81168AE981FA8184818F7D8483A98110
:108E2000BA81E981FA81948585E0989FC001112477
:108E3000FD0196878587E981FA818585968500976A
:108E400089F4E981FA8181858F3F61F0A981BA8136
:108E5000E981FA81918585E0989FC0011124FD0187
:108E600093878287E981FA8183E0878322960FB610
:108E7000F894DEBF0FBECDBFDF91CF910895CF93A1
:108E8000DF93CDB7DEB723970FB6F894DEBF0FBEE2
:108E9000CDBF19828981823210F5998185E2989F30
:108EA000C0011124875C9B4F9B838A83EA81FB81ED
:108EB0008785992788709070009749F4EA81FB8133
:108EC0008785992781709070009709F404C08A8182
:108ED0009B810E94D24689818F5F8983DBCF239655
:108EE0000FB6F894DEBF0FBECDBFDF91CF910895CE
:108EF000CF93DF93CDB7DEB725970FB6F894DEBFDB
:108F00000FBECDBF89838981282F33273D832C83D2
:108F10008C819D818C33910509F48FC02C813D811A
:108F20002D33310524F58C819D818833910509F419
:108F300050C02C813D812933310534F48C819D81D1
:108F400087339105C9F1D4C02C813D812933310586
:108F500009F44CC08C819D818A33910509F453C07A
:108F60002C813D812B33310509F45AC0C1C08C815D
:108F70009D818034910509F494C02C813D81213478
:108F800031056CF48C819D818E33910509F46FC09D
:108F90002C813D812F3331050CF076C05BC08C8174
:108FA0009D818134910509F489C02C813D81223451
:108FB000310509F490C09CC08091DF0D807780312D
:108FC00029F481E090E09B838A8394C01B821A82FB
:108FD00091C08091DF0D8077803229F421E030E06C
:108FE0003B832A8387C01B821A8284C08091DF0D55
:108FF0008077803329F481E090E09B838A837AC074
:109000001B821A8277C08091E20D8077803129F42B
:1090100021E030E03B832A836DC01B821A826AC044
:109020008091E20D8077803229F481E090E09B838B
:109030008A8360C01B821A825DC08091E20D8077B6
:10904000803329F421E030E03B832A8353C01B8224
:109050001A8250C08091E50D8077803129F481E03B
:1090600090E09B838A8346C01B821A8243C0809112
:10907000E50D8077803229F421E030E03B832A83BC
:1090800039C01B821A8236C08091E50D807780330B
:1090900029F481E090E09B838A832CC01B821A8292
:1090A00029C08091E80D8077803129F421E030E0FB
:1090B0003B832A831FC01B821A821CC08091E80D4B
:1090C0008077803229F481E090E09B838A8312C00C
:1090D0001B821A820FC08091E80D8077803329F4BB
:1090E00021E030E03B832A8305C01B821A8202C044
:1090F0001B821A828A819B8125960FB6F894DEBF67
:109100000FBECDBFDF91CF910895CF93DF93CDB741
:10911000DEB725970FB6F894DEBF0FBECDBF19821C
:109120001C8219828981823208F053C282E00E9437
:109130005984998185E2989FC0011124875C9B4FD7
:109140009B838A831C82EA81FB818085882341F589
:10915000EA81FB818181803F09F020C2EA81FB81A5
:10916000848188608483AA81BB81EA81FB818785B1
:109170008E7FFD018787AA81BB81EA81FB8187857C
:10918000877FFD018787AA81BB81EA81FB81878573
:109190008F7BFD018787EA81FB818FE08283FEC19F
:1091A000EA81FB818085882309F48FC0EA81FB81F5
:1091B0008085813208F089C0EA81FB818785992703
:1091C00088709070009709F050C0EA81FB81878514
:1091D000992781709070009709F047C0EA81FB8160
:1091E00080850E94571A882359F0EA81FB8181818A
:1091F0008F3009F0D3C18A819B810E94D246CEC1B3
:10920000EA81FB818181803F09F0C8C1EA81FB814D
:1092100081858F3F09F4C2C1EA81FB8182859385F4
:10922000009709F0BBC1EA81FB8184818860848357
:10923000AA81BB81EA81FB8187858E7FFD018787BB
:10924000AA81BB81EA81FB818785877FFD018787B2
:10925000AA81BB81EA81FB8187858F7BFD0187879E
:10926000EA81FB818FE0828399C1EA81FB8180855D
:109270000E94571A882309F091C1EA81FB818181FC
:10928000803F09F08BC1EA81FB81848188608483FF
:10929000AA81BB81EA81FB8187858E7FFD0187875B
:1092A000AA81BB81EA81FB818785877FFD01878752
:1092B000AA81BB81EA81FB8187858F7BFD0187873E
:1092C000EA81FB818FE0828369C1EA81FB8180852D
:1092D000813208F48FC0EA81FB818085853308F0F4
:1092E00089C0EA81FB8187859927887090700097F3
:1092F00009F050C0EA81FB818785992781709070C1
:10930000009709F047C0EA81FB8180850E9456A939
:10931000882359F0EA81FB8181818F3009F03EC1B9
:109320008A819B810E94D24639C1EA81FB81818179
:10933000803F09F033C1EA81FB8181858F3F09F4C9
:109340002DC1EA81FB8182859385009709F026C1B2
:10935000EA81FB81848188608483AA81BB81EA8160
:10936000FB8187858E7FFD018787AA81BB81EA818A
:10937000FB818785877FFD018787AA81BB81EA8181
:10938000FB8187858F7BFD018787EA81FB818FE0E9
:10939000828304C1EA81FB8180850E9456A98823CB
:1093A00009F0FCC0EA81FB818181803F09F0F6C0B1
:1093B000EA81FB81848188608483AA81BB81EA8100
:1093C000FB8187858E7FFD018787AA81BB81EA812A
:1093D000FB818785877FFD018787AA81BB81EA8121
:1093E000FB8187858F7BFD018787EA81FB818FE089
:1093F0008283D4C01C82EA81FB8180858533B1F4ED
:109400008091CB0D833069F08091CB0D843049F091
:109410008091CB0D813029F08091CB0D863009F001
:1094200003C081E08D832CC01D822AC0EA81FB81AC
:109430008085863371F48091CB0D853029F0809141
:10944000CB0D823009F003C081E08D8319C01D82ED
:1094500017C0EA81FB818085873360F0EA81FB8158
:109460008085833438F4EA81FB8180850E947847C7
:109470008D8306C0EA81FB8180850E9456838D839F
:109480008D818E3F09F1EA81FB818085803C31F43A
:109490008D81813001F581E08C831DC0EA81FB81E3
:1094A0008581813031F48D81813019F481E08C83A4
:1094B00012C0EA81FB818581803169F48D81882326
:1094C00051F481E08C8307C0EA81FB8180858F3F66
:1094D00011F481E08C838C818823E9F0EA81FB819F
:1094E00081818F3009F059C0EA81FB8187859927F6
:1094F00088709070009709F050C0EA81FB818785E1
:10950000992781709070009709F047C08A819B81EC
:109510000E94D24642C0EA81FB818181803F89F06E
:10952000EA81FB818785992788709070009749F4BC
:10953000EA81FB818785992781709070009709F4F3
:109540002CC0EA81FB8181858F3F39F1EA81FB8163
:1095500082859385009709F5EA81FB818481886083
:109560008483AA81BB81EA81FB8187858E7FFD018F
:109570008787AA81BB81EA81FB818785877FFD017F
:109580008787AA81BB81EA81FB8187858F7BFD016B
:109590008787EA81FB818FE082831C82EA81FB81DD
:1095A00081818F3091F4EA81FB81878599278970C9
:1095B0009070009751F4909111018981981729F4C6
:1095C00082E2809311011092E90D89818F5F898376
:1095D000A9CD25960FB6F894DEBF0FBECDBFDF91A3
:1095E000CF910895CF93DF93CDB7DEB722970FB613
:1095F000F894DEBF0FBECDBF89836A838A818093D2
:10960000330480913304823019F48FEF8093590929
:1096100022960FB6F894DEBF0FBECDBFDF91CF917B
:109620000895CF93DF93CDB7DEB727970FB6F894A1
:10963000DEBF0FBECDBF9A8389831B82E981FA8189
:109640008081833228F4E981FA818081882319F4AA
:109650001D821C82F2C0E981FA8180810E948C56B1
:109660008B83E981FA818181282F33273F832E83E1
:109670004E815F814F30510539F08E819F81803F4F
:10968000910509F45AC0D5C08B81282F332785E274
:1096900090E0289FA001299F500D389F500D112464
:1096A000CA01FC01E65CFB4F8FE080838B81282F91
:1096B000332785E290E0289FA001299F500D389F15
:1096C000500D1124CA01DC01A85BBB4F8B81282FF0
:1096D000332785E290E0289FA001299F500D389FF5
:1096E000500D1124CA01FC01E85BFB4F80818E7F85
:1096F0008C938B81282F332785E290E0289FA0014F
:10970000299F500D389F500D1124CA01DC01A85B20
:10971000BB4F8B81282F332785E290E0289FA00143
:10972000299F500D389F500D1124CA01FC01E85BA0
:10973000FB4F8081877F8C937CC08B81282F3327C0
:1097400085E290E0289FA001299F500D389F500D81
:109750001124CA01FC01E65CFB4F80EF80838B8102
:10976000282F332785E290E0289FA001299F500DE4
:10977000389F500D1124CA01DC01A85BBB4F8B81BF
:10978000282F332785E290E0289FA001299F500DC4
:10979000389F500D1124CA01FC01E85BFB4F80810A
:1097A0008E7F8C938B81282F332785E290E0289F32
:1097B000A001299F500D389F500D1124CA01DC01D2
:1097C000A85BBB4F8B81282F332785E290E0289F31
:1097D000A001299F500D389F500D1124CA01FC0192
:1097E000E85BFB4F8081877F8C938B81282F332709
:1097F00085E290E0289FA001299F500D389F500DD1
:109800001124CA01FC01E15BFB4F10828B81282FE0
:10981000332785E290E0289FA001299F500D389FB3
:10982000500D1124CA01FC01E35CFB4F80818F7D48
:10983000808381E090E09D838C838C819D8127963D
:109840000FB6F894DEBF0FBECDBFDF91CF91089564
:109850000F93CF93DF93CDB7DEB76C970FB6F89425
:10986000DEBF0FBECDBF1B861C861C821B821A82E8
:1098700019821D821E8210925B0910925A09109261
:109880005E091092600910925F090E947106809330
:109890005D0980913304882309F05DC61B828B81AA
:1098A000823210F00C94585682E00E9459841C8237
:1098B0001A8219829B8185E2989FC0011124875CDE
:1098C0009B4F9E878D87ED85FE85858D9927807FAF
:1098D0009070803A910519F481E48D8317C0ED856D
:1098E000FE85858D9927807F9070803B910519F4C6
:1098F00082E48D830BC0CE01039600E021E0AC0131
:109900006DE178E082E191E00E942F60ED85FE85B7
:10991000118A108AED85FE8584818470882309F080
:10992000C7C3ED85FE858081282F33273C8B2B8B89
:109930004B895C894130510509F4DCC18B899C89D4
:109940008034910509F0CAC3ED85FE858181E82F39
:10995000FF27F88BEF872F8538892F30310509F4E1
:109960001BC14F855889403F510509F0B7C3ED85AC
:10997000FE8584818270882379F4ED85FE8584815B
:109980008170882349F4ED85FE858785992780724B
:109990009070009709F42DC08B818A3041F480913A
:1099A000DA0D882321F082E08093DA0D15C08B81D7
:1099B0008B3041F48091CC0D882321F082E080939C
:1099C000CC0D0AC08B818C3039F48091CF0D882367
:1099D00019F082E08093CF0DAD85BE85ED85FE85C3
:1099E000858D8F70FD0141A16D810E94687719827C
:1099F00090C0ED85FE8585859685009709F089C024
:109A0000ED85FE858785992781709070009709F014
:109A100080C08B818A3021F58091DA0D882301F195
:109A20008091DA0D823070F4AD85BE85ED85FE85BE
:109A3000858D8F70FD0141A16D810E94F47681E0DA
:109A4000898367C08091DA0D813009F062C083E0BC
:109A50008093DA0D1092D10D1092D00D198259C059
:109A60008B818B3019F58091CC0D8823F9F0809192
:109A7000CC0D823070F4AD85BE85ED85FE85858D7B
:109A80008F70FD0141A16D810E94F47681E0898390
:109A900040C08091CC0D8130E1F583E08093CC0D06
:109AA0001092DC0D1092DB0D198233C08B818C304B
:109AB00019F58091CF0D8823F9F08091CF0D823078
:109AC00070F4AD85BE85ED85FE85858D8F70FD01B9
:109AD00041A16D810E94F47681E089831AC0809152
:109AE000CF0D8130B1F483E08093CF0D1092CE0D75
:109AF0001092CD0D19820DC0AD85BE85ED85FE8518
:109B0000858D8F70FD0141A16D810E94F47681E009
:109B10008983ED85FE8584818870882309F4DEC2FF
:109B2000ED85FE858481877F8483ED85FE85828136
:109B30008F3009F0D3C28B818A3041F48091DA0DE5
:109B4000882321F082E08093DA0D15C08B818B3061
:109B500041F48091CC0D882321F082E08093CC0DDC
:109B60000AC08B818C3039F48091CF0D882319F095
:109B700082E08093CF0DED85FE858FE08183AD85FA
:109B8000BE85ED85FE85858D8F70FD0141A16D81BE
:109B90000E9468771982A2C2ED85FE858481887053
:109BA000882309F49BC2ED85FE858481877F8483A9
:109BB000ED85FE858281803F09F090C2ED85FE85AE
:109BC00080EF8183ED85FE8585859685009709F078
:109BD00085C2ED85FE8584818270882309F07EC26E
:109BE000ED85FE8584818170882309F077C28B81A1
:109BF0008A3021F58091DA0D882301F18091DA0D08
:109C0000823070F4AD85BE85ED85FE85858D8F70C3
:109C1000FD0141A16D810E94F47681E089835EC2DD
:109C20008091DA0D823009F059C283E08093DA0D19
:109C30001092D10D1092D00D198250C28B818B30B1
:109C400021F58091CC0D882301F18091CC0D8230DB
:109C500070F4AD85BE85ED85FE85858D8F70FD0127
:109C600041A16D810E94F47681E0898337C28091A1
:109C7000CC0D823009F032C283E08093CC0D10927B
:109C8000DC0D1092DB0D198229C28B818C3021F5FD
:109C90008091CF0D882301F18091CF0D823070F437
:109CA000AD85BE85ED85FE85858D8F70FD0141A159
:109CB0006D810E94F47681E0898310C28091CF0D7E
:109CC000823009F00BC283E08093CF0D1092CE0D4D
:109CD0001092CD0D198202C2AD85BE85ED85FE853F
:109CE000858D8F70FD0141A16D810E94F47681E028
:109CF0008983F4C1ED85FE858181282F33273A8B36
:109D0000298B49895A894F30510509F424C1898921
:109D10009A89803F910509F0E1C1ED85FE85848136
:109D20008270882379F4ED85FE8584818170882393
:109D300049F4ED85FE85878599278072907000979C
:109D400009F42DC08B818A3041F48091DA0D88238B
:109D500021F082E08093DA0D15C08B818B3041F4C5
:109D60008091CC0D882321F082E08093CC0D0AC035
:109D70008B818C3039F48091CF0D882319F082E0EB
:109D80008093CF0DAD85BE85ED85FE85858D8F7069
:109D9000FD0141A16D810E946877198299C0ED850E
:109DA000FE8585859685009709F092C0ED85FE8534
:109DB0008785992781709070009709F089C0ED859B
:109DC000FE858785992788709070009709F080C07C
:109DD0008B818A3021F58091DA0D882301F1809101
:109DE000DA0D823070F4AD85BE85ED85FE85858DFA
:109DF0008F70FD0141A16D810E94F47681E089831D
:109E000067C08091DA0D823009F062C083E08093F0
:109E1000DA0D1092D10D1092D00D198259C08B819C
:109E20008B3019F58091CC0D8823F9F08091CC0D01
:109E3000823070F4AD85BE85ED85FE85858D8F7091
:109E4000FD0141A16D810E94F47681E0898340C0CB
:109E50008091CC0D8230E1F583E08093CC0D10929F
:109E6000DC0D1092DB0D198233C08B818C3019F51B
:109E70008091CF0D8823F9F08091CF0D823070F45E
:109E8000AD85BE85ED85FE85858D8F70FD0141A177
:109E90006D810E94F47681E089831AC08091CF0D94
:109EA0008230B1F483E08093CF0D1092CE0D1092EA
:109EB000CD0D19820DC0AD85BE85ED85FE85858DE4
:109EC0008F70FD0141A16D810E94F47681E089834C
:109ED000ED85FE8584818870882309F4FFC0ED85B7
:109EE000FE858481877F8483ED85FE8582818F3026
:109EF00009F0F4C08B818A3041F48091DA0D882317
:109F000021F082E08093DA0D15C08B818B3041F413
:109F10008091CC0D882321F082E08093CC0D0AC083
:109F20008B818C3039F48091CF0D882319F082E039
:109F30008093CF0DED85FE858FE08183AD85BE8555
:109F4000ED85FE85858D8F70FD0141A16D810E949B
:109F500068771982C3C0ED85FE8584818870882367
:109F600009F4BCC0ED85FE858481877F8483ED85FF
:109F7000FE858281803F09F0B1C0ED85FE8580EFCE
:109F80008183ED85FE8585859685009709F0A6C0BD
:109F9000ED85FE8584818270882309F09FC0ED8560
:109FA000FE8584818170882309F098C08B818A3076
:109FB00021F58091DA0D882301F18091DA0D82304C
:109FC00070F4AD85BE85ED85FE85858D8F70FD01B4
:109FD00041A16D810E94F47681E089837FC08091E8
:109FE000DA0D823009F07AC083E08093DA0D1092A6
:109FF000D10D1092D00D198271C08B818B3021F55B
:10A000008091CC0D882301F18091CC0D823070F4C9
:10A01000AD85BE85ED85FE85858D8F70FD0141A1E5
:10A020006D810E94F47681E0898358C08091CC0DC7
:10A03000823009F053C083E08093CC0D1092DC0D88
:10A040001092DB0D19824AC08B818C3019F58091FA
:10A05000CF0D8823F9F08091CF0D823070F4AD855B
:10A06000BE85ED85FE85858D8F70FD0141A16D81D9
:10A070000E94F47681E0898331C08091CF0D8230D7
:10A0800069F583E08093CF0D1092CE0D1092CD0D27
:10A09000198224C0AD85BE85ED85FE85858D8F70C6
:10A0A000FD0141A16D810E94F47681E0898316C093
:10A0B000ED85FE858181282F33273E8B2D8B4D89A1
:10A0C0005E894F30510549F08D899E89803F910509
:10A0D00009F004C081E0898301C01982ED85FE8505
:10A0E0008181803F09F08DC0ED85FE8582A18F3F83
:10A0F00009F487C0ED85FE8582A10E948603AA2708
:10A10000BB278F839887A987BA87ED85FE858F81C6
:10A11000988594A383A38B819927FC01ED5DF64F6D
:10A120008081282F3327442755278F819885A9853B
:10A13000BA85281739074A075B072CF01F82188653
:10A1400019861A8616C08B819927FC01ED5DF64FA2
:10A150008081282F3327442755278F819885A9850B
:10A16000BA85821B930BA40BB50B8F839887A987A5
:10A17000BA878F819885A985BA8583309105A10515
:10A18000B10534F18B81282F3327C901820F931F2A
:10A19000FC01EB5CF64F80819181AA27BB272F81C0
:10A1A000388549855A85BC01CD010E9403BDDC017B
:10A1B000CB0120EE31E040E050E0BC01CD010E9437
:10A1C00077BDDA01C9018F839887A987BA8704C050
:10A1D0001F82188619861A86ED85FE858F819885DF
:10A1E000918B808BED85FE8520915A0930915B091A
:10A1F00080899189820F931F90935B0980935A09FC
:10A2000004C0ED85FE85118A108A8981882351F466
:10A21000ED85FE85828D938D009721F0ED85FE857D
:10A22000138E128EED85FE85878599278870907034
:10A23000009709F0B3C0ED85FE85AD85BE85208908
:10A240003189FD01828993898217930708F05AC0EA
:10A25000ED85FE85828D938D009721F0ED85FE853D
:10A26000138E128EED85FE85848180728823C1F164
:10A27000ED85FE8584899589009709F08FC0AD85AD
:10A28000BE85ED85FE8587858860FD018787809185
:10A290005E098F5F80935E0981E08B87ED85FE8587
:10A2A00080818130A1F4AD85BE85ED85FE85858DEB
:10A2B0008F70FD0141A16D810E94687719828B81A9
:10A2C00080931101ED85FE8586818093FE09ED85E1
:10A2D000FE858B818F5F608971890E94B5645EC045
:10A2E000ED85FE85848180628483AD85BE85ED85A4
:10A2F000FE85968185E0989FC0011124FD01958B14
:10A30000848B4CC0ED85FE8584818F7D8483ED85B3
:10A31000FE85808D918D009709F440C08981882346
:10A3200039F1ED85FE85AD85BE8520893189FD0138
:10A33000808D918D28173907D8F4ED85FE85828DA3
:10A34000938D009759F5ED85FE8587859927807453
:10A350009070009719F5AD85BE85ED85FE85948DCD
:10A3600085E0989FC0011124FD01938F828F16C054
:10A37000ED85FE85828D938D009781F0ED85FE85BC
:10A38000AD85BE8520893189FD01808D918D821733
:10A39000930720F4ED85FE85138E128EED85FE85E4
:10A3A000868D9927807F9070803A910519F481E419
:10A3B0008E8317C0ED85FE85868D9927807F9070EE
:10A3C000803B910519F482E48E830BC0CE01039685
:10A3D00000E021E0AC016BED79E082E191E00E94C8
:10A3E0002F60AD85BE85ED85FE85868D8F70FD0164
:10A3F00041A16E810E9437788A83ED85FE85818137
:10A40000803F09F082C0ED85FE8587859927887099
:10A410009070009709F079C0ED85FE8587859927B2
:10A4200081709070009709F070C090915D098091E3
:10A430001001891708F069C08981813009F062C074
:10A440008A81882309F05EC0ED85FE858781882397
:10A4500009F05BC0ED85FE858485882309F055C031
:10A46000ED85FE858181803F09F04FC0ED85FE8539
:10A4700087898F3F41F0AD85BE85ED85FE85878953
:10A480008F5FFD01878BED85FE8587898630E8F13A
:10A49000AD85BE85ED85FE8586898F5FFD01868B46
:10A4A000ED85FE858689843198F4AD85BE85ED8580
:10A4B000FE85858D8F70FD0141A16D810E946877B9
:10A4C000ED85FE85178AED85FE8583E087831DC0B7
:10A4D000AD85BE85ED85FE85858D8F70FD0141A121
:10A4E0006D810E946877AD85BE85ED85FE85878587
:10A4F0008160FD0187878B818F5F0E943C6581E0D1
:10A500008B8703C0ED85FE85178AED85FE858785DF
:10A51000992781709070009729F0809160098F5F72
:10A5200080936009ED85FE858785992788709070F6
:10A53000009729F080915E098F5F80935E09ED8519
:10A54000FE858785882319F08C858F5F8C878B81AA
:10A550008F5F8B83A4C980913304813009F090C24E
:10A560001B828B81823208F0A3C38B81282F332773
:10A5700085E290E0289FA001299F500D389F500D43
:10A580001124CA01DC01A85BBB4F8B81282F332724
:10A5900085E290E0289FF001299FF00D389FF00D93
:10A5A0001124CF01FC01E85BFB4F80818F7D8C93F0
:10A5B0009B8185E2989FC0011124875C9B4F9E87F9
:10A5C0008D87ED85FE85858D9927807F9070803AF7
:10A5D000910519F481E48D830BC0ED85FE85858D91
:10A5E0009927807F9070803B910511F482E48D83E0
:10A5F000ED85FE8584818470882309F07EC0ED8519
:10A60000FE858081282F33273C8F2B8F4B8D5C8DCF
:10A610004130510509F441C08B8D9C8D80349105EA
:10A6200009F06BC0ED85FE858181E82FFF27F88F4B
:10A63000EF8B2F89388D2F303105A1F04F89588D40
:10A64000403F510509F059C0AD85BE85ED85FE85B9
:10A65000858D8F70FD0141A16D810E94F47681E0AE
:10A6600089834BC0AD85BE858B81282F332785E23A
:10A6700090E0289FA001299F500D389F500D112474
:10A68000CA01FC01EA5AFB4F80818F70FD0141A194
:10A690006D810E946877198230C0ED85FE858181C9
:10A6A000282F33273A8F298F498D5A8D4F305105E6
:10A6B000A1F0898D9A8D803F910509F01EC0AD856E
:10A6C000BE85ED85FE85858D8F70FD0141A16D8173
:10A6D0000E94F47681E0898310C0AD85BE85ED854A
:10A6E000FE85858D8F70FD0141A16D810E94687787
:10A6F000ED85FE858FE081831982ED85FE85818160
:10A70000803F09F08CC0ED85FE8582A18F3F09F462
:10A7100086C0ED85FE8582A10E948603AA27BB27FD
:10A720008F839887A987BA87ED85FE858F81988565
:10A7300094A383A38B819927FC01ED5DF64F808163
:10A74000282F3327442755278F819885A985BA85D7
:10A75000281739074A075B072CF01F8218861986CD
:10A760001A8616C08B819927FC01ED5DF64F80811A
:10A77000282F3327442755278F819885A985BA85A7
:10A78000821B930BA40BB50B8F839887A987BA877D
:10A790008F819885A985BA8583309105A105B1057A
:10A7A00034F18B81282F3327C901820F931FFC01BD
:10A7B000EB5CF64F80819181AA27BB272F813885DA
:10A7C00049855A85BC01CD010E9403BDDC01CB0146
:10A7D00020EE31E040E050E0BC01CD010E9477BDA9
:10A7E000DA01C9018F839887A987BA8704C01F82BD
:10A7F000188619861A86ED85FE858F819885918B3E
:10A80000808BED85FE8520915A0930915B09808906
:10A810009189820F931F90935B0980935A09ED856C
:10A82000FE85AD85BE8520893189FD0182899389A8
:10A830008217930708F050C0ED85FE8584818072F1
:10A840008823C1F1ED85FE8584899589009709F0FB
:10A850004CC0AD85BE85ED85FE8587858860FD0190
:10A86000878780915E098F5F80935E0981E08B8787
:10A87000ED85FE8580818130A1F4AD85BE85ED85B5
:10A88000FE85858D8F70FD0141A16D810E946877E5
:10A890001982ED85FE858FE08183ED85FE858FE051
:10A8A0008283ED85FE858B818F5F608971890E942F
:10A8B000B5641BC0ED85FE85848180628483AD858F
:10A8C000BE85ED85FE85968185E0989FC0011124A7
:10A8D000FD01958B848B09C0ED85FE8584818F7D7C
:10A8E0008483ED85FE85158A148AED85FE85868D27
:10A8F0009927807F9070803A910519F481E48E83C6
:10A900000BC0ED85FE85868D9927807F9070803BFA
:10A91000910511F482E48E83AD85BE85ED85FE85BB
:10A92000868D8F70FD0141A16E810E9437788A83E8
:10A93000ED85FE858785992788709070009709F0CE
:10A9400079C0ED85FE858785992781709070009785
:10A9500009F070C090915D0980911001891708F08D
:10A9600069C08981813009F062C08A81882309F039
:10A970005EC0ED85FE858781882309F05BC0ED858B
:10A98000FE858485882309F055C0ED85FE8581818B
:10A99000803F09F04FC0ED85FE8587898F3F41F0EC
:10A9A000AD85BE85ED85FE8587898F5FFD01878B2F
:10A9B000ED85FE8587898630E8F1AD85BE85ED851C
:10A9C000FE8586898F5FFD01868BED85FE858689F4
:10A9D000843198F4AD85BE85ED85FE85858D8F70BB
:10A9E000FD0141A16D810E946877ED85FE85178A82
:10A9F000ED85FE8583E087831DC0AD85BE85ED8531
:10AA0000FE85858D8F70FD0141A16D810E94687763
:10AA1000AD85BE85ED85FE8587858160FD018787D3
:10AA20008B818F5F0E943C6581E08B8703C0ED8541
:10AA3000FE85178AED85FE85878599278170907040
:10AA4000009729F0809160098F5F80936009ED8500
:10AA5000FE858785992788709070009729F08091EE
:10AA60005E098F5F80935E09ED85FE85878588236B
:10AA700019F08C858F5F8C878B818F5F8B8371CD75
:10AA800080913304823009F013C11B828B818232A2
:10AA900008F00EC19B8185E2989FC0011124875C5C
:10AAA0009B4F9E878D87ED85FE85858D9927807FBD
:10AAB0009070803A910519F481E48D830BC0ED8587
:10AAC000FE85858D9927807F9070803B910511F4DC
:10AAD00082E48D8380915909882319F18B8199270C
:10AAE0009C012F5F3F4F80915909992728173907FB
:10AAF00061F4AD85BE85ED85FE85858D8F70FD0188
:10AB000041A16D810E94F47617C0AD85BE85ED85AB
:10AB1000FE85858D8F70FD0141A16D810E94687752
:10AB20000BC0AD85BE85ED85FE85858D8F70FD01E1
:10AB300041A16D810E94F476ED85FE8582A18F3F53
:10AB400009F4B2C0ED85FE8582A10E948603AA2782
:10AB5000BB278F839887A987BA87ED85FE858F816C
:10AB6000988594A383A38091320499278170907073
:10AB7000009771F18B819927FC01ED5DF64F808183
:10AB8000282F3327442755278F819885A985BA8593
:10AB9000281739074A075B072CF01F821886198689
:10ABA0001A8616C08B819927FC01ED5DF64F8081D6
:10ABB000282F3327442755278F819885A985BA8563
:10ABC000821B930BA40BB50B8F839887A987BA8739
:10ABD0008F819885A985BA8583309105A105B10536
:10ABE0000CF44AC0809132049927827090700097CB
:10ABF00031F18B81282F3327C901820F931FFC016C
:10AC0000EB5CF64F80819181AA27BB272F81388585
:10AC100049855A85BC01CD010E9403BDDC01CB01F1
:10AC200020EE31E040E050E0BC01CD010E9477BD54
:10AC3000DA01C9018F839887A987BA8721C08F81DC
:10AC40009885A985BA8528EB31E040E050E0BC0149
:10AC5000CD010E9403BDDC01CB0120EE31E040E0DC
:10AC600050E0BC01CD010E9477BDDA01C9018F839C
:10AC70009887A987BA8704C01F82188619861A8602
:10AC8000ED85FE858F819885918B808BED85FE8586
:10AC900020915A0930915B0980899189820F931F15
:10ACA00090935B0980935A098B818F5F8B83EECEE3
:10ACB0008C85882331F410925F09109260091092FC
:10ACC00061090E94450680935C0990915C0980911E
:10ACD0003404891720F480915C0980933404209116
:10ACE0005A0930915B09809135049091360482179E
:10ACF000930740F480915A0990915B099093360430
:10AD0000809335046C960FB6F894DEBF0FBECDBFAE
:10AD1000DF91CF910F910895CF93DF93CDB7DEB739
:10AD200021970FB6F894DEBF0FBECDBF898389810E
:10AD30008150992721960FB6F894DEBF0FBECDBF84
:10AD4000DF91CF910895CF93DF93CDB7DEB72497EE
:10AD50000FB6F894DEBF0FBECDBF9A8389836B8395
:10AD60001C828B810E948C568C838C81833208F0EC
:10AD700012C08C81282F332785E290E0289FA00104
:10AD8000299F500D389F500D1124CA01FC01E15C30
:10AD9000FB4F8981808324960FB6F894DEBF0FBEE7
:10ADA000CDBFDF91CF910895CF93DF93CDB7DEB7BD
:10ADB00024970FB6F894DEBF0FBECDBF9A83898368
:10ADC0001B8280EC0E945683882319F08B8181605E
:10ADD0008B8381EC0E945683882319F08B818260DB
:10ADE0008B8382EC0E945683882319F08B818460C8
:10ADF0008B8381ED0E945683882319F08B818860B4
:10AE00008B8384EC0E945683882319F08B818061A8
:10AE10008B8385EC0E945683882319F08B81806296
:10AE20008B8386EC0E945683882319F08B81806483
:10AE30008B8387EC0E945683882319F08B8180686E
:10AE40008B831C8283EC0E945683882319F08C81AB
:10AE500081608C8382ED0E945683882319F08C8157
:10AE600082608C8383ED0E945683882319F08C8145
:10AE700084608C83E981FA818B818083E981FA8106
:10AE80008C8181831B8281E00E94571A882319F0EC
:10AE90008B8181608B8382E00E94571A882319F08E
:10AEA0008B8182608B8383E00E94571A882319F07C
:10AEB0008B8184608B8384E00E94571A882319F069
:10AEC0008B8188608B8385E00E94571A882319F054
:10AED0008B8180618B8386E00E94571A882319F04A
:10AEE0008B8180628B8387E00E94571A882319F038
:10AEF0008B8180648B8388E00E94571A882319F025
:10AF00008B8180688B83E981FA818B8182831B82AC
:10AF100089E00E94571A882319F08B8181608B8306
:10AF20008AE00E94571A882319F08B8182608B83F4
:10AF30008BE00E94571A882319F08B8184608B83E1
:10AF40008CE00E94571A882319F08B8188608B83CC
:10AF50008DE00E94571A882319F08B8180618B83C2
:10AF60008EE00E94571A882319F08B8180628B83B0
:10AF70008FE00E94571A882319F08B8180648B839D
:10AF800080E10E94571A882319F08B8180688B8397
:10AF9000E981FA818B8183831B8281E10E94571AA8
:10AFA000882319F08B8181608B8382E10E94571A7C
:10AFB000882319F08B8182608B8383E10E94571A6A
:10AFC000882319F08B8184608B8384E10E94571A57
:10AFD000882319F08B8188608B8385E10E94571A42
:10AFE000882319F08B8180618B8386E10E94571A38
:10AFF000882319F08B8180628B8387E10E94571A26
:10B00000882319F08B8180648B8388E10E94571A12
:10B01000882319F08B8180688B83E981FA818B8189
:10B0200084831B8289E10E94571A882319F08B813F
:10B0300081608B838AE10E94571A882319F08B81E3
:10B0400082608B838BE10E94571A882319F08B81D1
:10B0500084608B838CE10E94571A882319F08B81BE
:10B0600088608B838DE10E94571A882319F08B81A9
:10B0700080618B838EE10E94571A882319F08B819F
:10B0800080628B838FE10E94571A882319F08B818D
:10B0900080648B8380E20E94571A882319F08B8189
:10B0A00080688B83E981FA818B81858324960FB632
:10B0B000F894DEBF0FBECDBFDF91CF9108950F93FF
:10B0C0001F93CF93DF93CDB7DEB72B970FB6F894CE
:10B0D000DEBF0FBECDBF89837B836A831C828981DB
:10B0E0000E948C568C838C81833218F01B861A86C2
:10B0F00017C18C81282F332785E290E0289FA0017B
:10B10000299F500D389F500D1124CA01FC01E35CAA
:10B11000FB4F8081869586958170882309F083C0D6
:10B120008C81282F332785E290E0289FF001299F0A
:10B13000F00D389FF00D1124CF01FC01E65CFB4FB0
:10B140008081803F09F05AC08C81282F332785E207
:10B1500090E0289FA001299F500D389F500D112489
:10B16000CA01FC01EA5BFB4F80819181009709F0E5
:10B1700040C08C81282F332785E290E0289FF00182
:10B18000299FF00D389FF00D1124CF01FC01E35CE5
:10B19000FB4F808186958170813059F18C81282FF9
:10B1A000332785E290E0289FA001299F500D389F0A
:10B1B000500D1124CA01FC01E35CFB4F80818170BA
:10B1C0008130B9F08C81282F332785E290E0289FC9
:10B1D000F001299FF00D389FF00D1124CF01FC01E3
:10B1E000E85BFB4F8081992780729070009709F48B
:10B1F00005C0EA81FB818FE080835BC0AA81BB81AF
:10B200008C81282F332785E290E0289FA001299F79
:10B21000500D389F500D1124CA01FC01E65CFB4F14
:10B2200080818C9346C01F821D828D81853008F0FD
:10B2300040C08F818823E9F58D8199278295929569
:10B24000907F9827807F98278255964F9987888787
:10B25000E885F985818199278130910509F025C01C
:10B260001E828E81863008F5288539858E81992742
:10B27000820F931FFC013A9690818C81981789F474
:10B2800081E08F83E885F98580818470882329F0A7
:10B29000EA81FB818FE0808304C0EA81FB8180EF3B
:10B2A00080838E818F5F8E83DCCF8D818F5F8D83D6
:10B2B000BCCFAA81BB818C81282F332785E290E007
:10B2C000289FF001299FF00D389FF00D1124CF0128
:10B2D000FC01E85BFB4F8081FD018183AA81BB817A
:10B2E0008C81282F332785E290E0289FA001299F99
:10B2F000500D389F500D1124CA01FC01E75BFB4F34
:10B3000080819181FD01948383830A811B818981DE
:10B310000E94FB65F801828341E050E05B874A8729
:10B320008A859B852B960FB6F894DEBF0FBECDBFE6
:10B33000DF91CF911F910F910895CF93DF93CDB7F8
:10B34000DEB724970FB6F894DEBF0FBECDBF89835A
:10B350001A8289810E948C568A838A81833218F0EE
:10B360001C821B8243C08A81282F332785E290E00C
:10B37000289FA001299F500D389F500D1124CA010C
:10B38000FC01E65CFB4F8081803F71F58A81282FAC
:10B39000332785E290E0289FA001299F500D389F18
:10B3A000500D1124CA01FC01E35CFB4F808186959E
:10B3B00081708823C9F48A81282F332785E290E0A1
:10B3C000289FA001299F500D389F500D1124CA01BC
:10B3D000FC01E35CFB4F80818170882329F481E0CC
:10B3E00090E09C838B8302C01C821B828B819C819A
:10B3F00024960FB6F894DEBF0FBECDBFDF91CF917C
:10B400000895CF93DF93CDB7DEB724970FB6F894A6
:10B41000DEBF0FBECDBF89831A8289810E948C5600
:10B420008A838A81833218F01C821B822EC08A8113
:10B43000282F332785E290E0289FA001299F500DF7
:10B44000389F500D1124CA01FC01E85BFB4F80813D
:10B450008830A1F08A81282F332785E290E0289F49
:10B46000A001299F500D389F500D1124CA01FC01E5
:10B47000E85BFB4F8081813009F005C081E090E0FE
:10B480009C838B8302C01C821B828B819C812496AF
:10B490000FB6F894DEBF0FBECDBFDF91CF910895F8
:10B4A000CF93DF93CDB7DEB722970FB6F894DEBF08
:10B4B0000FBECDBF9A838983E981FA8180915A09B1
:10B4C00090915B0991838083E981FA8180915C0985
:10B4D0008283E981FA8180915D098383E981FA8120
:10B4E00080915E098483E981FA8180915F09858377
:10B4F000E981FA81809160098683E981FA818091EE
:10B500006109878322960FB6F894DEBF0FBECDBFC8
:10B51000DF91CF910895CF93DF93CDB7DEB7239717
:10B520000FB6F894DEBF0FBECDBF89838981882313
:10B5300089F08981833270F4998185E2989FC001F6
:10B54000112429E334E025523040820F931F9B835E
:10B550008A8302C01B821A828A819B8123960FB63E
:10B56000F894DEBF0FBECDBFDF91CF910895CF938A
:10B57000DF93CDB7DEB79EEF8091210089238093C2
:10B5800021009EEF80912200892380932200109257
:10B5900027001092280091EF80912A008923809340
:10B5A0002A0091EF80912B00892380932B00DF915B
:10B5B000CF9108950F93CF93DF93CDB7DEB7249744
:10B5C0000FB6F894DEBF0FBECDBF89831A82898182
:10B5D0000E948C568A838A81833168F000E020E0E3
:10B5E00040E050E060E87CE082E191E00E942F6062
:10B5F0001C821B8209C08A819927FC01ED5DF64FF0
:10B60000808199279C838B838B819C8124960FB6A4
:10B61000F894DEBF0FBECDBFDF91CF910F9108959B
:10B620000F93CF93DF93CDB7DEB724970FB6F8947F
:10B63000DEBF0FBECDBF89831A8289810E948C56DE
:10B640008A838A81833178F000E020E040E050E096
:10B650006EE87CE082E191E00E942F6040E652E2D9
:10B660005C834B8317C08A81282F3327C901820F3F
:10B67000931FFC01EB5CF64F2081318184E190E067
:10B68000289FA001299F500D389F500D1124CA01F9
:10B690009C838B838B819C8124960FB6F894DEBFAC
:10B6A0000FBECDBFDF91CF910F9108950F93CF9330
:10B6B000DF93CDB7DEB724970FB6F894DEBF0FBE89
:10B6C000CDBF89837B836A831C8289810E948C56CB
:10B6D0008C838C81833158F000E020E040E050E022
:10B6E0006DE97CE082E191E00E942F6017C08C81BF
:10B6F000282F3327C901820F931FFC01EB5CF64F03
:10B700008A819B8124E130E0B9010E942EBDCB01EA
:10B710009183808385E399E00E94D46B24960FB6D1
:10B72000F894DEBF0FBECDBFDF91CF910F9108958A
:10B73000CF93DF93CDB7DEB724970FB6F894DEBF73
:10B740000FBECDBF89831A8289810E948C568A835D
:10B750008A81833118F01C821B8214C08A81282FB1
:10B76000332785E290E0289FA001299F500D389F44
:10B77000500D1124CA01FC01E75BFB4F80819181D0
:10B780009C838B838B819C8124960FB6F894DEBFBB
:10B790000FBECDBFDF91CF910895CF93DF93CDB78B
:10B7A000DEB724970FB6F894DEBF0FBECDBF8983F6
:10B7B0001A8289810E948C568A838A81833118F08B
:10B7C0001C821B8214C08A81282F332785E290E0D7
:10B7D000289FA001299F500D389F500D1124CA01A8
:10B7E000FC01E45AFB4F808191819C838B838B8188
:10B7F0009C8124960FB6F894DEBF0FBECDBFDF91BB
:10B80000CF910895CF93DF93CDB7DEB722970FB6D0
:10B81000F894DEBF0FBECDBF89836A838981809390
:10B8200032048A818093590922960FB6F894DEBFBC
:10B830000FBECDBFDF91CF910895CF93DF93CDB7EA
:10B84000DEB728970FB6F894DEBF0FBECDBF1A82C1
:10B85000198289818231D8F5998185E2989FC0014A
:10B860001124875C9B4F98878F83EF81F885858DA6
:10B870009927807F9070803A910519F481E48A833A
:10B880000BC0EF81F885858D9927807F9070803B74
:10B89000910511F482E48A83EF81F88582A18F3FBC
:10B8A00091F0EF81F88582A10E948603AA27BB2729
:10B8B0008B839C83AD83BE8389819927FC01ED5DD9
:10B8C000F64F8B81808389818F5F8983C2CF83E22A
:10B8D00099E00E94626B28960FB6F894DEBF0FBE07
:10B8E000CDBFDF91CF910895CF93DF93CDB7DEB772
:10B8F00021970FB6F894DEBF0FBECDBF8091330401
:10B90000833079F083E08093330419828981823215
:10B9100040F461E089810E94422A89818F5F898396
:10B92000F5CF21960FB6F894DEBF0FBECDBFDF91E5
:10B93000CF910895CF93DF93CDB7DEB78091A7095C
:10B94000882361F08091A709882341F00E94B15CAF
:10B950000E94F25C86E699E00E947D5DDF91CF91C6
:10B960000895CF93DF93CDB7DEB780912400806236
:10B9700080932400809125008F7D80932500809105
:10B980002400806480932400809125008F7B809325
:10B9900025008AEA8093800089E1809381001092DB
:10B9A00085001092840080E395E090938700809357
:10B9B0008600109289001092880010928B001092DD
:10B9C0008A0010928D0010928C0060E070E081E09F
:10B9D0000E942B5D60E070E082E00E942B5DDF91B1
:10B9E000CF910895CF93DF93CDB7DEB7109290003B
:10B9F00084E0809391001092950010929400109230
:10BA00009700109296001092990010929800109250
:10BA10009B0010929A0010929D0010929C00109230
:10BA2000630910926209109265091092640980916D
:10BA3000690088608093690010926A0080913D00DF
:10BA4000826080933D0080913C00826080933C0046
:10BA5000DF91CF910895CF93DF93CDB7DEB72797CE
:10BA60000FB6F894DEBF0FBECDBF89837B836A8398
:10BA70008A819B819D838C838981282F33273F83F3
:10BA80002E838E819F8182309105D9F02E813F8156
:10BA90002330310534F48E819F818130910539F056
:10BAA00023C02E813F8123303105A9F01DC08C8138
:10BAB0009D81892F9927809389008C8180938800AC
:10BAC00013C08C819D81892F992780938B008C8155
:10BAD00080938A0009C08C819D81892F992780934A
:10BAE0008D008C8180938C0027960FB6F894DEBF72
:10BAF0000FBECDBFDF91CF910895CF93DF93CDB728
:10BB0000DEB722970FB6F894DEBF0FBECDBF9A8383
:10BB10008983E981FA8111821082E981FA81138295
:10BB20001282E981FA8185E090E095838483E9813E
:10BB3000FA81168222960FB6F894DEBF0FBECDBFF3
:10BB4000DF91CF910895CF93DF93CDB7DEB76097A4
:10BB50000FB6F894DEBF0FBECDBF9A83898389816B
:10BB60009A81FC0136968081982F8F5F8083963072
:10BB700078F060E375E081E00E942B5D60E375E0A2
:10BB800082E00E942B5DE981FA8186E086838CC089
:10BB9000E981FA8182819381AA27BB278B839C83C9
:10BBA000AD83BE83E981FA8180819181AA27BB2779
:10BBB0008F839887A987BA872B813C814D815E81CD
:10BBC000DA01C901689412F8880F991FAA1FBB1FD8
:10BBD0001694D1F7820F931FA41FB51F820F931FD6
:10BBE000A41FB51F8B839C83AD83BE838B819C81F7
:10BBF000AD81BE8125E830E040E050E0BC01CD01E0
:10BC00000E9403BDDC01CB018B839C83AD83BE838B
:10BC10008B819C81AD81BE812F81388549855A8574
:10BC2000BC01CD010E9455BDDA01C9018B879C87FB
:10BC3000AD87BE878B859C85988B8F878F859889EC
:10BC400024E08A36920730F48F85988984349105F0
:10BC500008F004C080E395E0988B8F878091A70956
:10BC6000882351F08091F304803F31F46F85788907
:10BC700081E00E942B5D05C060E375E081E00E94D9
:10BC80002B5D8091A809882351F080911B06803F8D
:10BC900031F46F85788982E00E942B5D05C060E3F6
:10BCA00075E082E00E942B5D60960FB6F894DEBFCF
:10BCB0000FBECDBFDF91CF9108951F920F920FB6A7
:10BCC0000F9211242F933F938F939F93CF93DF93E2
:10BCD000CDB7DEB72297DEBFCDBF80919400992704
:10BCE0009A83898389819A81982F88279A83898367
:10BCF00080919500282F332789819A81822B932B5D
:10BD00009A8389838091690099278C7090708C3018
:10BD10009105F1F489819A8190936709809366096E
:10BD200010929400109295008091370490913804FD
:10BD3000909369098093680910923804109237042F
:10BD400010926C09809169008B7F8093690013C009
:10BD50008091690099278C7090708830910559F412
:10BD600089819A8190933804809337048091690087
:10BD70008460809369002296F894DEBFCDBFDF9186
:10BD8000CF919F918F913F912F910F900FBE0F9068
:10BD90001F901895CF93DF93CDB7DEB72C970FB6D2
:10BDA000F894DEBF0FBECDBFCE0101969D838C837C
:10BDB00080EE90E09F838E8383E090E09987888770
:10BDC000888599859B878A878A859B85AE81BF8177
:10BDD000EC81FD81019724F00E94C9BD0192FACF48
:10BDE0009B878A87CD019F838E83CF019D838C8320
:10BDF00043E050E060E571E0CE0101960E94C1A2EF
:10BE0000882331F10E94375F80E591E09B878A8724
:10BE100080EE90E09987888783E090E09F838E830F
:10BE20008E819F819D838C838C819D81A885B9851E
:10BE3000EA85FB85019724F001900E94D1BDFACFDD
:10BE40009D838C83CD0199878887CF019B878A87C3
:10BE50008FE7909124008923809324002C960FB6BD
:10BE6000F894DEBF0FBECDBFDF91CF910895CF9381
:10BE7000DF93CDB7DEB7A8970FB6F894DEBF0FBE3D
:10BE8000CDBFCE010C9644E150E060E070E00E942E
:10BE9000E9BC19828981883070F5CE010C9699A38E
:10BEA00088A3998184E1989FC00111248C519F4FF0
:10BEB0009BA38AA384E190E09DA38CA38CA19DA168
:10BEC0009FA38EA38EA19FA1AAA1BBA1E8A1F9A1C6
:10BED000019724F001900E94D1BDFACF9FA38EA3B9
:10BEE000CD019BA38AA3CF0199A388A3A89589819B
:10BEF0008F5F8983CFCF1A82CE0102969FA38EA334
:10BF000083EE90E09DA38CA381E090E09BA38AA3A5
:10BF10008AA19BA199A388A388A199A1ACA1BDA145
:10BF2000EEA1FFA1019724F001900E94D1BDFACFAC
:10BF300099A388A3CD019DA38CA3CF019FA38EA31A
:10BF4000A8960FB6F894DEBF0FBECDBFDF91CF919C
:10BF50000895CF93DF93CDB7DEB72A970FB6F89445
:10BF6000DEBF0FBECDBFCE0101969B838A8383EED9
:10BF700090E09D838C8381E090E09F838E838E810F
:10BF80009F819987888788859985AC81BD81EA8161
:10BF9000FB81019724F00E94C9BD0192FACF9987D5
:10BFA0008887CD019D838C83CF019B838A83898180
:10BFB000893010F088E08983898199272A960FB605
:10BFC000F894DEBF0FBECDBFDF91CF910895CF9320
:10BFD000DF93CDB7DEB7A0970FB6F894DEBF0FBEE4
:10BFE000CDBF89837B836A83CE010496998F888F26
:10BFF000998184E1989FC001112480539F4F9B8FAA
:10C000008A8F84E190E09D8F8C8F8C8D9D8D9F8F8A
:10C010008E8F8E8D9F8DAA8DBB8DE88DF98D0197AA
:10C0200024F00E94C9BD0192FACF9F8F8E8FCD015F
:10C030009B8F8A8FCF01998F888FCE01049644E120
:10C0400050E0BC018A819B810E94DCBCA0960FB6A7
:10C05000F894DEBF0FBECDBFDF91CF9108950F934F
:10C06000CF93DF93CDB7DEB7ED970FB6F894DEBF71
:10C070000FBECDBF9A8389837C836B835E834D83A0
:10C080002F830887CE0109969EAB8DAB83EE90E09F
:10C0900098AF8FAB81E090E09AAF89AF89AD9AAD50
:10C0A0009CAF8BAF8BAD9CADAFA9B8ADEDA9FEA990
:10C0B000019724F00E94C9BD0192FACF9CAF8BAFCB
:10C0C000CD0198AF8FABCF019EAB8DAB898588300A
:10C0D00008F04BC11C86CE01819644E150E060E03F
:10C0E00070E00E94E9BCCE01819669817A810E944C
:10C0F000F3BC1A869A858985981708F08FC08C85BD
:10C10000882309F08BC0CE010D969CAF8BAF9A852A
:10C1100084E1989FC00111248C519F4F9AAF89AF41
:10C1200084E190E098AF8FAB8FA998AD9EAB8DABBB
:10C130008DA99EA9A9ADBAADEBADFCAD019724F0D8
:10C140000E94C9BD0192FACF9EAB8DABCD019AAFD3
:10C1500089AFCF019CAF8BAF298D3A8D8B819C81AC
:10C160002817390709F056C0CE010D9646E050E079
:10C1700069817A810E94C1A2882309F04BC081E0C5
:10C180008C878B8D8A3008F0F0C08B8D8F5F8B8F02
:10C190008F81853010F084E08F83CE010D9640961C
:10C1A00044E050E060E070E00E94E9BC8F81282FFD
:10C1B0003327CE010D964096A9016D817E810E94A4
:10C1C000DCBCCE010D969CAF8BAF9A8584E1989F25
:10C1D000C00111248C519F4F9AAF89AF84E190E048
:10C1E00098AF8FAB8FA998AD9EAB8DAB8DA99EA953
:10C1F000A9ADBAADEBADFCAD019724F001900E9462
:10C20000D1BDFACF9EAB8DABCD019AAF89AFCF0137
:10C210009CAF8BAF8A858F5F8A876CCF8C85882394
:10C2200009F07FC08985883008F07BC089858F5FE1
:10C230008987CE010D964CE050E060E070E00E94EE
:10C24000E9BC89819A810E94FABC8B878B858C30EE
:10C2500010F08BE08B871A869A858B859817B8F437
:10C260008A85282F3327CE010196820F931FDC0188
:10C270001C968A85282F332789819A81F901E80F36
:10C28000F91F80818C938A858F5F8A87E5CF8B81A8
:10C290009C819A8F898F81E08B8F8F81853010F000
:10C2A00084E08F838F818C8FCE010D96409644E081
:10C2B00050E060E070E00E94E9BC8F81282F3327B6
:10C2C000CE010D964096A9016D817E810E94DCBC55
:10C2D000CE010D969CAF8BAF998584E1989FC001EC
:10C2E000112480539F4F9AAF89AF84E190E098AFBB
:10C2F0008FAB8FA998AD9EAB8DAB8DA99EA9A9AD33
:10C30000BAADEBADFCAD019724F001900E94D1BD18
:10C31000FACF9EAB8DABCD019AAF89AFCF019CAF69
:10C320008BAFCE0109969CAF8BAF83EE90E09AAFB6
:10C3300089AF81E090E098AF8FAB8FA998AD9EABAD
:10C340008DAB8DA99EA9A9ADBAADEBADFCAD0197A2
:10C3500024F001900E94D1BDFACF9EAB8DABCD01F0
:10C360009AAF89AFCF019CAF8BAFED960FB6F89423
:10C37000DEBF0FBECDBFDF91CF910F910895CF9358
:10C38000DF93CDB7DEB7DF91CF910895CF93DF93E1
:10C39000CDB7DEB729970FB6F894DEBF0FBECDBF7D
:10C3A00042E150E060E070E08AEE9DE00E94E9BC6E
:10C3B00040E150E060E070E08CEF9DE00E94E9BC5D
:10C3C0008EE19EE09A83898388E990E09C838B8349
:10C3D00082E190E09E838D838D819E8198878F83FB
:10C3E0008F819885AB81BC81E981FA81019724F026
:10C3F0000E94C9BD0192FACF98878F83CD019C839B
:10C400008B83CF019A83898380E39EE098878F8313
:10C410008AEA90E09E838D8382E190E09C838B8307
:10C420008B819C819A83898389819A81AD81BE8128
:10C43000EF81F885019724F00E94C9BD0192FACFDF
:10C440009A838983CD019E838D83CF0198878F83C3
:10C4500082E49EE098878F838CEB90E09E838D83AF
:10C4600080E190E09C838B838B819C819A8389837C
:10C4700089819A81AD81BE81EF81F885019724F091
:10C480000E94C9BD0192FACF9A838983CD019E8310
:10C490008D83CF0198878F838CE09EE098878F8370
:10C4A0008DEC90E09E838D8382E190E09C838B8372
:10C4B0008B819C819A83898389819A81AD81BE8198
:10C4C000EF81F885019724F00E94C9BD0192FACF4F
:10C4D0009A838983CD019E838D83CF0198878F8333
:10C4E00084E09AE098878F8385E990E09E838D832E
:10C4F00081E090E09C838B838B819C819A838983EC
:10C5000089819A81AD81BE81EF81F885019724F000
:10C510000E94C9BD0192FACF9A838983CD019E837F
:10C520008D83CF0198878F8385E09AE098878F83EA
:10C5300086E990E09E838D8382E090E09C838B83EC
:10C540008B819C819A83898389819A81AD81BE8107
:10C55000EF81F885019724F00E94C9BD0192FACFBE
:10C560009A838983CD019E838D83CF0198878F83A2
:10C5700029960FB6F894DEBF0FBECDBFDF91CF91E5
:10C580000895CF93DF93CDB7DEB76B970FB6F894CE
:10C59000DEBF0FBECDBF42E150E060E070E0CE01F3
:10C5A00001960E94E9BCCE0101969C8B8B8B88E999
:10C5B00090E09E8B8D8B82E190E0988F8F8B8F899E
:10C5C000988D9A8F898F898D9A8DAD89BE89EB89D7
:10C5D000FC89019724F001900E94D1BDFACF9A8F77
:10C5E000898FCD019E8B8D8BCF019C8B8B8BCE0148
:10C5F00001969A8F898F8AEA90E0988F8F8B82E1DB
:10C6000090E09E8B8D8B8D899E899C8B8B8B8B89EB
:10C610009C89AF89B88DE98DFA8D019724F001903E
:10C620000E94D1BDFACF9C8B8B8BCD01988F8F8BC5
:10C63000CF019A8F898FCE0101969A8F898F8CEBCB
:10C6400090E0988F8F8B80E190E09E8B8D8B8D8911
:10C650009E899C8B8B8B8B899C89AF89B88DE98D4A
:10C66000FA8D019724F001900E94D1BDFACF9C8BE6
:10C670008B8BCD01988F8F8BCF019A8F898FCE01B5
:10C6800001969A8F898F8DEC90E0988F8F8B82E145
:10C6900090E09E8B8D8B8D899E899C8B8B8B8B895B
:10C6A0009C89AF89B88DE98DFA8D019724F00190AE
:10C6B0000E94D1BDFACF9C8B8B8BCD01988F8F8B35
:10C6C000CF019A8F898F0E94C6616B960FB6F8943E
:10C6D000DEBF0FBECDBFDF91CF910895CF93DF9323
:10C6E000CDB7DEB72C970FB6F894DEBF0FBECDBF27
:10C6F0000E94782B898399818091040A891738F5E3
:10C7000089818093040A84E09AE09D838C8385E983
:10C7100090E09F838E8381E090E099878887888569
:10C7200099859B878A878A859B85AE81BF81EC81AD
:10C73000FD81019724F001900E94D1BDFACF9B8723
:10C740008A87CD019F838E83CF019D838C830E9436
:10C750006D2B9B838A832A813B818091050A90916E
:10C76000060A8217930750F58A819B819093060AE7
:10C770008093050A85E09AE09B878A8786E990E0A6
:10C780009987888782E090E09F838E838E819F8146
:10C790009D838C838C819D81A885B985EA85FB85E5
:10C7A000019724F001900E94D1BDFACF9D838C8324
:10C7B000CD0199878887CF019B878A872C960FB6F2
:10C7C000F894DEBF0FBECDBFDF91CF910895CF9318
:10C7D000DF93CDB7DEB78091040A9927DF91CF911F
:10C7E0000895CF93DF93CDB7DEB78091050A90917E
:10C7F000060ADF91CF910895CF93DF93CDB7DEB7CF
:10C8000024970FB6F894DEBF0FBECDBF1982898181
:10C81000823108F075C089819927FC01E651F24FF9
:10C8200080819927817090700097C1F18981992743
:10C83000DC01A651B24F89819927FC01E651F24FE4
:10C8400080818E7F8C938981992788569F4F9B8307
:10C850008A8389819927FC01E25EF14F80818C8374
:10C86000AA81BB818C81082E0E94D1BDBB83AA8383
:10C870008981992786559F4F9B838A838981992730
:10C88000FC01E05DF14F80818C83AA81BB818C81AA
:10C89000082E0E94D1BDBB83AA835EC089819927DF
:10C8A000FC01E651F24F80819927827090700097C9
:10C8B00019F189819927DC01A651B24F8981992705
:10C8C000FC01E651F24F80818D7F8C9389819927FD
:10C8D00083539F4F9B838A8389819927FC01E45F5F
:10C8E000F14F80818C83AA81BB818C81082E0E94AC
:10C8F000D1BDBB83AA8330C089818F5F898387CFF5
:10C9000019828981803140F589819927FC01E450A1
:10C91000F24F80818130E1F489819927FC01E45054
:10C92000F24F10828981992784549F4F9B838A8379
:10C9300089819927FC01EE5BF14F80818C83AA816C
:10C94000BB818C81082E0E94D1BDBB83AA8304C009
:10C9500089818F5F8983D5CF24960FB6F894DEBF87
:10C960000FBECDBFDF91CF910895CF93DF93CDB7A9
:10C97000DEB725970FB6F894DEBF0FBECDBF898313
:10C980007B836A83898181508D838981882309F41F
:10C990006AC08981833108F066C08D819927FC01C6
:10C9A000E25EF14F80819927807F90709595879501
:10C9B0009595879595958795959587958F30910550
:10C9C0000CF051C08D819927FC01E25EF14F80810E
:10C9D0009927807F907095958795959587959595E2
:10C9E0008795959587958C838C818F5F8C838D81BE
:10C9F0009927DC01A25EB14F8C8199279C01229579
:10CA00003295307F3227207F32278D819927FC0194
:10CA1000E25EF14F80818F70820F8C938A819B81BF
:10CA200083709070009719F081E08C8301C01C82A4
:10CA30008D819927FC01E05DF14F8A819B8196955C
:10CA40008795969587952C81820F80838D81992774
:10CA5000DC01A651B24F8D819927FC01E651F24FBE
:10CA6000808181608C9325960FB6F894DEBF0FBE4F
:10CA7000CDBFDF91CF910895CF93DF93CDB7DEB7D0
:10CA800023970FB6F894DEBF0FBECDBF898389818F
:10CA900081508B8389818823C9F189818331B0F5E5
:10CAA0008B819927FC01E25EF14F808199278F707D
:10CAB00090708F3091050CF052C08B819927FC014A
:10CAC000E25EF14F80818F708A838A818F5F8A83D3
:10CAD0008B819927DC01A25EB14F8B819927FC01E4
:10CAE000E25EF14F90EF808198238A81890F8C93C9
:10CAF0008B819927DC01A651B24F8B819927FC01CC
:10CB0000E651F24F808181608C9329C08981833105
:10CB100030F18981833218F5898183518B838B8130
:10CB20009927FC01EE5BF14F808199278F709070FF
:10CB30008F309105A4F48B819927DC01AE5BB14F56
:10CB40008B819927FC01EE5BF14F80818F5F8C9385
:10CB50008B819927FC01E450F24F81E0808323967A
:10CB60000FB6F894DEBF0FBECDBFDF91CF91089511
:10CB7000CF93DF93CDB7DEB722970FB6F894DEBF21
:10CB80000FBECDBF8983898181508A8389818823A3
:10CB900049F18981833130F58A819927FC01E45F6D
:10CBA000F14F808199278F7090708F309105D4F468
:10CBB0008A819927DC01A45FB14F8A819927FC0102
:10CBC000E45FF14F80818F5F8C938A819927DC012C
:10CBD000A651B24F8A819927FC01E651F24F80811C
:10CBE00082608C9322960FB6F894DEBF0FBECDBF45
:10CBF000DF91CF910895CF93DF93CDB7DEB7249720
:10CC00000FB6F894DEBF0FBECDBF898389818150F6
:10CC10008A8389818823C9F089818331B0F48A812C
:10CC20009927FC01E25EF14F8081882349F48A81D3
:10CC30009927FC01E45FF14F8081882309F41BC030
:10CC400081E090E09C838B8318C08981833198F0C8
:10CC50008981833280F4898183518A838A819927EB
:10CC6000FC01EE5BF14F8081882329F081E090E0A8
:10CC70009C838B8302C01C821B828B819C812496A7
:10CC80000FB6F894DEBF0FBECDBFDF91CF910895F0
:10CC9000CF93DF93CDB7DEB72B970FB6F894DEBFF7
:10CCA0000FBECDBF9A83898389819A819C838B83B0
:10CCB00080E991E09E838D838EE090E098878F835A
:10CCC0008F8198859A87898789859A85AD81BE816C
:10CCD000EB81FC81019724F001900E94D1BDFACF35
:10CCE0009A878987CD019E838D83CF019C838B8317
:10CCF00089819A810296E981FA81A981BA81AC0180
:10CD000061818C910E94822B2B960FB6F894DEBF26
:10CD10000FBECDBFDF91CF910895CF93DF93CDB7F5
:10CD2000DEB72B970FB6F894DEBF0FBECDBF9A8348
:10CD3000898389819A819C838B8380E991E09E839A
:10CD40008D838EE090E098878F838F8198859A8776
:10CD5000898789859A85AD81BE81EB81FC810197A8
:10CD600024F00E94C9BD0192FACF9A878987CD012C
:10CD70009E838D83CF019C838B832B960FB6F89473
:10CD8000DEBF0FBECDBFDF91CF910895CF93DF936C
:10CD9000CDB7DEB72B970FB6F894DEBF0FBECDBF71
:10CDA0009A83898389819A819C838B838EE991E020
:10CDB0009E838D838BE290E098878F838F81988507
:10CDC0009A87898789859A85AD81BE81EB81FC81AF
:10CDD000019724F001900E94D1BDFACF9A878987EC
:10CDE000CD019E838D83CF019C838B832B960FB6C1
:10CDF000F894DEBF0FBECDBFDF91CF910895CF93E2
:10CE0000DF93CDB7DEB72B970FB6F894DEBF0FBE1A
:10CE1000CDBF9A83898389819A819C838B838EE994
:10CE200091E09E838D838BE290E098878F838F8142
:10CE300098859A87898789859A85AD81BE81EB819E
:10CE4000FC81019724F00E94C9BD0192FACF9A8714
:10CE50008987CD019E838D83CF019C838B832B9605
:10CE60000FB6F894DEBF0FBECDBFDF91CF9108950E
:10CE7000CF93DF93CDB7DEB72B970FB6F894DEBF15
:10CE80000FBECDBF9A83898389819A819C838B83CE
:10CE900085EC9AE09E838D8388E090E098878F836D
:10CEA0008F8198859A87898789859A85AD81BE818A
:10CEB000EB81FC81019724F001900E94D1BDFACF53
:10CEC0009A878987CD019E838D83CF019C838B8335
:10CED0002B960FB6F894DEBF0FBECDBFDF91CF917A
:10CEE0000895CF93DF93CDB7DEB72B970FB6F894A5
:10CEF000DEBF0FBECDBF9A83898389819A819C83CF
:10CF00008B8385EC9AE09E838D8388E090E0988700
:10CF10008F838F8198859A87898789859A85AD8146
:10CF2000BE81EB81FC81019724F00E94C9BD019272
:10CF3000FACF9A878987CD019E838D83CF019C8309
:10CF40008B832B960FB6F894DEBF0FBECDBFDF915B
:10CF5000CF9108950F93CF93DF93CDB7DEB72E9780
:10CF60000FB6F894DEBF0FBECDBF89837B836A8383
:10CF70008981853060F000E021E0AE014F5F5F4FB6
:10CF800067E470E084E591E00E942F602DC09981F4
:10CF90008BE1989FC0011124895D914F9D838C8303
:10CFA0008A819B819F838E838C819D8199878887CD
:10CFB0008BE190E09B878A878A859B859D878C87FC
:10CFC0008C859D85A885B985EE81FF81019724F028
:10CFD00001900E94D1BDFACF9D878C87CD019987A2
:10CFE0008887CF019F838E832E960FB6F894DEBF7D
:10CFF0000FBECDBFDF91CF910F9108950F93CF93C7
:10D00000DF93CDB7DEB72E970FB6F894DEBF0FBE15
:10D01000CDBF89837B836A838981853060F000E09E
:10D0200021E0AE014F5F5F4F64E570E084E591E081
:10D030000E942F602DC099818BE1989FC00111241F
:10D04000895D914F9D838C838A819B819F838E8391
:10D050008C819D81998788878BE190E09B878A8767
:10D060008A859B859D878C878C859D85A885B985BC
:10D07000EE81FF81019724F00E94C9BD0192FACF91
:10D080009D878C87CD0199878887CF019F838E8369
:10D090002E960FB6F894DEBF0FBECDBFDF91CF91B5
:10D0A0000F9108950F93CF93DF93CDB7DEB72C97F1
:10D0B0000FB6F894DEBF0FBECDBF89837B836A8332
:10D0C0008981803260F000E021E0AE014F5F5F4F68
:10D0D00060E670E084E591E00E942F6029C08A81BB
:10D0E0009B819D838C8399818CE2989FC001112440
:10D0F0008D549D4F9F838E838CE290E09987888723
:10D10000888599859B878A878A859B85AE81BF8123
:10D11000EC81FD81019724F001900E94D1BDFACFEE
:10D120009B878A87CD019F838E83CF019D838C83CC
:10D130002C960FB6F894DEBF0FBECDBFDF91CF9116
:10D140000F9108950F93CF93DF93CDB7DEB72C9750
:10D150000FB6F894DEBF0FBECDBF89837B836A8391
:10D160008981803260F000E021E0AE014F5F5F4FC7
:10D170006AE670E084E591E00E942F6029C08A8110
:10D180009B819D838C8399818CE2989FC00111249F
:10D190008D549D4F9F838E838CE290E09987888782
:10D1A000888599859B878A878A859B85AE81BF8183
:10D1B000EC81FD81019724F00E94C9BD0192FACF54
:10D1C0009B878A87CD019F838E83CF019D838C832C
:10D1D0002C960FB6F894DEBF0FBECDBFDF91CF9176
:10D1E0000F9108950F93CF93DF93CDB7DEB72C97B0
:10D1F0000FB6F894DEBF0FBECDBF89837B836A83F1
:10D200008981843160F000E021E0AE014F5F5F4F23
:10D2100064E770E084E591E00E942F6029C08A8174
:10D220009B819D838C83998188E1989FC001112403
:10D230008B5C974F9F838E8388E190E099878887E6
:10D24000888599859B878A878A859B85AE81BF81E2
:10D25000EC81FD81019724F001900E94D1BDFACFAD
:10D260009B878A87CD019F838E83CF019D838C838B
:10D270002C960FB6F894DEBF0FBECDBFDF91CF91D5
:10D280000F9108950F93CF93DF93CDB7DEB72C970F
:10D290000FB6F894DEBF0FBECDBF89837B836A8350
:10D2A0008981843160F000E021E0AE014F5F5F4F83
:10D2B0006EE770E084E591E00E942F6029C08A81CA
:10D2C0009B819D838C83998188E1989FC001112463
:10D2D0008B5C974F9F838E8388E190E09987888746
:10D2E000888599859B878A878A859B85AE81BF8142
:10D2F000EC81FD81019724F00E94C9BD0192FACF13
:10D300009B878A87CD019F838E83CF019D838C83EA
:10D310002C960FB6F894DEBF0FBECDBFDF91CF9134
:10D320000F910895CF93DF93CDB7DEB7A2970FB6D5
:10D33000F894DEBF0FBECDBF9A8389836B838B8148
:10D34000882339F08B81833220F48B8181508B8349
:10D3500003C01AA219A249C0E981FA8180818C8395
:10D36000E981FA8181818D83E981FA8182818E83CD
:10D37000E981FA8183818F83E981FA8187818B87B3
:10D38000E981FA8187898B8FE981FA81808D8C8F81
:10D39000E981FA818481958199878887E981FA8179
:10D3A00086818A8789819A819C01285F3F4FCE01BF
:10D3B000049608964FE050E0B9010E94DCBC89E178
:10D3C0008E8F9B818E8D989FC00111248B52954F1B
:10D3D00098A38F8FCE0104966F8D78A10E94256B44
:10D3E0008D8F8D8D99279AA389A389A19AA1A29641
:10D3F0000FB6F894DEBF0FBECDBFDF91CF91089579
:10D40000CF93DF93CDB7DEB7A7970FB6F894DEBF03
:10D410000FBECDBF9A8389836B838B81882309F4E8
:10D4200067C08B81833208F063C08B8181508B830E
:10D430009B8189E1989FC00111248B52954F9E8F4B
:10D440008D8FCE01049698A38F8F8D8D9E8D9AA37C
:10D4500089A389E190E09CA38BA38BA19CA19EA3AF
:10D460008DA38DA19EA1A9A1BAA1EF8DF8A10197CD
:10D4700024F00E94C9BD0192FACF9EA38DA3CD01D5
:10D480009AA389A3CF0198A38F8FE981FA818C8118
:10D490008083E981FA818D818183E981FA818E819E
:10D4A0008283E981FA818F818383E981FA818B8587
:10D4B0008783E981FA818B8D878BE981FA818C8D55
:10D4C000808FE981FA818885998595838483E981B4
:10D4D000FA818A858683CE0104969C01285F3F4F9E
:10D4E00089819A8108964FE050E0B9010E94DCBC26
:10D4F000A7960FB6F894DEBF0FBECDBFDF91CF91D8
:10D500000895CF93DF93CDB7DEB72E970FB6F8947B
:10D51000DEBF0FBECDBF89837B836A838981882369
:10D5200009F43FC089818C3008F03BC0898181506B
:10D5300089838981992782959295907F9827807F0A
:10D5400098278B5E954F9D838C838A819B819F83D7
:10D550008E838981992782959295907F9827807FE5
:10D5600098278B5E954F9987888780E190E09B870D
:10D570008A878A859B859D878C878C859D85A885D4
:10D58000B985EE81FF81019724F001900E94D1BD01
:10D59000FACF9D878C87CD0199878887CF019F839C
:10D5A0008E832E960FB6F894DEBF0FBECDBFDF91EF
:10D5B000CF910895CF93DF93CDB7DEB72C970FB6F9
:10D5C000F894DEBF0FBECDBF89837B836A838981D8
:10D5D000882391F189818C3078F589818150898304
:10D5E0008A819B819D838C838981992782959295DD
:10D5F000907F9827807F98278B5E954F9F838E839F
:10D6000080E190E099878887888599859B878A87BC
:10D610008A859B85AE81BF81EC81FD81019724F0D5
:10D620000E94C9BD0192FACF9B878A87CD019F8353
:10D630008E83CF019D838C832C960FB6F894DEBF2A
:10D640000FBECDBFDF91CF910895CF93DF93CDB7BC
:10D65000DEB72D970FB6F894DEBF0FBECDBF9A830D
:10D6600089837C836B8389819A819E838D838B815F
:10D670009C8198878F8389E190E09A878987898543
:10D680009A859C878B878B859C85AF81B885ED813A
:10D69000FE81019724F001900E94D1BDFACF9C87B2
:10D6A0008B87CD0198878F83CF019E838D8381E007
:10D6B00090E02D960FB6F894DEBF0FBECDBFDF9180
:10D6C000CF910895CF93DF93CDB7DEB72B970FB6E9
:10D6D000F894DEBF0FBECDBF9A83898389819A817A
:10D6E0009C838B8380E190E09E838D8382E190E038
:10D6F00098878F838F8198859A87898789859A856E
:10D70000AD81BE81EB81FC81019724F001900E94E4
:10D71000D1BDFACF9A878987CD019E838D83CF01B2
:10D720009C838B832B960FB6F894DEBF0FBECDBFC4
:10D73000DF91CF910895CF93DF93CDB7DEB72B97CD
:10D740000FB6F894DEBF0FBECDBF9A83898389815F
:10D750009A819C838B8380E190E09E838D8382E11C
:10D7600090E098878F838F8198859A8789878985AC
:10D770009A85AD81BE81EB81FC81019724F00E94E6
:10D78000C9BD0192FACF9A878987CD019E838D8387
:10D79000CF019C838B832B960FB6F894DEBF0FBE10
:10D7A000CDBFDF91CF910895CF93DF93CDB7DEB793
:10D7B0002B970FB6F894DEBF0FBECDBF9A83898337
:10D7C00089819A819C838B8380E390E09E838D8303
:10D7D00084E290E098878F838F8198859A878987E4
:10D7E00089859A85AD81BE81EB81FC81019724F00A
:10D7F00001900E94D1BDFACF9A878987CD019E837F
:10D800008D83CF019C838B832B960FB6F894DEBF5C
:10D810000FBECDBFDF91CF910895CF93DF93CDB7EA
:10D82000DEB72B970FB6F894DEBF0FBECDBF9A833D
:10D83000898389819A819C838B8380E390E09E8396
:10D840008D8384E290E098878F838F8198859A8773
:10D85000898789859A85AD81BE81EB81FC8101979D
:10D8600024F00E94C9BD0192FACF9A878987CD0121
:10D870009E838D83CF019C838B832B960FB6F89468
:10D88000DEBF0FBECDBFDF91CF910895CF93DF9361
:10D89000CDB7DEB72D970FB6F894DEBF0FBECDBF64
:10D8A0009A83898389EC91E09C838B8389819A8117
:10D8B0009E838D838B819C8198878F8388E190E004
:10D8C0009A87898789859A859C878B878B859C8594
:10D8D000AF81B885ED81FE81019724F001900E940F
:10D8E000D1BDFACF9C878B87CD0198878F83CF01DD
:10D8F0009E838D832D960FB6F894DEBF0FBECDBFED
:10D90000DF91CF910895CF93DF93CDB7DEB72D97F9
:10D910000FB6F894DEBF0FBECDBF9A83898389EC22
:10D9200091E09C838B8389819A819E838D838B81F7
:10D930009C8198878F8388E190E09A878987898581
:10D940009A859C878B878B859C85AF81B885ED8177
:10D95000FE81019724F00E94C9BD0192FACF9C87F5
:10D960008B87CD0198878F83CF019E838D832D96E2
:10D970000FB6F894DEBF0FBECDBFDF91CF910895F3
:10D980000F93CF93DF93CDB7DEB72D970FB6F894F3
:10D99000DEBF0FBECDBF9A838983E981FA81808182
:10D9A000882329F481EE91E09C838B831FC0E98159
:10D9B000FA818081813029F487E292E09C838B8315
:10D9C00015C0E981FA818081823029F48DE692E0E8
:10D9D0009C838B830BC000E021E049815A8167E47E
:10D9E00071E084E591E00E942F6024C089819A81D2
:10D9F0009E838D838B819C8198878F8386E490E0C2
:10DA00009A87898789859A859C878B878B859C8552
:10DA1000AF81B885ED81FE81019724F001900E94CD
:10DA2000D1BDFACF9C878B87CD0198878F83CF019B
:10DA30009E838D832D960FB6F894DEBF0FBECDBFAB
:10DA4000DF91CF910F9108950F93CF93DF93CDB7CF
:10DA5000DEB72E970FB6F894DEBF0FBECDBF898319
:10DA60007B836A838981882329F481EE91E09D83F9
:10DA70008C831CC08981813029F487E292E09D83E8
:10DA80008C8314C08981823029F48DE692E09D83D5
:10DA90008C830CC000E021E0AE014F5F5F4F60E679
:10DAA00071E084E591E00E942F6024C08A819B810F
:10DAB0009F838E838C819D819987888786E490E0FF
:10DAC0009B878A878A859B859D878C878C859D858A
:10DAD000A885B985EE81FF81019724F00E94C9BD18
:10DAE0000192FACF9D878C87CD0199878887CF01D6
:10DAF0009F838E832E960FB6F894DEBF0FBECDBFE8
:10DB0000DF91CF910F910895CF93DF93CDB7DEB71B
:10DB10006B970FB6F894DEBF0FBECDBFCE01019656
:10DB20009A8B898B1C8A1B8A80E190E09E8B8D8B5F
:10DB30008D899E89988F8F8B8F89988DAB89BC89B1
:10DB4000E989FA89019724F00E94C9BD0192FACFB0
:10DB5000988F8F8BCD019C8B8B8BCF019A8B898B70
:10DB60008B858F3129F48FE190E09B8F8A8F0CC0D9
:10DB70008B85803229F480E290E09B8F8A8F04C0ED
:10DB80008FE190E09B8F8A8F8A8D9B8D6B960FB66D
:10DB9000F894DEBF0FBECDBFDF91CF910895CF9334
:10DBA000DF93CDB7DEB7AA970FB6F894DEBF0FBEEE
:10DBB000CDBFCE0101969BA38AA31DA21CA284E027
:10DBC00090E09FA38EA38EA19FA199A788A788A567
:10DBD00099A5ACA1BDA1EAA1FBA1019724F00E94E7
:10DBE000C9BD0192FACF99A788A7CD019DA38CA3A7
:10DBF000CF019BA38AA344E050E068E671E0CE0128
:10DC000001960E94C1A2882309F498C04EE150E019
:10DC100060E070E0CE0101960E94E9BCCE01019661
:10DC200098A38F8F45E050E068E671E08F8D98A152
:10DC30000E94DCBC8F8D98A1049644E050E060E027
:10DC400070E00E94E9BCEF8DF8A11086EF8DF8A17D
:10DC50001186EF8DF8A112860E947D418F8D98A1CB
:10DC600099A788A71FA21EA280E190E09DA38CA384
:10DC70008CA19DA19BA38AA38AA19BA1AEA1BFA1B8
:10DC8000E8A5F9A5019724F001900E94D1BDFACF33
:10DC90009BA38AA3CD019FA38EA3CF0199A788A799
:10DCA000CE01019699A788A71FA21EA284E090E04A
:10DCB0009DA38CA38CA19DA19BA38AA38AA19BA1B8
:10DCC000AEA1BFA1E8A5F9A5019724F001900E949B
:10DCD000D1BDFACF9BA38AA3CD019FA38EA3CF0171
:10DCE00099A788A744E150E060E070E0CE0101967A
:10DCF0000E94E9BCCE01019699A788A78EE19FE01A
:10DD00009FA38EA384E190E09DA38CA38CA19DA1F1
:10DD10009BA38AA38AA19BA1AEA1BFA1E8A5F9A557
:10DD2000019724F001900E94D1BDFACF9BA38AA352
:10DD3000CD019FA38EA3CF0199A788A7CE010196FD
:10DD400099A788A780E891E09FA38EA38AE090E03E
:10DD50009DA38CA38CA19DA19BA38AA38AA19BA117
:10DD6000AEA1BFA1E8A5F9A5019724F00E94C9BD05
:10DD70000192FACF9BA38AA3CD019FA38EA3CF01CB
:10DD800099A788A74AE050E06FE871E0CE010196BC
:10DD90000E94C1A2882309F460C00E94B5410E947C
:10DDA000B0190E9428A70E945D080E94CD164EE17E
:10DDB00050E060E070E0CE0101960E94E9BC6DE6A3
:10DDC00071E0CE0101960E94F3BCCE01019699A7A5
:10DDD00088A780E790E09FA38EA380E190E09DA3B9
:10DDE0008CA38CA19DA19BA38AA38AA19BA1AEA178
:10DDF000BFA1E8A5F9A5019724F001900E94D1BD2B
:10DE0000FACF9BA38AA3CD019FA38EA3CF0199A78D
:10DE100088A78FE891E099A788A780E891E09FA361
:10DE20008EA38AE090E09DA38CA38CA19DA19BA3CF
:10DE30008AA38AA19BA1AEA1BFA1E8A5F9A50197DC
:10DE400024F001900E94D1BDFACF9BA38AA3CD01FB
:10DE50009FA38EA3CF0199A788A7CE01019699A76A
:10DE600088A780EE90E09FA38EA383E090E09DA31F
:10DE70008CA38CA19DA19BA38AA38AA19BA1AEA1E7
:10DE8000BFA1E8A5F9A5019724F00E94C9BD0192A0
:10DE9000FACF9BA38AA3CD019FA38EA3CF0199A7FD
:10DEA00088A743E050E066E771E0CE0101960E944A
:10DEB000C1A2882331F10E94375F86E791E099A7DC
:10DEC00088A780EE90E09FA38EA383E090E09DA3BF
:10DED0008CA38CA19DA19BA38AA38AA19BA1AEA187
:10DEE000BFA1E8A5F9A5019724F001900E94D1BD3A
:10DEF000FACF9BA38AA3CD019FA38EA3CF0199A79D
:10DF000088A7CE01019699A788A780E990E09FA3F2
:10DF10008EA385E090E09DA38CA38CA19DA19BA3E3
:10DF20008AA38AA19BA1AEA1BFA1E8A5F9A50197EB
:10DF300024F00E94C9BD0192FACF9BA38AA3CD0110
:10DF40009FA38EA3CF0199A788A745E050E06AE779
:10DF500071E0CE0101960E94C1A2882309F404C198
:10DF60004EE150E060E070E0CE0101960E94E9BC15
:10DF7000CE01019699A788A78CEC90E09FA38EA371
:10DF800081E090E09DA38CA38CA19DA19BA38AA37B
:10DF90008AA19BA1AEA1BFA1E8A5F9A5019724F094
:10DFA00001900E94D1BDFACF9BA38AA3CD019FA36C
:10DFB0008EA3CF0199A788A7CE01019699A788A71C
:10DFC00085E990E09FA38EA381E090E09DA38CA3C0
:10DFD0008CA19DA19BA38AA38AA19BA1AEA1BFA155
:10DFE000E8A5F9A5019724F001900E94D1BDFACFD0
:10DFF0009BA38AA3CD019FA38EA3CF0199A788A736
:10E00000CE01019699A788A786E990E09FA38EA3E9
:10E0100082E090E09DA38CA38CA19DA19BA38AA3E9
:10E020008AA19BA1AEA1BFA1E8A5F9A5019724F003
:10E0300001900E94D1BDFACF9BA38AA3CD019FA3DB
:10E040008EA3CF0199A788A7CE01019699A788A78B
:10E0500088E990E09FA38EA382E190E09DA38CA32A
:10E060008CA19DA19BA38AA38AA19BA1AEA1BFA1C4
:10E07000E8A5F9A5019724F001900E94D1BDFACF3F
:10E080009BA38AA3CD019FA38EA3CF0199A788A7A5
:10E09000CE01019699A788A78CEB90E09FA38EA351
:10E0A00080E190E09DA38CA38CA19DA19BA38AA35A
:10E0B0008AA19BA1AEA1BFA1E8A5F9A5019724F073
:10E0C00001900E94D1BDFACF9BA38AA3CD019FA34B
:10E0D0008EA3CF0199A788A7CE01019699A788A7FB
:10E0E0008DEC90E09FA38EA382E190E09DA38CA392
:10E0F0008CA19DA19BA38AA38AA19BA1AEA1BFA134
:10E10000E8A5F9A5019724F001900E94D1BDFACFAE
:10E110009BA38AA3CD019FA38EA3CF0199A788A714
:10E120008AE791E099A788A780E990E09FA38EA352
:10E1300085E090E09DA38CA38CA19DA19BA38AA3C5
:10E140008AA19BA1AEA1BFA1E8A5F9A5019724F0E2
:10E1500001900E94D1BDFACF9BA38AA3CD019FA3BA
:10E160008EA3CF0199A788A7CE01019699A788A76A
:10E170008EE19FE09FA38EA389E090E09DA38CA3F6
:10E180008CA19DA19BA38AA38AA19BA1AEA1BFA1A3
:10E19000E8A5F9A5019724F00E94C9BD0192FACF24
:10E1A0009BA38AA3CD019FA38EA3CF0199A788A784
:10E1B00019A289A1883008F054C089A1282F3327DB
:10E1C000CE010196F901E80FF91F808118160CF0B5
:10E1D00048C089A1282F3327CE010196F901E80F05
:10E1E000F91F8081803364F089A1282F3327CE0165
:10E1F0000196F901E80FF91F80818A330CF42DC0D4
:10E2000049E050E060E070E0CE0101960E94E9BC78
:10E21000CE01019699A788A78EE19FE09FA38EA3C8
:10E2200089E090E09DA38CA38CA19DA19BA38AA3D0
:10E230008AA19BA1AEA1BFA1E8A5F9A5019724F0F1
:10E2400001900E94D1BDFACF9BA38AA3CD019FA3C9
:10E250008EA3CF0199A788A704C089A18F5F89A346
:10E26000A8CFCE01019699A788A787E29FE09FA338
:10E270008EA389E090E09DA38CA38CA19DA19BA37C
:10E280008AA38AA19BA1AEA1BFA1E8A5F9A5019788
:10E2900024F00E94C9BD0192FACF9BA38AA3CD01AD
:10E2A0009FA38EA3CF0199A788A719A289A188301F
:10E2B00008F054C089A1282F3327CE010196F90117
:10E2C000E80FF91F808118160CF048C089A1282F8B
:10E2D0003327CE010196F901E80FF91F80818033C1
:10E2E00064F089A1282F3327CE010196F901E80FA8
:10E2F000F91F80818A330CF42DC049E050E060E0C2
:10E3000070E0CE0101960E94E9BCCE01019699A76A
:10E3100088A787E29FE09FA38EA389E090E09DA35A
:10E320008CA38CA19DA19BA38AA38AA19BA1AEA132
:10E33000BFA1E8A5F9A5019724F001900E94D1BDE5
:10E34000FACF9BA38AA3CD019FA38EA3CF0199A748
:10E3500088A704C089A18F5F89A3A8CFAA960FB60A
:10E36000F894DEBF0FBECDBFDF91CF910895C4EF0B
:10E37000D0E1DEBFCDBF0E9466A00E9468740E94FB
:10E38000BD2B0E94EB060E949DA00E941E850E944C
:10E39000CA5E0E94CF6D8AEB9DE09A83898380E8F4
:10E3A00090E09C838B8380E190E09E838D838D81C0
:10E3B0009E8198878F838F819885AB81BC81E9810D
:10E3C000FA81019724F00E94C9BD0192FACF988783
:10E3D0008F83CD019C838B83CF019A838983809126
:10E3E000BA0D9091BB0D9B878A878A859B858A3F52
:10E3F000910589F18A859B858B3F910558F48A8523
:10E400009B858436910599F08A859B858D3791058A
:10E41000C1F03EC08A859B8521E0843F920729F1A7
:10E420008A859B8523E0883E920749F131C086E2C8
:10E430008093E20084E08093E30083E18093E40032
:10E4400027C08EE18093E20084E08093E30083E1C3
:10E450008093E4001DC08EE08093E20084E080930E
:10E46000E30083E18093E40013C086E08093E20040
:10E4700084E08093E30083E18093E40009C082E0BC
:10E480008093E20084E08093E30083E18093E400E2
:10E490000E942A178091BC0D9091BD0D8530910589
:10E4A00038F485E090E09093BD0D8093BC0D0EC0D4
:10E4B0008091BC0D9091BD0D27E0813D920730F019
:10E4C00080ED97E09093BD0D8093BC0D8091BE0DC3
:10E4D0009091BF0D28E08030920760F08091BE0DD2
:10E4E0009091BF0D29E08939920721F01092BF0D5C
:10E4F0001092BE0D8091C60D992781709070009783
:10E5000021F082E08093CC0D02C01092CC0D80915E
:10E51000C60D992782709070009721F082E0809359
:10E52000CF0D02C01092CF0D8091C60D9927847037
:10E530009070009721F082E08093DA0D02C0109273
:10E54000DA0D8091C70D8A3028F08091C70D8B3F7E
:10E5500008F403C08FE48093C70D0E9499780E944D
:10E5600055A60E94C5430E943E8487E00E9427B7BB
:10E5700078940E94309EA89580E00E9459840E9461
:10E580002F85FACFCF93DF93CDB7DEB723970FB6A2
:10E59000F894DEBF0FBECDBF89836A8380913400BB
:10E5A000877F809334008981992787709070880FC6
:10E5B000991F81640E947EA08A810E947EA080E0D3
:10E5C0000E947EA08B838091340088608093340009
:10E5D0008B81992723960FB6F894DEBF0FBECDBF6F
:10E5E000DF91CF910895CF93DF93CDB7DEB7239717
:10E5F0000FB6F894DEBF0FBECDBF89836A834B830D
:10E6000080913400877F80933400898199278770B7
:10E610009070880F991F80640E947EA08A810E945A
:10E620007EA08B810E947EA08091340088608093C0
:10E63000340023960FB6F894DEBF0FBECDBFDF9136
:10E64000CF910895CF93DF93CDB7DEB78091070ABE
:10E65000882389F581E08093070A4CE16AE080E035
:10E660000E94F37240E060E080E00E94F3724FEF9E
:10E6700061E080E00E94F37240E062E080E00E948E
:10E68000F37240E063E080E00E94F37240E064E0F7
:10E6900080E00E94F37240E065E080E00E94F37247
:10E6A00040E06CE080E00E94F37240E06DE080E0CA
:10E6B0000E94F3720AC18091070A813089F54CE10A
:10E6C0006AE081E00E94F37240E060E081E00E9435
:10E6D000F3724FEF61E081E00E94F37240E062E08C
:10E6E00081E00E94F37240E063E081E00E94F372F7
:10E6F00040E064E081E00E94F37240E065E081E088
:10E700000E94F37240E06CE081E00E94F37240E00E
:10E710006DE081E00E94F37282E08093070AD5C029
:10E720008091070A823089F54CE16AE082E00E941C
:10E73000F37240E060E082E00E94F3724FEF61E02C
:10E7400082E00E94F37240E062E082E00E94F37295
:10E7500040E063E082E00E94F37240E064E082E027
:10E760000E94F37240E065E082E00E94F37240E0B4
:10E770006CE082E00E94F37240E06DE082E00E9473
:10E78000F37283E08093070AA0C08091070A833068
:10E7900089F54CE16AE083E00E94F37240E060E0BA
:10E7A00083E00E94F3724FEF61E083E00E94F37216
:10E7B00040E062E083E00E94F37240E063E083E0C7
:10E7C0000E94F37240E064E083E00E94F37240E054
:10E7D00065E083E00E94F37240E06CE083E00E9419
:10E7E000F37240E06DE083E00E94F37284E0809376
:10E7F000070A6BC08091070A843089F54CE16AE012
:10E8000084E00E94F3724CEF60E084E00E94F372B7
:10E810004FEF61E084E00E94F37240E062E084E048
:10E820000E94F37240E063E084E00E94F37240E0F3
:10E8300064E084E00E94F37240E065E084E00E94BE
:10E84000F37240E06CE084E00E94F37240E06DE01F
:10E8500084E00E94F37285E08093070A36C08091BD
:10E86000070A853081F54CE16AE085E00E94F37289
:10E8700040E060E085E00E94F37240EF61E085E0F7
:10E880000E94F37240E062E085E00E94F37240E093
:10E8900063E085E00E94F37240E064E085E00E945E
:10E8A000F37240E065E085E00E94F37240E06CE0C6
:10E8B00085E00E94F37240E06DE085E00E94F37213
:10E8C0001092070A02C01092070ADF91CF910895B3
:10E8D000CF93DF93CDB7DEB780913300886080930C
:10E8E0003300809134008860809334004CE16AE00A
:10E8F00080E00E94F37240E064E180E00E94F372E5
:10E9000040E060E080E00E94F3724FEF61E080E061
:10E910000E94F37240E062E080E00E94F37240E007
:10E9200063E080E00E94F37240E064E080E00E94D7
:10E93000F37240E065E080E00E94F37240E06CE03A
:10E9400080E00E94F37240E06DE080E00E94F3728C
:10E950004CE16AE081E00E94F37240E064E181E012
:10E960000E94F37240E060E081E00E94F3724FEF9A
:10E9700061E081E00E94F37240E062E081E00E9489
:10E98000F37240E063E081E00E94F37240E064E0F3
:10E9900081E00E94F37240E065E081E00E94F37242
:10E9A00040E06CE081E00E94F37240E06DE081E0C5
:10E9B0000E94F3724CE16AE082E00E94F37240E050
:10E9C00064E182E00E94F37240E060E082E00E9435
:10E9D000F3724FEF61E082E00E94F37240E062E088
:10E9E00082E00E94F37240E063E082E00E94F372F2
:10E9F00040E064E082E00E94F37240E065E082E083
:10EA00000E94F37240E06CE082E00E94F37240E00A
:10EA10006DE082E00E94F3724CE16AE083E00E94C4
:10EA2000F37240E064E183E00E94F37240E060E052
:10EA300083E00E94F3724FEF61E083E00E94F37283
:10EA400040E062E083E00E94F37240E063E083E034
:10EA50000E94F37240E064E083E00E94F37240E0C1
:10EA600065E083E00E94F37240E06CE083E00E9486
:10EA7000F37240E06DE083E00E94F3724CE16AE0E3
:10EA800084E00E94F37240E064E184E00E94F3724B
:10EA90004CEF60E084E00E94F3724FEF61E084E0AD
:10EAA0000E94F37240E062E084E00E94F37240E072
:10EAB00063E084E00E94F37240E064E084E00E943E
:10EAC000F37240E065E084E00E94F37240E06CE0A5
:10EAD00084E00E94F37240E06DE084E00E94F372F3
:10EAE0004CE16AE085E00E94F37240E064E185E079
:10EAF0000E94F37240E065E185E00E94F37240E01D
:10EB000060E085E00E94F37240EF61E085E00E94E2
:10EB1000F37240E062E085E00E94F37240E063E05F
:10EB200085E00E94F37240E064E085E00E94F372A9
:10EB300040E065E085E00E94F37240E06CE085E033
:10EB40000E94F37240E06DE085E00E94F372DF9175
:10EB5000CF910895CF93DF93CDB7DEB72C970FB643
:10EB6000F894DEBF0FBECDBF89836A834B831C82BE
:10EB70001E821D828A81813621F421E030E03E83AD
:10EB80002D8318861F828A81813421F481E090E0F0
:10EB900098878F838D819E812F813885822B932B3F
:10EBA0000097B9F060E08B810E94C2728C838981EA
:10EBB000282F332781E090E002C0880F991F2A9503
:10EBC000E2F72C81822B8C834C8160E08B810E9448
:10EBD000F3721A8619868A81823621F481E090E0E8
:10EBE0009A8789871C861B868A81823421F421E0DA
:10EBF00030E03C872B8789859A852B853C85822B45
:10EC0000932B0097B9F061E08B810E94C2728C83D4
:10EC10008981282F332781E090E002C0880F991F57
:10EC20002A95E2F72C81822B8C834C8161E08B81C9
:10EC30000E94F3722C960FB6F894DEBF0FBECDBFC4
:10EC4000DF91CF910895CF93DF93CDB7DEB72C97A7
:10EC50000FB6F894DEBF0FBECDBF89836A834B83A6
:10EC60001C821E821D828A81813621F421E030E0DF
:10EC70003E832D8318861F828A81813421F481E0AE
:10EC800090E098878F838D819E812F813885822B9C
:10EC9000932B0097C9F060E08B810E94C2728C8335
:10ECA0008981282F332781E090E002C0880F991FC7
:10ECB0002A95E2F7982F90958C8189238C834C813B
:10ECC00060E08B810E94F3721A8619868A818236EF
:10ECD00021F481E090E09A8789871C861B868A81CF
:10ECE000823421F421E030E03C872B8789859A85A6
:10ECF0002B853C85822B932B0097C9F061E08B819B
:10ED00000E94C2728C838981282F332781E090E092
:10ED100002C0880F991F2A95E2F7982F90958C8151
:10ED200089238C834C8161E08B810E94F3722C9645
:10ED30000FB6F894DEBF0FBECDBFDF91CF9108951F
:10ED4000CF93DF93CDB7DEB72B970FB6F894DEBF26
:10ED50000FBECDBF89836A834B831D821C828A814B
:10ED6000813621F421E030E03D832C831F821E8216
:10ED70008A81813421F481E090E09F838E838C81AD
:10ED80009D812E813F81822B932B009729F0498111
:10ED900064E18B810E94F372198618868A8182361B
:10EDA00021F481E090E0998788871B861A868A8102
:10EDB000823421F421E030E03B872A8788859985D9
:10EDC0002A853B85822B932B009729F0498165E1A9
:10EDD0008B810E94F3722B960FB6F894DEBF0FBEA4
:10EDE000CDBFDF91CF910895CF93DF93CDB7DEB73D
:10EDF0002C970FB6F894DEBF0FBECDBF89836A8310
:10EE00004B831C821E821D828A81813621F421E07F
:10EE100030E03E832D8318861F828A81813421F45D
:10EE200081E090E098878F838D819E812F81388546
:10EE3000822B932B009791F062E18B810E94C2722A
:10EE40008C838981282F332781E090E002C0880FCE
:10EE5000991F2A95E2F72C81822B8C831A861986BA
:10EE60008A81823621F481E090E09A8789871C8626
:10EE70001B868A81823421F421E030E03C872B8795
:10EE800089859A852B853C85822B932B009791F061
:10EE900063E18B810E94C2728C838981282F332782
:10EEA00081E090E002C0880F991F2A95E2F72C813B
:10EEB000822B8C834B816A818C810E94A0762C9658
:10EEC0000FB6F894DEBF0FBECDBFDF91CF9108958E
:10EED000CF93DF93CDB7DEB72C970FB6F894DEBF94
:10EEE0000FBECDBF89836A834B831C821E821D8225
:10EEF0008A81813621F421E030E03E832D8318861B
:10EF00001F828A81813421F481E090E098878F8389
:10EF10008D819E812F813885822B932B0097A9F0BC
:10EF200062E18B810E94C2728C838981282F3327F2
:10EF300081E090E0022E02C0880F991F0A94E2F748
:10EF4000982F90958C8189238C831A8619868A81C3
:10EF5000823621F481E090E09A8789871C861B869F
:10EF60008A81823421F421E030E03C872B87898537
:10EF70009A852B853C85822B932B0097A1F063E12A
:10EF80008B810E94C2728C838981282F332781E074
:10EF900090E002C0880F991F2A95E2F7982F90956C
:10EFA0008C8189238C834B816A818C810E94A0761D
:10EFB0002C960FB6F894DEBF0FBECDBFDF91CF9178
:10EFC0000895CF93DF93CDB7DEB72B970FB6F894A4
:10EFD000DEBF0FBECDBF89836A831B821D821C8268
:10EFE0008981813621F421E030E03D832C831F822A
:10EFF0001E828981813421F481E090E09F838E8399
:10F000008C819D812E813F81822B932B009729F04B
:10F0100062E18A810E94C2728B8319861886898177
:10F02000823621F481E090E0998788871B861A86D2
:10F030008981823421F421E030E03B872A8788856A
:10F0400099852A853B85822B932B009729F063E1D4
:10F050008A810E94C2728B838B8199272B960FB66F
:10F06000F894DEBF0FBECDBFDF91CF910895CF934F
:10F07000DF93CDB7DEB72C970FB6F894DEBF0FBE87
:10F08000CDBF89836A834B831C821E821D828A8145
:10F09000813621F421E030E03E832D8318861F82E3
:10F0A0008A81813421F481E090E098878F838D817B
:10F0B0009E812F813885822B932B009729F062E166
:10F0C0008B810E94C2728C831A8619868A8182364D
:10F0D00021F481E090E09A8789871C861B868A81CB
:10F0E000823421F421E030E03C872B8789859A85A2
:10F0F0002B853C85822B932B009729F063E18B8134
:10F100000E94C2728C838981282F332781E090E08E
:10F1100002C0880F991F2A95E2F72C818223992734
:10F120002C960FB6F894DEBF0FBECDBFDF91CF9106
:10F130000895CF93DF93CDB7DEB70E944C1F85E6CD
:10F140009AE09093FC0A8093FB0A1092FD0A1092B9
:10F15000F40A1092F50A84EF9AE00E945A1F88235D
:10F1600009F0F9CF1092F30A8DE69AE09093080B1C
:10F170008093070B1092090B1092000B1092010B59
:10F1800080E09BE00E945A1F882309F0F9CF10927B
:10F19000FF0A85E79AE09093140B8093130B10926B
:10F1A000150B10920C0B10920D0B8CE09BE00E9443
:10F1B0005A1F882309F0F9CF10920B0B8DE79AE0C4
:10F1C0009093200B80931F0B1092210B1092180B21
:10F1D0001092190B88E19BE00E945A1F882309F0C6
:10F1E000F9CF1092170B85E19AE090938D0A8093E6
:10F1F0008C0A10928E0A1092850A82E08093860A09
:10F2000085E89AE00E945A1F882309F0F9CF8DE122
:10F210009AE09093980A8093970A1092990A109214
:10F22000900A82E08093910A80E99AE00E945A1F36
:10F23000882309F0F9CF85E29AE09093A30A80939E
:10F24000A20A1092A40A10929B0A82E080939C0A60
:10F250008BE99AE00E945A1F882309F0F9CF8DE2CA
:10F260009AE09093AE0A8093AD0A1092AF0A109282
:10F27000A60A82E08093A70A86EA9AE00E945A1FB3
:10F28000882309F0F9CF85E39AE09093B90A809337
:10F29000B80A1092BA0A1092B10A82E08093B20AB8
:10F2A00081EB9AE00E945A1F882309F0F9CF8DE381
:10F2B0009AE09093C40A8093C30A1092C50A1092F0
:10F2C000BC0A82E08093BD0A8CEB9AE00E945A1F30
:10F2D000882309F0F9CF85E49AE09093CF0A8093D0
:10F2E000CE0A1092D00A1092C70A82E08093C80A10
:10F2F00087EC9AE00E945A1F882309F0F9CF8DE429
:10F300009AE09093DA0A8093D90A1092DB0A10925D
:10F31000D20A82E08093D30A82ED9AE00E945A1FBB
:10F32000882309F0F9CF85E59AE09093E50A809368
:10F33000E40A1092E60A1092DD0A82E08093DE0A67
:10F340008DED9AE00E945A1F882309F0F9CF8DE5D0
:10F350009AE09093F00A8093EF0A1092F10A1092CB
:10F36000E80A82E08093E90A88EE9AE00E945A1F38
:10F37000882309F0F9CFDF91CF910895CF93DF93E0
:10F38000CDB7DEB78091F30A8823D1F08091F30ADC
:10F39000813051F484EF9AE00E945A1F882381F44F
:10F3A00082E08093F30A0CC08091F30A823041F42A
:10F3B00084EF9AE00E942921882311F41092F30A25
:10F3C0008091FF0A8823D1F08091FF0A813051F4A7
:10F3D00080E09BE00E945A1F882381F482E08093A2
:10F3E000FF0A0CC08091FF0A823041F480E09BE06C
:10F3F0000E942921882311F41092FF0A80910B0B9F
:10F400008823D1F080910B0B813051F48CE09BE08C
:10F410000E945A1F882381F482E080930B0B0CC05A
:10F4200080910B0B823041F48CE09BE00E942921FB
:10F43000882311F410920B0B8091170B8823D1F0C5
:10F440008091170B813051F488E19BE00E945A1F94
:10F45000882381F482E08093170B0CC08091170BF6
:10F46000823041F488E19BE00E942921882311F435
:10F470001092170BDF91CF910895CF93DF93CDB703
:10F48000DEB724970FB6F894DEBF0FBECDBF9A83C8
:10F49000898385E89AE00E942921882309F073C0B6
:10F4A000E981FA818091870A9091880AAA27BB276F
:10F4B00080839183A283B383A981BA81E0918C0A6E
:10F4C000F0918D0A8081FD018583A981BA818091A7
:10F4D0008C0A90918D0AFC0131968081FD01868312
:10F4E000A981BA8180918C0A90918D0AFC01329693
:10F4F0008081FD018783A981BA8180918C0A9091D6
:10F500008D0AFC0133968081FD018087A981BA8133
:10F5100080918C0A90918D0AFC0134968081FD01C6
:10F520008187A981BA8180918C0A90918D0AFC0112
:10F5300035968081FD018287A981BA8180918C0AEC
:10F5400090918D0AFC0136968081FD018387A98107
:10F55000BA8180918C0A90918D0AFC013796808146
:10F56000FD018487E981FA8180918B0A848385E893
:10F570009AE00E945A1F882309F0F9CF81E090E0B9
:10F580009C838B8352C480E99AE00E9429218823BE
:10F5900009F073C0E981FA818091920A9091930AEF
:10F5A000AA27BB2780839183A283B383A981BA81D1
:10F5B000E091970AF091980A8081FD018583A981E5
:10F5C000BA818091970A9091980AFC0131968081C6
:10F5D000FD018683A981BA818091970A9091980A4A
:10F5E000FC0132968081FD018783A981BA818091D7
:10F5F000970A9091980AFC0133968081FD018087DB
:10F60000A981BA818091970A9091980AFC01349659
:10F610008081FD018187A981BA818091970A9091AB
:10F62000980AFC0135968081FD018287A981BA8103
:10F630008091970A9091980AFC0136968081FD018D
:10F640008387A981BA818091970A9091980AFC01D9
:10F6500037968081FD018487E981FA818091960A3D
:10F66000848380E99AE00E945A1F882309F0F9CF29
:10F6700081E090E09C838B83D8C38BE99AE00E9461
:10F680002921882309F073C0E981FA8180919D0ABC
:10F6900090919E0AAA27BB2780839183A283B3837C
:10F6A000A981BA81E091A20AF091A30A8081FD01AB
:10F6B0008583A981BA818091A20A9091A30AFC0155
:10F6C00031968081FD018683A981BA818091A20A49
:10F6D0009091A30AFC0132968081FD018783A98164
:10F6E000BA818091A20A9091A30AFC01339680818D
:10F6F000FD018087A981BA818091A20A9091A30A15
:10F70000FC0134968081FD018187A981BA818091B5
:10F71000A20A9091A30AFC0135968081FD0182879F
:10F72000A981BA818091A20A9091A30AFC01369620
:10F730008081FD018387A981BA818091A20A90917D
:10F74000A30AFC0137968081FD018487E981FA8153
:10F750008091A10A84838BE99AE00E945A1F882332
:10F7600009F0F9CF81E090E09C838B835EC386EA49
:10F770009AE00E942921882309F073C0E981FA8167
:10F780008091A80A9091A90AAA27BB278083918318
:10F79000A283B383A981BA81E091AD0AF091AE0A48
:10F7A0008081FD018583A981BA818091AD0A909104
:10F7B000AE0AFC0131968081FD018683A981BA8160
:10F7C0008091AD0A9091AE0AFC0132968081FD01D4
:10F7D0008783A981BA818091AD0A9091AE0AFC011C
:10F7E00033968081FD018087A981BA818091AD0A1D
:10F7F0009091AE0AFC0134968081FD018187A98138
:10F80000BA818091AD0A9091AE0AFC013596808153
:10F81000FD018287A981BA818091AD0A9091AE0ADB
:10F82000FC0136968081FD018387A981BA81809190
:10F83000AD0A9091AE0AFC0137968081FD01848764
:10F84000E981FA818091AC0A848386EA9AE00E9479
:10F850005A1F882309F0F9CF81E090E09C838B83C5
:10F86000E4C281EB9AE00E942921882309F073C049
:10F87000E981FA818091B30A9091B40AAA27BB2743
:10F8800080839183A283B383A981BA81E091B80A6E
:10F89000F091B90A8081FD018583A981BA818091A7
:10F8A000B80A9091B90AFC0131968081FD018683E6
:10F8B000A981BA818091B80A9091B90AFC01329667
:10F8C0008081FD018783A981BA818091B80A9091D6
:10F8D000B90AFC0133968081FD018087A981BA8134
:10F8E0008091B80A9091B90AFC0134968081FD019B
:10F8F0008187A981BA818091B80A9091B90AFC01E7
:10F9000035968081FD018287A981BA818091B80AEC
:10F910009091B90AFC0136968081FD018387A98107
:10F92000BA818091B80A9091B90AFC01379680811A
:10F93000FD018487E981FA818091B70A848381EB94
:10F940009AE00E945A1F882309F0F9CF81E090E0E5
:10F950009C838B836AC28CEB9AE00E9429218823C6
:10F9600009F073C0E981FA818091BE0A9091BF0AC3
:10F97000AA27BB2780839183A283B383A981BA81FD
:10F98000E091C30AF091C40A8081FD018583A981B9
:10F99000BA818091C30A9091C40AFC01319680819A
:10F9A000FD018683A981BA818091C30A9091C40A1E
:10F9B000FC0132968081FD018783A981BA81809103
:10F9C000C30A9091C40AFC0133968081FD018087AF
:10F9D000A981BA818091C30A9091C40AFC0134962E
:10F9E0008081FD018187A981BA818091C30A9091AC
:10F9F000C40AFC0135968081FD018287A981BA8104
:10FA00008091C30A9091C40AFC0136968081FD0161
:10FA10008387A981BA818091C30A9091C40AFC01AD
:10FA200037968081FD018487E981FA818091C20A3D
:10FA300084838CEB9AE00E945A1F882309F0F9CF47
:10FA400081E090E09C838B83F0C187EC9AE00E9478
:10FA50002921882309F073C0E981FA818091C90ABC
:10FA60009091CA0AAA27BB2780839183A283B3837C
:10FA7000A981BA81E091CE0AF091CF0A8081FD017F
:10FA80008583A981BA818091CE0A9091CF0AFC0129
:10FA900031968081FD018683A981BA818091CE0A49
:10FAA0009091CF0AFC0132968081FD018783A98164
:10FAB000BA818091CE0A9091CF0AFC013396808161
:10FAC000FD018087A981BA818091CE0A9091CF0AE9
:10FAD000FC0134968081FD018187A981BA818091E2
:10FAE000CE0A9091CF0AFC0135968081FD01828774
:10FAF000A981BA818091CE0A9091CF0AFC013696F5
:10FB00008081FD018387A981BA818091CE0A90917D
:10FB1000CF0AFC0137968081FD018487E981FA8153
:10FB20008091CD0A848387EC9AE00E945A1F882333
:10FB300009F0F9CF81E090E09C838B8376C182ED60
:10FB40009AE00E942921882309F073C0E981FA8193
:10FB50008091D40A9091D50AAA27BB2780839183EC
:10FB6000A283B383A981BA81E091D90AF091DA0A1C
:10FB70008081FD018583A981BA818091D90A909104
:10FB8000DA0AFC0131968081FD018683A981BA8160
:10FB90008091D90A9091DA0AFC0132968081FD01A8
:10FBA0008783A981BA818091D90A9091DA0AFC01F0
:10FBB00033968081FD018087A981BA818091D90A1D
:10FBC0009091DA0AFC0134968081FD018187A98138
:10FBD000BA818091D90A9091DA0AFC013596808128
:10FBE000FD018287A981BA818091D90A9091DA0AB0
:10FBF000FC0136968081FD018387A981BA818091BD
:10FC0000D90A9091DA0AFC0137968081FD01848738
:10FC1000E981FA818091D80A848382ED9AE00E947A
:10FC20005A1F882309F0F9CF81E090E09C838B83F1
:10FC3000FCC08DED9AE00E942921882309F073C051
:10FC4000E981FA818091DF0A9091E00AAA27BB2717
:10FC500080839183A283B383A981BA81E091E40A6E
:10FC6000F091E50A8081FD018583A981BA818091A7
:10FC7000E40A9091E50AFC0131968081FD018683BA
:10FC8000A981BA818091E40A9091E50AFC0132963B
:10FC90008081FD018783A981BA818091E40A9091D6
:10FCA000E50AFC0133968081FD018087A981BA8134
:10FCB0008091E40A9091E50AFC0134968081FD016F
:10FCC0008187A981BA818091E40A9091E50AFC01BB
:10FCD00035968081FD018287A981BA818091E40AED
:10FCE0009091E50AFC0136968081FD018387A98108
:10FCF000BA818091E40A9091E50AFC0137968081EF
:10FD0000FD018487E981FA818091E30A84838DED86
:10FD10009AE00E945A1F882309F0F9CF81E090E011
:10FD20009C838B8382C088EE9AE00E9429218823DD
:10FD300009F073C0E981FA818091EA0A9091EB0A97
:10FD4000AA27BB2780839183A283B383A981BA8129
:10FD5000E091EF0AF091F00A8081FD018583A9818D
:10FD6000BA818091EF0A9091F00AFC01319680816E
:10FD7000FD018683A981BA818091EF0A9091F00AF2
:10FD8000FC0132968081FD018783A981BA8180912F
:10FD9000EF0A9091F00AFC0133968081FD01808783
:10FDA000A981BA818091EF0A9091F00AFC01349602
:10FDB0008081FD018187A981BA818091EF0A9091AC
:10FDC000F00AFC0135968081FD018287A981BA8104
:10FDD0008091EF0A9091F00AFC0136968081FD0136
:10FDE0008387A981BA818091EF0A9091F00AFC0182
:10FDF00037968081FD018487E981FA818091EE0A3E
:10FE0000848388EE9AE00E945A1F882309F0F9CF74
:10FE100081E090E09C838B8308C0E981FA811082A5
:10FE20001182128213821C821B828B819C812496F8
:10FE30000FB6F894DEBF0FBECDBFDF91CF9108950E
:10FE4000CF93DF93CDB7DEB722970FB6F894DEBF1E
:10FE50000FBECDBF9A8389838091F30A882339F43A
:10FE600083EF9AE09093240B8093230B21C0809121
:10FE7000FF0A882339F48FEF9AE09093240B809344
:10FE8000230B16C080910B0B882339F48BE09BE089
:10FE90009093240B8093230B0BC08091170B882326
:10FEA00009F08DC087E19BE09093240B8093230B96
:10FEB000E091230BF091240BA085B185E981FA81B3
:10FEC00085818C93E091230BF091240B80859185A3
:10FED000DC011196E981FA8186818C93E091230BF4
:10FEE000F091240B80859185DC011296E981FA81DD
:10FEF00087818C93E091230BF091240B8085918571
:10FF0000DC011396E981FA8180858C93E091230BC3
:10FF1000F091240B80859185DC011496E981FA81AA
:10FF200081858C93E091230BF091240B8085918542
:10FF3000DC011596E981FA8182858C93E091230B8F
:10FF4000F091240B80859185DC011696E981FA8178
:10FF500083858C93E091230BF091240B8085918510
:10FF6000DC011796E981FA8184858C93A091230B9B
:10FF7000B091240BE981FA818481FD018783A091EE
:10FF8000230BB091240BE981FA8180819181FD01DD
:10FF900094838383E091230BF091240B1286E091EC
:10FFA000230BF091240B1182E091230BF091240B91
:10FFB0001282E091230BF091240B81E08083229642
:10FFC0000FB6F894DEBF0FBECDBFDF91CF9108957D
:10FFD000CF93DF93CDB7DEB788E09AE00E943D7AF9
:10FFE000882309F430C088E09AE00E94561B88E01C
:10FFF0009AE00E943D7A882309F425C088E09AE0BF
:020000021000EC
:100000000E94561B88E09AE00E943D7A882309F4FA
:100010001AC088E09AE00E94561B88E09AE00E948D
:100020003D7A882309F40FC088E09AE00E94561BAD
:1000300088E09AE00E943D7A882309F404C088E0B1
:100040009AE00E94561BDF91CF910895CF93DF93E2
:10005000CDB7DEB761970FB6F894DEBF0FBECDBF48
:10006000198289818B3098F589819927FC01EB5D94
:10007000F44F80818C7F80839E012E5F3F4F89816A
:100080008F5FB9010E94DA6A89819927FC01EB5DD3
:10009000F44F89898170982F990F990F990F80815A
:1000A000877F892B808389819927FC01EB5DF44F41
:1000B00080818F70808389819927FC01EB5DF44FEB
:1000C00080818B7F808389818F5F8983CACF61968E
:1000D0000FB6F894DEBF0FBECDBFDF91CF9108956C
:1000E000CF93DF93CDB7DEB724970FB6F894DEBF7A
:1000F0000FBECDBF9A838983E981FA8180818370A5
:10010000282F33273C832B838B819C81009731F0F0
:100110002B813C812130310571F04EC0E981FA819B
:1001200080818F7080628083E981FA8180818C7FF9
:100130008160808341C0E981FA818081807F88234A
:10014000D9F5E981FA81808188708823F1F4E98109
:10015000FA8180818370823079F1E981FA8180812E
:100160008C7F82608083E981FA818081847088231A
:1001700031F0E981FA8180818B7F80831DC0E98124
:10018000FA8180818460808317C0E981FA8180814F
:100190008470882331F0E981FA8180818B7F8083AC
:1001A00005C0E981FA81808184608083E981FA81D8
:1001B00080818C7F8260808324960FB6F894DEBFA6
:1001C0000FBECDBFDF91CF910895CF93DF93CDB711
:1001D000DEB724970FB6F894DEBF0FBECDBF9A836B
:1001E0008983E981FA8180818370282F33273C83BA
:1001F0002B838B819C81813091056CF12B813C811B
:100200002330310534F08B819C818330910569F076
:1002100022C0E981FA8180818F7080628083E981C8
:10022000FA8180818360808316C0E981FA818081B0
:10023000807F882381F4E981FA8180818C7F8083AB
:10024000E981FA8180818870882329F0E981FA8127
:1002500080818B7F808324960FB6F894DEBF0FBE1B
:10026000CDBFDF91CF910895CF93DF93CDB7DEB7A8
:1002700025970FB6F894DEBF0FBECDBF8983898165
:10028000282F33273D832C838C819D81853C9105CC
:1002900009F499C02C813D81263C310524F58C81DF
:1002A0009D81823C910509F461C02C813D81233CF4
:1002B000310564F48C819D81803C9105C9F12C81CC
:1002C0003D81213C310509F442C0D4C08C819D811F
:1002D000833C910509F4A1C02C813D81243C31056A
:1002E00009F462C0C7C08C819D81813D910509F4EC
:1002F0004CC02C813D81223D31056CF48C819D8167
:10030000863C910509F46EC02C813D81273C310566
:1003100009F477C0AFC08C819D81823D910509F4BD
:100320008BC02C813D81233D310509F494C0A2C0CE
:1003300080912600992781709070009729F081E0C4
:1003400090E09B838A8398C01B821A8295C080911B
:100350002600992782709070009729F421E030E000
:100360003B832A8389C01B821A8286C08091260023
:10037000992784709070009729F481E090E09B8326
:100380008A837AC01B821A8277C0809129009927BC
:1003900082709070009729F421E030E03B832A833B
:1003A0006BC01B821A8268C08091260099278071D9
:1003B0009070009729F481E090E09B838A835CC071
:1003C0001B821A8259C080912600992780729070F2
:1003D000009729F421E030E03B832A834DC01B8243
:1003E0001A824AC0809126009927807490700097E5
:1003F00029F481E090E09B838A833EC01B821A82AD
:100400003BC08091260088232CF021E030E03B8324
:100410002A8332C01B821A822FC08091260099271E
:1004200088709070009729F481E090E09B838A8324
:1004300023C01B821A8220C08091290099278470D2
:100440009070009729F421E030E03B832A8314C0A8
:100450001B821A8211C080912900992788709070A0
:10046000009729F481E090E09B838A8305C01B827A
:100470001A8202C01B821A828A819B8125960FB63E
:10048000F894DEBF0FBECDBFDF91CF910895CF931B
:10049000DF93CDB7DEB723970FB6F894DEBF0FBE5C
:1004A000CDBF198289818B30F8F4898199278B5DC2
:1004B000944F9B838A83EA81FB818081807F88239C
:1004C00079F0AA81BB81EA81FB81808182958F705E
:1004D0008150982F9295907F8C918F70892B8C935F
:1004E00089818F5F8983DECF85E29BE09B838A834E
:1004F00080912600992781709070009729F08A8159
:100500009B810E94708004C08A819B810E94E5804B
:1005100086E29BE09B838A838091260099278270E4
:100520009070009729F48A819B810E94708004C09A
:100530008A819B810E94E58087E29BE09B838A837E
:1005400080912600992784709070009729F48A8101
:100550009B810E94708004C08A819B810E94E580FB
:1005600088E29BE09B838A8380912900992782708F
:100570009070009729F48A819B810E94708004C04A
:100580008A819B810E94E58089E29BE09B838A832C
:1005900080912600992780719070009729F48A81B4
:1005A0009B810E94708004C08A819B810E94E580AB
:1005B0008AE29BE09B838A83809126009927807240
:1005C0009070009729F48A819B810E94708004C0FA
:1005D0008A819B810E94E5808BE29BE09B838A83DA
:1005E00080912600992780749070009729F48A8161
:1005F0009B810E94708004C08A819B810E94E5805B
:100600008CE29BE09B838A838091260088232CF0D8
:100610008A819B810E94708004C08A819B810E9494
:10062000E5808DE29BE09B838A8380912600992759
:1006300088709070009729F48A819B810E94708055
:1006400004C08A819B810E94E5808EE29BE09B83AF
:100650008A8380912900992784709070009729F4EB
:100660008A819B810E94708004C08A819B810E9444
:10067000E5808FE29BE09B838A8380912900992704
:1006800088709070009729F48A819B810E94708005
:1006900004C08A819B810E94E58023960FB6F8945E
:1006A000DEBF0FBECDBFDF91CF910895CF93DF9313
:1006B000CDB7DEB725970FB6F894DEBF0FBECDBF1E
:1006C00089838981282F33273D832C838C819D81C9
:1006D000853C910509F479C02C813D81263C31058A
:1006E0001CF58C819D81823C910509F453C02C81BD
:1006F0003D81233C31055CF48C819D81803C9105DA
:10070000B9F12C813D81213C3105D9F194C08C8116
:100710009D81833C910509F473C02C813D81243C6B
:10072000310509F449C087C08C819D81813D9105C7
:10073000D1F12C813D81223D31056CF48C819D816C
:10074000863C910509F44AC02C813D81273C310546
:1007500009F44DC070C08C819D81823D910509F4E2
:1007600058C02C813D81233D310509F45BC063C035
:100770008091250B86958695817099279B838A8326
:100780005EC08091260B86958695817099279B8304
:100790008A8355C08091270B86958695817099270D
:1007A0009B838A834CC08091280B869586958170A7
:1007B00099279B838A8343C08091290B86958695D0
:1007C000817099279B838A833AC080912A0B8695F2
:1007D0008695817099279B838A8331C080912B0BEA
:1007E00086958695817099279B838A8328C08091FE
:1007F0002C0B86958695817099279B838A831FC0D1
:1008000080912D0B86958695817099279B838A838D
:1008100016C080912E0B86958695817099279B83B3
:100820008A830DC080912F0B8695869581709927BC
:100830009B838A8304C08EEF90E09B838A838A81A6
:100840009B8125960FB6F894DEBF0FBECDBFDF911A
:10085000CF910895CF93DF93CDB7DEB71092B60056
:1008600087E08093B0001092B2008EE48093B300D2
:1008700082E080937000DF91CF910895CF93DF9352
:10088000CDB7DEB70E942A841092320B1092330B40
:100890001092340B1092350B10923A0B10923B0BC6
:1008A0000E9426800E94F8070E94C661DF91CF91C6
:1008B0000895CF93DF93CDB7DEB721970FB6F894A5
:1008C000DEBF0FBECDBF89838091300B882311F02E
:1008D0001092300BA8950E94E87F8981823011F038
:1008E0000E94BE798981823009F472C08091310BF7
:1008F000882309F447C08091310B81508093310BDC
:100900000E94BD228091320B8F5F8093320B823028
:1009100040F01092320B0E9447820E944A240E94AB
:10092000EE098091330B8F5F8093330B843040F05E
:100930001092330B0E94D6240E9461A70E94CEA081
:100940008091340B8F5F8093340B8A3038F0109293
:10095000340B8981813011F00E943B1B8091350B53
:100960008F5F8093350B843168F01092350B809146
:100970003A0B8F5F80933A0B0E9422730E943427B8
:100980000E948D1A80913A0B8A3010F110923A0B26
:100990008091360B9091370BA091380BB091390BA9
:1009A0000196A11DB11D8093360B9093370BA09338
:1009B000380BB093390B0E94FC6380913B0B8F5F27
:1009C00080933B0B8C3320F010923B0B0E946E63A4
:1009D00021960FB6F894DEBF0FBECDBFDF91CF9149
:1009E0000895CF93DF93CDB7DEB78091360B90910A
:1009F000370BA091380BB091390BBC01CD01DF91C1
:100A0000CF9108951F920F920FB60F9211248F93DA
:100A1000CF93DF93CDB7DEB71092B20081E0809321
:100A2000300B8091310B8F5F8093310BDF91CF9131
:100A30008F910F900FBE0F901F901895CF93DF935B
:100A4000CDB7DEB70E94939E0E9466A160E076E972
:100A500080E090E00E949DA1DF91CF910895CF9317
:100A6000DF93CDB7DEB721970FB6F894DEBF0FBE88
:100A7000CDBF0E94A89E882339F00E94D79E89830B
:100A800089810E94559FF5CF21960FB6F894DEBF5D
:100A90000FBECDBFDF91CF910895CF93DF93CDB738
:100AA000DEB724970FB6F894DEBF0FBECDBF9A8392
:100AB00089836B831C828B8181508B838F3F59F09C
:100AC00089819A81FC013C812081232701969A83A8
:100AD00089832C83F0CF8C81992724960FB6F894C4
:100AE000DEBF0FBECDBFDF91CF9108950F931F934F
:100AF000CF93DF93CDB7DEB722970FB6F894DEBF62
:100B00000FBECDBF9A83898309811A81E981FA8159
:100B10008181282F215089819A810196622F0E941C
:100B20004D85F8018083E981FA8181819927BC0193
:100B300089819A810E94049F22960FB6F894DEBFA5
:100B40000FBECDBFDF91CF911F910F910895CF932D
:100B5000DF93CDB7DEB7C350D1400FB6F894DEBFF8
:100B60000FBECDBF9A838983E981FA818181282FC5
:100B7000215089819A810196622F0E944D858D8333
:100B8000E981FA8190818D81981711F00C941D9E56
:100B9000E981FA818281882309F0F9C1E981FA812A
:100BA0008381282F3327C250DF4F39832883CE5FBC
:100BB000D040C250DF4F88819981CE5FD0408135CF
:100BC000910509F475C0C250DF4FE881F981CE5F0D
:100BD000D040E235F105A4F4C250DF4F28813981BD
:100BE000CE5FD0402033310551F1C250DF4F8881B4
:100BF0009981CE5FD0408035910509F444C0C7C1CA
:100C0000C250DF4FE881F981CE5FD040E335F10576
:100C100009F4B8C0C250DF4F28813981CE5FD0407F
:100C2000233531050CF49AC0C250DF4F8881998179
:100C3000CE5FD0408435910509F427C1A8C1CE010B
:100C4000C39640E550E060E070E00E94E9BC85E1B9
:100C50008CAB1DAA80E88EABE981FA8184818FABD1
:100C60008FA9482F552789819A819C012B5F3F4F7F
:100C7000CE01C3960596B9010E94DCBCCE01C39695
:100C80000E94768584C1CE01C39640E550E060E0C5
:100C900070E00E94E9BC85E08CAB1DAA80EA8EABB7
:100CA0000E94A95F8FABCE01C3960E9476856FC16B
:100CB000E981FA8184818E83CE01C39640E550E0BC
:100CC00060E070E00E94E9BC89E18CAB1DAA81EA7A
:100CD0008EABCE018D579F4FBC018E810E94E75F86
:100CE0008E818FAB9E012D573F4FCE01C396059647
:100CF0004CE050E0B9010E94DCBCDE01AC5BBF4FB0
:100D0000FE01ED57FF4F848595858D939C93DE0101
:100D1000AA5BBF4FFE01ED57FF4F86858C93DE0126
:100D2000A95BBF4FFE01ED57FF4F87858C93FE01F6
:100D3000ED57FF4F8785482F5527CE018D579F4F81
:100D40009C01205F3F4FCE01C3964596B9010E949A
:100D5000DCBCCE01C3960E94768519C10E94375F24
:100D6000CE01C39640E550E060E070E00E94E9BC2F
:100D700084E08CAB1DAA82EA8EABCE01C3960E94A2
:100D8000768505C1DE01AD52BF4FE981FA818581CB
:100D9000968111969C938E93E981FA8184818C834C
:100DA0008C81813108F0F3C0CE01C39640E550E05C
:100DB00060E070E00E94E9BC87E18CAB1DAA83EA89
:100DC0008EABFE01ED52FF4F8081918199AF88AFCC
:100DD0008C818FABFE01EF50FF4FCE01C39607967B
:100DE00091838083DE01AD50BF4FFE01ED52FF4F76
:100DF000808191818D939C93FE01EB50FF4F8C81FC
:100E0000992791838083DE01A950BF4FFE01EB50EB
:100E1000FF4F808191818D939C939E0129503F4F7C
:100E2000F90180819181FE01ED50FF4FA081B181D8
:100E3000FE01EF50FF4F0190F081E02DCE5FDE4FBD
:100E4000F983E883C250D140CE5FDE4FE881F9815B
:100E5000C250D140019724F00E94C9BD0192FACF3F
:100E6000AF01F90191838083FE01ED50FF4FCD0169
:100E700091838083FE01EF50FF4FCA0191838083ED
:100E8000CE01C3960E94768582C0DE01AD52BF4F6F
:100E9000E981FA818581968111969C938E93E981EF
:100EA000FA8184818C838C81813108F070C0FE01CD
:100EB000E950FF4F89819A81079691838083DE01F3
:100EC000AB50BF4FFE01ED52FF4F808191818D935A
:100ED0009C93FE01ED50FF4F8C8199279183808375
:100EE000DE01AF50BF4FFE01ED50FF4F8081918179
:100EF0008D939C939E012F503F4FF90180819181EA
:100F0000FE01EB50FF4FA081B181FE01E950FF4F80
:100F10000190F081E02DCE5FDE4FF983E883C2506F
:100F2000D140CE5FDE4FE881F981C250D1400197B8
:100F300024F001900E94D1BDFACFAF01F901918355
:100F40008083FE01EB50FF4FCD0191838083FE0132
:100F5000E950FF4FCA0191838083CE01C39640E5DB
:100F600050E060E070E00E94E9BC87E08CAB1DAA15
:100F700084EA8EABFE01ED52FF4F8081918199AFE3
:100F800088AF8C818FABCE01C3960E947685E981B4
:100F9000FA818281813011F00C94269EE981FA81D8
:100FA0008381282F3327C050DF4F39832883C050D7
:100FB000D140C050DF4F88819981C050D1408035E9
:100FC000910509F461C7C050DF4FE881F981C05035
:100FD000D140E135F1050CF055C1C050DF4F2881FB
:100FE0003981C050D1402332310509F49DC5C0502C
:100FF000DF4F88819981C050D140843291050CF037
:101000009CC0C050DF4FE881F981C050D140E6302C
:10101000F10509F482C4C050DF4F28813981C050E6
:10102000D140273031050CF03FC0C050DF4F8881E0
:101030009981C050D1408330910509F4AEC3C050AE
:10104000DF4FE881F981C050D140E430F105B4F4BC
:10105000C050DF4F28813981C050D1402130310547
:1010600009F471C2C050DF4F88819981C050D140CE
:101070008230910509F4D3C20C940E9EC050DF4F0C
:10108000E881F981C050D140E430F10509F4B4C3DE
:10109000C050DF4F28813981C050D1402530310503
:1010A00009F416C40C940E9EC050DF4F88819981BC
:1010B000C050D1408930910509F48BC4C050DF4F36
:1010C000E881F981C050D140EA30F105B4F4C05054
:1010D000DF4F28813981C050D1402730310509F4D4
:1010E00063C4C050DF4F88819981C050D14088309F
:1010F000910509F45DC40C940E9EC050DF4FE88149
:10110000F981C050D140E132F10509F473C4C050F7
:10111000DF4F28813981C050D140223231050CF097
:1011200085C4C050DF4F88819981C050D140803242
:10113000910509F4D9C40C940E9EC050DF4FE8818C
:10114000F981C050D140EA32F10511F40C94CE94EB
:10115000C050DF4F28813981C050D1402B3231053A
:101160000CF043C0C050DF4F88819981C050D140FE
:101170008632910511F40C94CE92C050DF4FE88175
:10118000F981C050D140E732F105BCF4C050DF4FC7
:1011900028813981C050D1402432310509F4D6C4A8
:1011A000C050DF4F88819981C050D1408532910570
:1011B00011F40C942B920C940E9EC050DF4FE881DA
:1011C000F981C050D140E832F10511F40C94CE936E
:1011D000C050DF4F28813981C050D14029323105BC
:1011E00014F00C9420940C946B93C050DF4F8881C2
:1011F0009981C050D1408234910511F40C946295CC
:10120000C050DF4FE881F981C050D140E334F1058F
:10121000B4F4C050DF4F28813981C050D140203410
:10122000310509F4E3C4C050DF4F88819981C05073
:10123000D1408134910509F4ADC50C940E9EC05087
:10124000DF4FE881F981C050D140E434F10511F459
:101250000C94CF95C050DF4F28813981C050D140C8
:101260002434310514F40C949895C050DF4F8881D4
:101270009981C050D1408534910511F40C94F995B1
:101280000C940E9EC050DF4FE881F981C050D140D0
:10129000EE35F10511F40C94FC9CC050DF4F288111
:1012A0003981C050D1402F3531050CF0A7C0C05056
:1012B000DF4F88819981C050D1408635910511F466
:1012C0000C949A9CC050DF4FE881F981C050D14006
:1012D000E735F1050CF043C0C050DF4F288139815C
:1012E000C050D1402335310511F40C94E596C0501F
:1012F000DF4F88819981C050D14084359105BCF47D
:10130000C050DF4FE881F981C050D140E135F1058F
:1013100009F41EC7C050DF4F28813981C050D14029
:101320002235310511F40C9407960C940E9EC05092
:10133000DF4F88819981C050D1408435910511F4E7
:101340000C94BF97C050DF4FE881F981C050D14065
:10135000E535F10511F40C942C980C940E9EC050B8
:10136000DF4F28813981C050D1402935310511F432
:101370000C945F99C050DF4F88819981C050D14053
:101380008A359105C4F4C050DF4FE881F981C0501F
:10139000D140E735F10511F40C94AA9CC050DF4F01
:1013A00028813981C050D1402835310511F40C9481
:1013B00047990C940E9EC050DF4F88819981C05090
:1013C000D1408B35910511F40C94D09CC050DF4F67
:1013D000E881F981C050D140EB35F10514F40C944B
:1013E000BA9CC050DF4F28813981C050D1402C3584
:1013F000310511F40C94E89C0C940E9EC050DF4F04
:1014000088819981C050D1408536910511F40C94A2
:10141000E998C050DF4FE881F981C050D140E636ED
:10142000F1050CF041C0C050DF4F28813981C05018
:10143000D1402136310509F400C7C050DF4F888103
:101440009981C050D14082369105B4F4C050DF4F2D
:10145000E881F981C050D140EF35F10509F419C692
:10146000C050DF4F28813981C050D140203631052E
:1014700009F47CC60C940E9EC050DF4F8881998180
:10148000C050D1408336910511F40C94B09DC050EA
:10149000DF4FE881F981C050D140E436F10514F006
:1014A0000C948B980C94529DC050DF4F2881398149
:1014B000C050D1402836310511F40C941F9AC05009
:1014C000DF4F88819981C050D14089369105C4F49D
:1014D000C050DF4FE881F981C050D140E636F105B8
:1014E00011F40C947799C050DF4F28813981C05096
:1014F000D1402736310511F40C94FC990C940E9EC2
:10150000C050DF4F88819981C050D1408A36910503
:1015100011F40C94389BC050DF4FE881F981C05022
:10152000D140EA36F10514F40C94DA9AC050DF4F3A
:1015300028813981C050D1402B36310511F40C94EB
:10154000E99B0C940E9E0E94745CE981FA8184816F
:101550008E838E81833210F00C94269E8E81882398
:1015600011F40C94269E1B828B818F30B8F48B81F2
:10157000282F3327CE010196820F931FDC011E9680
:1015800029813A818B819927820F931FFC013A961A
:1015900080818C938B818F5F8B83E6CFE981FA8189
:1015A00085818F83E981FA8186818887E981FA8143
:1015B00087818987E981FA81838D948D9C878B87C8
:1015C000E981FA81858D8D87E981FA8180858E8711
:1015D000E981FA8181858A87E981FA81818D8E8FFF
:1015E000E981FA81828D8F8FCE0107966E810E94EC
:1015F0009269CE0107966E810E94CC451BAA85E0B8
:101600008CAB81E08DAB81E88EAB1FAACE01C39677
:101610000E94768581E00E9459840C94269EE9817F
:10162000FA8184818E838E81833208F053C08E814B
:10163000882309F44FC0CE0107966E810E94006A8C
:101640008EE18CAB81E08DAB82E88EAB8E818FAB6F
:101650008F8188AF888589AF89858AAF8A858CAF6D
:10166000FE01E25BFF4F8B859C8591838083FE01A9
:10167000E05BFF4F8D8580831B828B818F30C0F4B0
:101680008B81282F3327CE010196820F931FDC0117
:10169000DC968B81282F3327CE010196820F931F72
:1016A000FC013E9680818C938B818F5F8B83E5CF8D
:1016B0008E858BAFFE01E45BFF4F8E8D8083FE0134
:1016C000E35BFF4F8F8D8083CE01C3960E947685AA
:1016D0000C94269E8E818F3F11F00C94269E1C82C6
:1016E0008C81823210F00C94269E8C81282F2F5FE3
:1016F000CE010796622F0E94006A8EE18CAB81E0DA
:101700008DAB82E88EAB8C818F5F8FAB8F8188AF82
:10171000888589AF89858AAF8A858CAFFE01E25BB7
:10172000FF4F8B859C8591838083FE01E05BFF4F9B
:101730008D8580831B828B818F30C0F48B81282F15
:101740003327CE010196820F931FDC01DC968B813B
:10175000282F3327CE010196820F931FFC013E965E
:1017600080818C938B818F5F8B83E5CF8E858BAF50
:10177000FE01E45BFF4F8E8D8083FE01E35BFF4F34
:101780008F8D8083CE01C3960E94768581E00E9472
:1017900059848C818F5F8C83A3CF0E94745CE98114
:1017A000FA8184818E8389819A8105969E012D57C5
:1017B0003F4F4FE050E0BC01C9010E94DCBCDE019C
:1017C000AD57BF4FE981FA818489FD018787CE013A
:1017D0008D579F4FBC018E810E94816A81E08DAB45
:1017E00083E88EAB8E818FAB85E08CABCE01C39648
:1017F0000E9476850C94269EE981FA8184818E83ED
:101800008E818B3058F58E81882341F181E08DAB3C
:1018100084E88EAB8E818FABCE018D579F4FBC017C
:101820008E810E94DA6A9E012D573F4FCE01C396EA
:1018300005964FE050E0B9010E94DCBCDE01A95BD7
:10184000BF4FFE01ED57FF4F87858C9385E18CAB31
:10185000CE01C3960E9476850C94269E8E818F3F82
:1018600011F00C94269E1C828C818B3010F00C940D
:10187000269E81E08DAB84E88EAB8C818F5F8FAB31
:101880009E012D573F4F8C818F5FB9010E94DA6A0C
:101890009E012D573F4FCE01C39605964FE050E075
:1018A000B9010E94DCBCDE01A95BBF4FFE01ED5710
:1018B000FF4F87858C9385E18CABCE01C3960E9448
:1018C000768581E00E9459848C818F5F8C83CCCF98
:1018D000A8950E94745C0E94BD2BA8950E94B541FA
:1018E000A8950E94C543A8950E94B019A8950E948A
:1018F00028A7A8950E945D08A8950E94C1620E9431
:10190000CD1681E08DAB86E88EAB84E08CABCE014A
:10191000C3960E9476850C94269E84E18CAB81E070
:101920008DAB87E88EABCE01C39604964DE050E0B8
:1019300062E871E00E94DCBC0E94F184DC01CB0112
:10194000FE01E351FF4F80839183A283B3839E0105
:101950002C5B3F4FFE01E351FF4F80819181A281BB
:10196000B381CD01AA27BB27F90180839E012B5BA0
:101970003F4FFE01E351FF4F80819181A281B381EE
:10198000892F9A2FAB2FBB27F9018083DE01AA5B39
:10199000BF4FFE01E351FF4F80818C93CE01C39670
:1019A0000E9476850C94269E0C9400000C94269E32
:1019B00089819A8104960E94386781E08DAB89E81D
:1019C0008EAB84E08CABCE01C3960E9476850C94DE
:1019D000269E81E08DAB8AE88EAB8CE08CABCE018D
:1019E000C39604960E947167CE01C3960E947685C5
:1019F0000C94269ECE018D960E94D45681E08DAB2C
:101A000081EA8EAB8DA58FAB8EA588AF8FA589AFF0
:101A100088A98AAF89A98BAF8AA98CAF8AE08CABE1
:101A2000CE01C3960E9476850C94269EE981FA81A8
:101A300084818E838E81823210F5CE018896BC011E
:101A40008E810E945F5881E08DAB82EA8EAB8E81E1
:101A50008FAB89A589AF8AA58CAF88A588AF8BA5E8
:101A60009CA58070892F99278AAF8BA58BAF8AE0C0
:101A70008CABCE01C3960E9476850C94269E8E81F7
:101A80008F3F11F00C94269E1C828C81823210F0C4
:101A90000C94269E9E01285D3F4F8C818F5FB9017B
:101AA0000E945F5881E08DAB82EA8EAB8C818F5FA4
:101AB0008FAB89A589AF8AA58CAF88A588AF8BA588
:101AC0009CA58070892F99278AAF8BA58BAF8AE060
:101AD0008CABCE01C3960E94768581E00E9459842A
:101AE0008C818F5F8C83D1CFCE0180960E94505A1B
:101AF0008AE08CAB81E08DAB80EA8EAB8EA18FABA0
:101B00008CA188AF88A199A18070892F992789AF6E
:101B100088A18AAF8BA18BAF8AA18CAFCE01C3966F
:101B20000E9476850C94269EE981FA81648180E08A
:101B30000E94F24A84E08CAB81E08DAB83EA8EABED
:101B4000CE01C3960E9476850C94269EDE01AB5290
:101B5000BF4FE981FA8184818C93DE01AB52BF4F84
:101B6000E981FA818581FD018183DE01AB52BF4F9E
:101B7000E981FA818681FD018283DE01AB52BF4F8C
:101B8000E981FA818781FD018383DE01AB52BF4F7A
:101B9000E981FA818085FD018483DE01AB52BF4F6C
:101BA000E981FA818185FD018583DE01AB52BF4F5A
:101BB000E981FA818285FD018683DE01AB52BF4F48
:101BC000E981FA818385FD018783CE018B529F4F86
:101BD0000E94114B84E08CAB81E08DAB84EA8EAB2C
:101BE000CE01C3960E9476850C94269EFE01E95094
:101BF000FF4FCE018D579F4F91838083FE01EB50A5
:101C0000FF4F11821082FE01ED50FF4F80E190E006
